:020000040800F2
:10000000E819012041020008A5240008A7240008DF
:10001000AB240008AF240008B3240008000000004F
:10002000000000000000000000000000B7240008ED
:10003000B924000800000000BB240008BD2400080B
:100040005B0200085B0200085B0200085B0200081C
:100050005B0200085B0200085B0200085B0200080C
:100060005B0200085B0200085B0200085B020008FC
:100070005B0200085B0200085B0200085B020008EC
:100080005B0200085B0200085B0200085B020008DC
:100090005B0200085B0200085B0200085B020008CC
:1000A0005B0200085B0200085B0200085B020008BC
:1000B0005B020008D52800085B0200085B0200080C
:1000C0005B0200085B0200085B0200085B0200089C
:1000D0005B0200085B0200085B0200085B0200088C
:1000E0005B0200085B0200085B0200085B0200087C
:1000F0005B0200085B0200085B0200085B0200086C
:100100005B0200085B0200085B0200085B0200085B
:100110005B0200085B0200085B0200085B0200084B
:100120005B0200085B0200085B0200085B0200083B
:1001300000000000000000000000000000000000BF
:1001400000000000000000000000000000000000AF
:100150005B0200085B0200085B0200080000000070
:10016000000000000000000000000000000000008F
:10017000000000000000000000000000000000007F
:10018000000000000000000000000000000000006F
:10019000000000000000000000000000000000005F
:1001A000000000000000000000000000000000004F
:1001B000000000000000000000000000000000003F
:1001C000000000000000000000000000000000002F
:1001D000000000000000000000000000000000001F
:1001E000000000000000000000000000000000000F
:1001F00000000000000000000000000000000000FF
:1002000000000000000000000000000000000000EE
:1002100000000000000000000000000000000000DE
:10022000DFF810D022F0C6F800480047D5200008BB
:10023000AFF30080E81901200848804708480047CC
:100240000648804706480047FEE7FEE7FEE7FEE770
:10025000FEE7FEE7FEE7FEE7FEE7FEE79323000882
:100260002102000831490143314A1160704770B5DD
:10027000002100230F22C47804B32D4C246804F419
:10028000E064C4F5E064210AC1F10403CA40447883
:1002900004FA03F18478144021430901254C0678BF
:1002A000A155047804F01F050124AC4005786D11B8
:1002B000AD0005F1E025C5F8004109E0047804F03F
:1002C0001F050124AC401C4D0678761145F82640E8
:1002D00070BD1A4A0A400243154B1B1F1A60704733
:1002E00039B1134A121D12680243114B1B1D1A60CB
:1002F00006E00F4A121D126882430D4B1B1D1A6047
:100300007047042808D14FF0E021096941F0040149
:100310004FF0E022116107E04FF0E021096921F080
:1003200004014FF0E0221161704700000000FA055F
:100330000CED00E000E400E080E100E080FFFF1F42
:10034000F148006840F00100EF4908600846406845
:10035000EE490840EC49486008460068EC4908400E
:10036000E94908600846006820F4802008600846D3
:10037000406820F4FE0048604FF41F00886070471A
:10038000E149096821F48031DF4A116011460968AA
:1003900021F480211160B0F5803F03D0B0F5802FAB
:1003A0000ED106E0D849096841F48031D64A11607F
:1003B00007E0D549096841F4A021D34A116000E063
:1003C00000BF00BF704710B5014600220023002087
:1003D0004A11012A02D1CC4C236806E0022A02D13C
:1003E000C94C236A01E0C84C636A01F01F02012472
:1003F00094401C400CB1012000E0002010BD38B535
:10040000002000900024002500BF3120FFF7DBFF13
:1004100005460098401C00900098B0F5706F01D020
:10042000002DF2D03120FFF7CEFF08B1012400E00B
:100430000024204638BD01460020B34A106820F051
:10044000F80040EAC10010607047B2490860704788
:1004500002460020AC4B586820F47C1042EA0103AD
:100460001843A94B58607047AA490866704701466F
:100470000020A54A506820F00300084350607047F0
:10048000A148406800F00C007047014600209E4AD9
:10049000506820F0F000084350607047014600208B
:1004A000994A506820F4E060084350607047014664
:1004B0000020954A506820F4605040EAC100506026
:1004C000704729B1904A527A02438F4B5A7204E026
:1004D0008D4A527A82438C4B5A7270478A494968D6
:1004E0008D4A1140884A5160114649680143516064
:1004F000704701460020844A5068884A10400843EB
:10050000814A5060704700217F4A203211707E4A34
:1005100082F82010012802D004280AD104E0012129
:10052000794A2032117005E00521774A2032117096
:1005300000E000BF00BF704779490860704772490A
:10054000096A0143704A116270477549443908606D
:100550007047F0B500210022002500236A4E76681E
:1005600006F00C0121B1042905D008292ED105E09F
:100570006C4E06602DE06B4E06602AE0624E766897
:1005800006F47012604E766806F480355E4E76682A
:10059000C6F300762EB10124260146EA9246721C6B
:1005A00002E0022606EB92421DB95F4E56430660FA
:1005B0000BE0554E766806F400361EB15A4E56438F
:1005C000066002E0574E5643066002E0554E066054
:1005D00000BF00BF4C4E766806F0F0010909534E8B
:1005E000735C0668DE404660474E766806F4E0615C
:1005F000090A4E4E735C4668DE408660424E76685D
:1006000006F46051C90A494E735C4668DE40C66014
:100610003D4E7668414FFF4306EA07010C2606EA85
:10062000D166C1F3813746EA0701414E735CC66863
:10063000B6FBF3F60661F0BD29B1334A52690243B5
:10064000314B5A6104E0304A526982432E4B5A6161
:10065000704729B12C4A926902432B4B9A6104E0FE
:10066000294A92698243284B9A61704729B1264AE8
:10067000D2690243244BDA6104E0234AD2698243FF
:10068000214BDA61704729B11F4AD26802431E4BE1
:10069000DA6004E01C4AD26882431B4BDA60704780
:1006A00029B1194A12690243174B1A6104E0164A2C
:1006B00012698243144B1A61704719494039086026
:1006C00070471449C8647047072802DC0E49C87196
:1006D00002E007210C4AD171811F0B4A1163704758
:1006E0000948406A40F080700749486270470146F7
:1006F0000020054A92680A400AB1012000E000206B
:100700007047014988727047001002400000FFF8EE
:10071000FFFFF6FE00004242FFFF3F7FFF3FFF9FCB
:100720008004424200127A0000093D0000000020CF
:100730001000002010B50446E248844208D101218F
:100740000420FFF7A0FF00210420FFF79CFF46E0F4
:10075000DD48844208D101210820FFF794FF0021E1
:100760000820FFF790FF3AE0D848844208D10121E1
:100770001020FFF788FF00211020FFF784FF2EE0F4
:10078000D348844208D101212020FFF77CFF0021BB
:100790002020FFF778FF22E0CE48844208D10121D3
:1007A0004020FFF770FF00214020FFF76CFF16E0AC
:1007B000C948844208D101218020FFF764FF00214D
:1007C0008020FFF760FF0AE0C448844207D101217E
:1007D0008015FFF758FF0021A015FFF754FF10BD4B
:1007E00010B501210846FFF74EFF00210120FFF759
:1007F0004AFF10BD2DE9F0410246002500260020E9
:1008000000230024002791F803C00CF00F0591F895
:1008100003C00CF0100CBCF1000F03D091F802C023
:100820004CEA050591F800C0BCF1000F31D0146806
:1008300000202BE04FF0010C0CFA00F3B1F800C0DF
:100840000CEA03069E4220D183004FF00F0C0CFAF5
:1008500003F7BC4305FA03FC4CEA040491F803C017
:10086000BCF1280F06D14FF0010C0CFA00FCC2F8C5
:1008700014C00AE091F803C0BCF1480F05D14FF055
:10088000010C0CFA00FCC2F810C0401C0828D1D39F
:100890001460B1F800C0BCF1FF0F34DD54680020D3
:1008A0002EE000F1080C4FF0010808FA0CF3B1F843
:1008B00000C00CEA03069E4221D183004FF00F0CCA
:1008C0000CFA03F7BC4305FA03FC4CEA040491F864
:1008D00003C0BCF1280F05D100F1080C08FA0CF890
:1008E000C2F8148091F803C0BCF1480F07D100F1A1
:1008F000080C4FF0010808FA0CF8C2F81080401CF0
:100900000828CED35460BDE8F0814FF6FF71018016
:10091000022181700421C170704702460020936853
:100920000B400BB1012000E00020704701468868B1
:1009300080B2704702460020D3680B400BB1012003
:1009400000E0002070470146C86880B2704701612E
:100950007047416170470AB1016100E04161704731
:10096000C16070474FF480320A43826181618261C5
:1009700082698269704702460020594B18684FF619
:100980008073184040EA02100843554B18607047C6
:100990005449C8617047F0B50A460023002400217D
:1009A000002500F00046B6F1004F02D14C4EF1692F
:1009B00001E04B4E7168C0F3034583B200F440166A
:1009C000B6F5401F08D121F07061454E766826F0DB
:1009D0007066434F7E6012E000F48016B6F5801F0B
:1009E00006D1032606FA05F4A14341F0706106E042
:1009F000460D360103FA06F6B14341F0706122B1AB
:100A0000460D360103FA06F6314300F00046B6F112
:100A1000004F02D1324EF16101E0314E7160F0BD04
:100A2000B0F1804F01D1012200E00022B0F1004F6F
:100A300001D1012300E000231A434AB1284AD269B8
:100A400022F04042264BDA611A46D2690243DA614B
:100A5000704730B500228B071C0F0F2303FA04F2F6
:100A60001F4B08338C1053F8243093431C4C08342C
:100A70008D1044F8253023468C1053F824308C0711
:100A8000240F00FA04F42343154C08348D1044F865
:100A9000253030BD1349DC310860704719B14FF083
:100AA000A532426302E04FF0FF3242637047026BAF
:100AB0000A4302637047026B4FF480338B401A4342
:100AC0000263704700080140000C01400010014023
:100AD0000014014000180140001C014000200140AA
:100AE000000001400000204210B50446F74884424F
:100AF00009D101218803FFF7C6FD00214FF4804092
:100B0000FFF7C1FD32E0F248844209D101214804D7
:100B1000FFF7C6FD00214FF40030FFF7C1FD25E0CF
:100B2000EC48844209D101218804FFF7B9FD002176
:100B30004FF48020FFF7B4FD18E0E748844209D164
:100B40000121C804FFF7ACFD00214FF40020FFF79E
:100B5000A7FD0BE0E148844208D101210805FFF719
:100B60009FFD00214FF48010FFF79AFD10BD2DE985
:100B7000F04786B005460E460024A24600BFA146B7
:100B80000027B08900B100BF2F462C8A4CF6FF70B9
:100B90000440F08804432C82AC894EF6F3100440E4
:100BA000B08831890843718908430443AC81AC8A19
:100BB0004FF6FF400440B0890443AC8201A8FFF720
:100BC000C8FCC248874204D164210498B0FBF1FA02
:100BD00003E064210398B0FBF1FAA88900F4004017
:100BE00058B164213068B0FBF1F040000AEBCA0153
:100BF00001EB0A11B1FBF0F80AE064213068B0FBA8
:100C0000F1F080000AEBCA0101EB0A11B1FBF0F828
:100C10006420B8FBF0F004012009642101FB108975
:100C2000A88900F4004040B1322000EBC900B0FBBD
:100C3000F1F000F00700044308E0322000EB091057
:100C40006421B0FBF1F000F00F0004432C8106B0EA
:100C5000BDE8F0874FF41651016000218180C1800A
:100C600001810C21418100218181704710B502462C
:100C70000020108A4FF2FF0318400B884C88234352
:100C80008C882343CC8823431843108210BD002155
:100C9000018041808180C180704721B1828942F406
:100CA0000052828104E082894DF6FF731A408281EE
:100CB0007047F0B50346002400260025002040F6CA
:100CC0006A17B94200D100BF1846C1F3421401F0BF
:100CD0001F06012707FA06F5012C01D10C3004E0AC
:100CE000022C01D1103000E014301AB107682F43F4
:100CF000076002E00768AF430760F0BD1AB1838A5E
:100D00000B43838202E0838A8B4383827047028A8B
:100D10004FF6F0731A400282028A0A430282704739
:100D200082894FF2FF731A40828182890A4382814D
:100D3000704721B1828942F00202828104E08289F7
:100D40004FF6FD731A4082817047028A4FF6DF73B7
:100D50001A400282028A0A430282704721B1028A43
:100D600042F48042028204E0028A4BF6FF731A408A
:100D700002827047C1F3080282807047014688886A
:100D8000C0F308007047818941F0010181817047FB
:100D9000028BD2B20283028B42EA012202837047A5
:100DA000028B02F47F420283028B0A430283704764
:100DB00021B1828A42F02002828204E0828A4FF6C8
:100DC000DF731A408282704721B1828A42F010029A
:100DD000828204E0828A4FF6EF731A408282704763
:100DE00021B1828A42F00802828204E0828A4FF6B0
:100DF000F7731A408282704721B1828942F400421F
:100E0000828103E08289C2F30E028281704721B1A0
:100E1000828A42F40062828204E0828A4FF2FF7387
:100E20001A4082827047828A4FF6FB731A40828290
:100E3000828A0A438282704721B1828A42F002028A
:100E4000828204E0828A4FF6FD731A4082827047E4
:100E500002460020B1F5007F00D100BF13880B408F
:100E60000BB1012000E00020704701F40072B2F5E0
:100E7000007F00D100BFCA430280704770B50246B0
:100E8000002400230025002040F66A16B14200D15C
:100E900000BFC1F3421501F01F03012606FA03F358
:100EA000012D02D19689334006E0022D02D1168A27
:100EB000334001E0968A33400C12012606FA04F40E
:100EC0001688344063B15CB101200AE0003801406B
:100ED0000044004000480040004C004000500040EA
:100EE000002070BD10B50022002340F66A14A14214
:100EF00000D100BF0A1201249440A3B2DC43048055
:100F000010BD000010B50446BE48844208D101213E
:100F10008014FFF7B8FB0021A014FFF7B4FB16E024
:100F2000B948844208D101210014FFF7B9FB002120
:100F30002014FFF7B5FB0AE0B448844207D1012131
:100F4000C013FFF7ADFB0021E013FFF7A9FB10BDB5
:100F500010B50022028802F441520B884C882343CA
:100F60008C882343CC8823430C8923434C89234317
:100F70008C892343CC8923431A430280838B4FF20D
:100F8000FF74234083830B8A038210BD2DE9F04F49
:100F900085B005460C464FF0000902274FF00008C7
:100FA0004FF0010B0026B246A88B4FF240010840DB
:100FB000A88302202884B5F81C90A068022801D1DB
:100FC00000BF38E0A08810B94FF0010B01E04FF0EE
:100FD000020B8D48854200D100E000BF6846FFF754
:100FE000B8FADDF800A0E088B0F5007F0AD14FEA3A
:100FF0001A2000EB80004000A168B0FBF1F0401D1A
:1010000086B20BE04FEA4B10BAFBF0F000EB800029
:101010004000A168B0FBF1F0401D86B20A20B6FB8B
:10102000F0F606F00108A6EB0800C0F34F074FF6F4
:10103000FF7000EA0828022F01DBFF2F02DD0227E4
:101040004FF00008E08840EA080038432884A08870
:10105000A1890843618808432188084340F400605F
:1010600040EA0909A5F81C9005B0BDE8F08F002101
:10107000018041808180C180018141818181C18164
:101080000721018270470021018041808180C18059
:101090000221816000218181704721B1028842F0E4
:1010A0004002028004E002884FF6BF731A400280BB
:1010B000704721B1828B42F48062828304E0828B8C
:1010C0004FF6FF331A408283704730B50024002367
:1010D0000C110125A540ABB21AB185881D4385804E
:1010E00002E085889D43858030BD1AB183880B431B
:1010F000838002E083888B438380704781817047BF
:101100000146888970474FF6FF62914204D00288F9
:1011100042F48072028004E002884FF6FF631A40B6
:101120000280704721B1828842F00402828004E08C
:1011300082884FF6FB731A408280704702884FF214
:10114000FF731A40028002880A43028070470188B8
:1011500041F480510180704721B1028842F400526D
:10116000028004E002884DF6FF731A400280704747
:1011700002460020012901D0108B00E0908A7047C0
:101180000146088A7047B1F5804F04D1028842F4C5
:101190008042028004E002884BF6FF731A4002800E
:1011A00070470246002013890B400BB1012000E07C
:1011B00000207047CA4302817047F0B50246002004
:1011C00000240023002501F00F070126BE40B4B221
:1011D0000B1101269E40B3B2968806EA03051689D4
:1011E000264016B10DB1012000E00020F0BD10B581
:1011F000002201F00F040123A3409AB2D3430381DC
:1012000010BD00000030014000380040003C0040AC
:1012100010B50446FA48844208D10121C014FFF7F2
:1012200032FA0021E014FFF72EFA9DE0B4F1804F6E
:1012300008D101210846FFF733FA00210120FFF70A
:101240002FFA91E0EF48844208D101210220FFF7F4
:1012500027FA00210220FFF723FA85E0EA488442BA
:1012600008D101210420FFF71BFA00210420FFF719
:1012700017FA79E0E548844208D101210820FFF7F8
:101280000FFA00210820FFF70BFA6DE0E0488442D6
:1012900008D101211020FFF703FA00211020FFF7E9
:1012A000FFF961E0DB48844208D101212020FFF7EB
:1012B000F7F900212020FFF7F3F955E0D6488442E2
:1012C00008D101214014FFF7DEF900216014FFF777
:1012D000DAF949E0D148844209D10121C804FFF775
:1012E000D2F900214FF40020FFF7CDF93CE0CC48C3
:1012F000844209D101210805FFF7C5F900214FF407
:101300008010FFF7C0F92FE0C648844209D10121BF
:101310004805FFF7B8F900214FF40010FFF7B3F9C3
:1013200022E0C148844208D101214020FFF7B8F9EA
:1013300000214020FFF7B4F916E0BC48844208D1F0
:1013400001218020FFF7ACF900218020FFF7A8F9E8
:101350000AE0B748844207D101218015FFF7A0F9C0
:101360000021A015FFF79CF910BD00220288A44BB4
:1013700098420ED0A84B98420BD0B0F1804F08D0C5
:10138000A04B984205D0A04B984202D09F4B984268
:1013900004D14FF68F731A404B881A439C4B9842E6
:1013A00007D09C4B984204D04FF6FF431A40CB889D
:1013B0001A4302808B8883850B880385904B984263
:1013C00002D0954B984201D10B7A03860123838288
:1013D000704770B5002400220023058C4FF6FE767E
:1013E00035400584028C8388048B4FF68F752C4022
:1013F000B51E2C400D882C43751E2A400D892A43AA
:101400004D882A437E4DA84202D0834DA84213D175
:101410004FF6F7752A404D892A434FF6FB752A404F
:101420008D882A434FF6FF652B404FF6FF552B4022
:101430008D892B43CD892B4383800483CD8885867A
:10144000028470BD70B5002400220023058C4FF685
:10145000EF7635400584028C8388048B48F6FF754F
:101460002C404FF6FF452C400D884FF6FF7606EADC
:1014700005252C434FF6DF752A400D8906EA051530
:101480002A434D8806EA05152A435D4DA84202D03D
:10149000614DA8421DD14FF67F752A404D894FF608
:1014A000FF7606EA05152A434FF6BF752A408D8858
:1014B00006EA05152A434FF6FF352B404FF2FF751C
:1014C0002B408D8906EA85052B43CD8906EA8505E3
:1014D0002B4383800483CD880587028470BD70B55B
:1014E000002400220023058C4FF6FF66354005845A
:1014F000028C8388848B4FF68F752C404FF6FC75D9
:101500002C400D882C434FF6FF552A400D894FF68D
:10151000FF7606EA05252A434D8806EA05252A4373
:10152000374DA84202D03C4DA8421DD14FF2FF7565
:101530002A404D894FF6FF7606EA05252A434FF6E5
:10154000FF352A408D8806EA05252A434EF6FF75A9
:101550002B404DF6FF752B408D8906EA05152B4370
:10156000CD8906EA05152B4383808483CD88858742
:10157000028470BD70B5002200230024058C4EF655
:10158000FF7635400584038C8488828B48F6FF758E
:101590002A404FF6FF452A400D884FF6FF7606EAAF
:1015A00005252A434DF6FF752B400D8906EA0535C2
:1015B0002B434D8806EA05352B43114DA84202D036
:1015C000154DA84208D14BF6FF752C408D894FF67A
:1015D000FF7606EA85152C4384808283CD88A0F8A7
:1015E0004050038470BD828B4FF2FF331A408283D8
:1015F000828B4FF6FF7303EA01231A4382837047FD
:10160000002C01400004004000080040000C004095
:10161000001000400014004000340140004C014024
:10162000005001400054014000180040001C0040E0
:1016300000200040F0B50C4615460022002100268F
:10164000078C4EF6FF7C07EA0C070784828B018C1F
:101650004FF6FF7707EA043640F6FF473A404FF669
:10166000FF7707EA05273A434FF6FF7707EA033784
:101670003A43F64FB8420ED0F54FB8420BD0B0F116
:10168000804F08D0F34FB84205D0F34FB84202D094
:10169000F24FB84206D14DF6FF77394046F48057F5
:1016A000394305E047F6FF57394044F48057394342
:1016B00082830184F0BD828B4FF6F3731A408283DC
:1016C000828B0A4382837047F0B50C461546002290
:1016D00000210026078C4FF6FF6C07EA0C070784F1
:1016E000828B018C4FF6FF7707EA04264FF60C77C2
:1016F0003A404FF6FF7707EA03172F433A43D34F99
:10170000B8420ED0D24FB8420BD0B0F1804F08D0C3
:10171000D04FB84205D0D04FB84202D0CF4FB842D8
:1017200006D14FF6FF57394046F48077394305E03C
:101730004FF2FF57394044F4807739438283018464
:10174000F0BD028B4FF2FF331A400283028B4FF63B
:10175000FF7303EA01231A4302837047F0B50C4676
:101760001546002200210026078C4FF6EF7C07EA81
:101770000C070784028B018C4FF6FF7707EA0416EB
:1017800040F6FF473A404FF6FF7707EA03373A4300
:101790004FF6FF7707EA05273A43AC4FB8420ED021
:1017A000AB4FB8420BD0B0F1804F08D0A94FB84230
:1017B00005D0A94FB84202D0A84FB84206D14FF683
:1017C000DF77394046F01007394305E04FF65F7781
:1017D000394044F01007394302830184F0BD028B85
:1017E0004FF6F3731A400283028B0A430283704759
:1017F000F0B50C46154600220021068C4FF6FE7708
:101800003E400684028B018C4FF60C7632407E1CE3
:1018100006EA03162E4332438C4EB0420ED08C4E55
:10182000B0420BD0B0F1804F08D08A4EB04205D004
:10183000894EB04202D0894EB04206D14FF6FD76B5
:10184000314044F00106314305E04FF6F576314072
:1018500044F00106314302830184F0BD70B50546B2
:101860000C467A4885420ED0794885420BD0B5F1B6
:10187000804F08D07748854205D07748854202D00E
:101880007648854200D100E000BF208850B9238906
:10189000A28861882846FFF7ABFFE1882846FFF75A
:1018A0009EFF25E0208804280AD12389A288618828
:1018B0002846FFF753FFE1882846FFF742FF17E06D
:1018C000208808280AD12389A28861882846FFF742
:1018D000FBFEE1882846FFF7EEFE09E02389A28897
:1018E00061882846FFF7A6FEE1882846FFF77BFEC1
:1018F00070BD2DE9F04105460C46002601276088A1
:1019000008B9022600E00026A088012801D102279C
:1019100000E001272088A0B92389A2886188284691
:10192000FFF766FFE1882846FFF759FF23893A460B
:1019300031462846FFF712FFE1882846FFF701FFEE
:1019400013E02389A28861882846FFF707FFE18812
:101950002846FFF7F6FE23893A4631462846FFF728
:1019600047FFE1882846FFF73AFFBDE8F0810A8883
:101970004B881A438B881A43CB881A430B891A4326
:101980004B891A438B891A43A0F8442070474FF6BD
:10199000FF71818000210180C18041800172704708
:1019A0000021018041808180C1800181418181814C
:1019B000C181704700210180418001218180002187
:1019C000C180018170470021018041808180C180F8
:1019D000018141818181704721B1028842F0010279
:1019E000028004E002884FF6FE731A4002807047BE
:1019F00031B1B0F8442042F40042A0F8442005E0A0
:101A0000B0F84420C2F30E02A0F8442070471AB187
:101A100083890B43838102E083898B4383817047F1
:101A20008182704741EA0203A0F8483070471AB13A
:101A300083890B43838102E083898B4383817047D1
:101A400001894FF6F872114001817047002C014066
:101A5000003401400004004000080040000C004039
:101A60000A46002101894FF68F7319401143018105
:101A7000704730B504460D4629462046FFF7F0FF73
:101A8000208940F00700208130BD2DE9F041044657
:101A90000D4616461F46602D06D13B4601223146B3
:101AA0002046FFF75BFE05E03B460122314620461B
:101AB000FFF79EFE29462046FFF7D2FF208940F01F
:101AC00007002081BDE8F08130B50C460021018976
:101AD000C9B24FF6FF7505EA03251543254329438F
:101AE000018130BD2DE9F04105460E461746984666
:101AF000002443463A4631462846FFF7E5FF2C8945
:101B00004FF6F870044044F007044FF68F7004401D
:101B100044F070042C81BDE8F081F0B504460D4618
:101B200016461F463B46324629462046FFF7CCFF65
:101B3000208940F480402081F0BD01858282704779
:101B40000A46002101884FF68F7319401143018026
:101B50007047F0B50C4615461E46002100220023B2
:101B60000189028B038C4FF6F877394021434FF6F9
:101B7000FC473A4040F201173A434FF6DD773B40CD
:101B80004FF6FF7707EA06172F433B430181028395
:101B90000384F0BD0A460021018B4FF68F73194074
:101BA0001143018370470A460021018B48F6FF73F9
:101BB00019404FF6FF7303EA02231943018370476C
:101BC0000A460021818B4FF68F73194011438183A0
:101BD00070470A460021818B48F6FF7319404FF683
:101BE000FF7303EA022319438183704721B10288FE
:101BF00042F08002028004E002884FF67F731A40B0
:101C00000280704721B1828842F00402828004E0A1
:101C100082884FF6FB731A408280704721B1828818
:101C200042F00802828004E082884FF6F7731A407F
:101C30008280704721B1828842F00102828004E0F4
:101C400082884FF6FE731A40828070470A46002150
:101C5000018B4FF6F77319401143018370470A4611
:101C60000021018B4FF2FF7319404FF6FF7303EA17
:101C700002231943018370470A460021818B4FF6E6
:101C8000F77319401143818370470A460021818B05
:101C90004FF2FF7319404FF6FF7303EA0223194313
:101CA000818370470A460021018B4FF6FB73194070
:101CB0001143018370470A460021018B4FF6FF3321
:101CC00019404FF6FF7303EA02231943018370475B
:101CD0000A460021818B4FF6FB7319401143818323
:101CE00070470A460021818B4FF6FF3319404FF6AB
:101CF000FF7303EA02231943818370470A460021D8
:101D0000018B4FF67F7319401143018370470A46D8
:101D10000021018BC1F30E014FF6FF7303EA02238A
:101D20001943018370470A460021818B4FF67F7368
:101D300019401143818370470A460021818BC1F30A
:101D40000E014FF6FF7303EA0223194381837047A4
:101D50000A460021018C4FF6FD731940114301849E
:101D600070470A460021018C4FF6F7731940114362
:101D7000018470470A460021018C4FF6DF73194039
:101D80004FF6FF7303EA02131943018470470A46B2
:101D90000021018C4FF67F7319404FF6FF7303EA61
:101DA00002131943018470470A460021018C4FF643
:101DB000FF5319404FF6FF7303EA022319430184CE
:101DC00070470A460021018C4FF2FF7319404FF60D
:101DD000FF7303EA02231943018470470A46002176
:101DE000018C4DF6FF7319404FF6FF7303EA02337F
:101DF00019430184704730B5002301248C40A3B2FD
:101E0000048C9C430484048C02FA01F5ADB22C438B
:101E1000048430BD30B5002304248C40A3B2048C6C
:101E20009C430484048C02FA01F5ADB22C43048473
:101E300030BD70B503460020002418461830012537
:101E40008D40ACB21D8CA5431D8409B1082909D170
:101E500000EB6100056825F0700505600568154315
:101E600005600EE00D1FC5F34E052844056825F4F6
:101E7000E045056005684FF6FF7606EA0226354321
:101E8000056070BD21B1028842F00202028004E0C8
:101E900002884FF6FD731A400280704721B1028814
:101EA00042F00402028004E002884FF6FB731A40FD
:101EB0000280704721B1828842F08002828004E073
:101EC00082884FF67F731A408280704702884FF6EF
:101ED000F7731A40028002880A43028070478288A2
:101EE0004FF68F731A40828082880A43828070473F
:101EF00002894FF6F8731A40028102890A4302816F
:101F0000704702894FF67F731A40028102890A43A3
:101F10000281704781847047818570478186704750
:101F20000187704781877047A0F84010704702888A
:101F30004FF6FF431A40028002880A43028070472E
:101F40000146888E70470146088F70470146888F8A
:101F500070470146B1F8400070470146888C7047D1
:101F60000146088D704702460020138A0B400BB1D2
:101F7000012000E000207047CA430282704730B55C
:101F80000246002000230024158A05EA01039589F2
:101F900005EA010413B10CB1012000E0002030BDBE
:101FA000CA4302827047000001460120454A126878
:101FB00002F0010282B1434A121D12680A60414ACE
:101FC000121D12684A603F4A121D12688A603D4A1B
:101FD000121D1268CA60002070473A49103108602B
:101FE000704740B137490C31096841F08051354A9A
:101FF0000C32116007E033490C31096821F080513F
:10200000304A0C32116070472E490C31096821F4B6
:10201000704141EA00312B4A0C321160704730B1F7
:102020002849096841F01001264A116005E0254958
:10203000096821F01001234A1160704701462148C8
:102040000068084008B1012070470020FCE71D49E6
:10205000096881431B4A116070471A480C300068B8
:1020600020F4704017490C3108601648006820F0D1
:10207000010014490860704712480C30006840F4B1
:10208000704010490C310860704770B101210E4A50
:1020900011600E490E4A11600D49CC31096841F0BA
:1020A00001010B4ACC3211600AE00021064A11609E
:1020B0000749CC31096821F00101054ACC32116091
:1020C0007047000000080650F01002402635EDCDA4
:1020D000006C01401CB5002500F008FD00F074FC08
:1020E0004FF4E13000F020FC39A020F07FFF012008
:1020F0003D4908603D483E49086007203C49CC31D5
:1021000008600120FFF7C1FF00F0ACFB20F0CAFD22
:1021100000F0F1F93749384800F0B1FA20F07EFCC0
:102120000446E0B2210EC4F30723C4F30742009033
:10213000324820F05BFF32A020F058FF41F2883295
:1021400001213A481DF0A9FA002000900346384AC0
:102150004FF4FA61019035481DF03EF93349087893
:1021600040F2BB12324900F057FE40F2BB12304938
:102170002E481DF09EFA2FA020F038FF39A020F045
:1021800035FF2A49C868C82115F00CFE40491A4895
:1021900020F056FF18481FF015FF06463246164934
:1021A00022481DF066FC12E040F2FF7212491F48FF
:1021B0001DF055FC0546002D09DD294635A020F00F
:1021C00015FF00200C49485536A020F00FFFEBE723
:1021D0005735354D4833322020544C5320457861D3
:1021E0006D706C650D0A0000F01002402635EDCDD3
:1021F000006C01402000002040010020AC5B020880
:1022000057495A6E65742043415244204372797095
:102210007420546573742056312E302073746172AB
:10222000742E2E2E2E2E2E0D0A00000040090020A6
:10223000370000205735354D483332204D626564F4
:10224000544C53205472616E736D697373696F6E71
:1022500020746573742073746172742E2E2E2E2E6A
:102260002E0D0A005735354D4833322067657420EE
:1022700062616964752E636F6D2068746D6C206394
:102280006F6E74656E742E2E2E2E2E2E0D0A00008B
:10229000445B0208726563765F6C656E3A25640D77
:1022A0000A00000052656365697665643A2025730B
:1022B000000000000CB500200190009070480068FC
:1022C00040F480306E49086000BF6D48006800F43B
:1022D000003000900198401C0190009818B90198B6
:1022E000B0F5706FF1D16648006800F4003010B1AD
:1022F0000120009001E0002000900098012843D1C7
:102300006048006840F010005E49086008460068B8
:1023100020F0030008600846006840F002000860F2
:102320005748406856494860084640684860084633
:10233000406840F4806048600846406820F47C10A3
:1023400048600846406840F4E81048600846006865
:1023500040F08070086000BF4948006800F00070DD
:102360000028F9D04648406820F0030044494860FE
:102370000846406840F00200486000BF404840689E
:1023800000F00C000828F9D10CBD10B5FFF792FF42
:1023900010BD10B53A48006840F0010038490860A7
:1023A0000846406838490840354948600846006892
:1023B00036490840324908600846006820F4802009
:1023C00008600846406820F4FE0048604FF41F0093
:1023D0008860FFF7DAFF4FF000602D49086010BDFC
:1023E00010B5002100200022254B5B6803F00C0192
:1023F00021B1042906D0082931D107E0254B264C0C
:10240000236030E0234B244C23602CE01C4B5B68A2
:1024100003F470101A4B5B6803F48032184B5B684E
:1024200003F080531BB1112303EB904002E0022321
:1024300003EB904022B9194B4343174C23600DE046
:102440000F4B5B6803F4003323B1144B4343124C2E
:10245000236003E00F4B43430F4C236003E00D4B1D
:102460000D4C236000BF00BF054B5B68C3F3031333
:102470000B4CE15C084B1B68CB40074C236010BD44
:1024800000100240002002400000FFF8FFFFF6FEAF
:1024900008ED00E000127A003C00002000093D0039
:1024A00040000020704700BFFEE700BFFEE700BF0E
:1024B000FEE700BFFEE770477047704770470000B7
:1024C00010B54FF4385020F017F8044604F002001D
:1024D00008B1642000E00A20014674A020F086FDC7
:1024E00004F0040008B17AA000E07CA001467EA0C0
:1024F00020F07CFD10BD08B500BF4FF47A7000F0ED
:10250000ADFA69460F2001F094FD9DF80000012806
:1025100005D17DA020F06AFDFFF7D2FF02E07DA08B
:1025200020F064FD9DF800000028E6D008BD00B54D
:1025300089B003A801F04CFE9DF82200022807D1C3
:10254000784820F053FD78A17AA020F04FFD06E0F6
:10255000744820F04BFD74A180A020F047FD9DF849
:1025600011109DF810009DF80F20CDE90020029178
:102570009DF80E309DF80D209DF80C1081A020F0E4
:1025800035FD9DF8150000909DF814309DF813203E
:102590009DF8121087A020F029FD9DF819000090E9
:1025A0009DF818309DF817209DF8161089A020F08E
:1025B0001DFD9DF81D0000909DF81C309DF81B200E
:1025C0009DF81A108BA020F011FD03A8407D00900B
:1025D00003A8037D9DF81F209DF81E108DA020F0FC
:1025E00005FD944820F002FD09B000BDF0B587B0AC
:1025F00005460E46012700243146284602F06EFEAD
:102600008DA020F0F3FC39E002F08BFD28B1042806
:1026100005D10CB90124002701E0002700BF00BF4D
:10262000002F2BD10CB188A000E089A001468AA020
:1026300020F0DCFC02F049FEF4B10DF10A0002F0DA
:10264000E6FE0DF1120002F0EFFE0DF10E0002F0B9
:10265000F8FE0DF1160002F001FF02208DF81A00BD
:10266000062201A94FF410601FF09AFF01A801F0A3
:10267000D8FD012007B0F0BD0020FBE7C4E770B52E
:1026800006460C46204601F0CCFDA07D02280AD16A
:1026900031460020FFF7AAFF054625B90120A075A5
:1026A000204601F0BEFDFFF742FF70BD5468652073
:1026B00063757272656E74204D62746973207370F5
:1026C000656564203A2025644D6270730D0A000030
:1026D00046756C6C2D4475706C65780048616C664D
:1026E0002D4475706C65780054686520637572724E
:1026F000656E74204475706C6578204D6F6465203C
:102700003A2025730D0A0000504859206C696E6B01
:102710000D0A0000504859206E6F206C696E6B0DD9
:102720000A000000685C02085735354D4833320016
:1027300000000000202573206E6574776F726B2097
:10274000636F6E66696775726174696F6E203A2097
:10275000444843500D0A0D0A000000002025732054
:102760006E6574776F726B20636F6E6669677572E2
:102770006174696F6E203A207374617469630D0A25
:102780000D0A0000204D4143202020202020202041
:10279000203A20253032583A253032583A25303206
:1027A000583A253032583A253032583A2530325886
:1027B0000D0A000020495020202020202020202029
:1027C000203A2025642E25642E25642E25640D0ACA
:1027D00000000000205375626E6574204D61736BBC
:1027E000203A2025642E25642E25642E25640D0AAA
:1027F0000000000020476174657761792020202067
:10280000203A2025642E25642E25642E25640D0A89
:102810000000000020444E532020202020202020B3
:10282000203A2025642E25642E25642E25640D0A69
:1028300000000000FC5B0208444843502072756EA3
:102840006E696E670D0A00007375636365737300CC
:102850006661696C000000004448435020257321E4
:102860000D0A000000B589B001210220FDF7FEFE2F
:102870006846FDF76EFE40F2E730ADF81C002649D1
:102880000198B0FBF1F0401E80B2ADF818000020B6
:10289000ADF81E00ADF81A0006A92048FEF765FD48
:1028A000012211461D48FFF7B2F81D208DF81400D3
:1028B00000208DF8150003208DF8160001208DF8FA
:1028C000170005A8FDF7D3FC01211448FFF784F891
:1028D00009B000BD10B501211048FFF750FBB8B199
:1028E0000F480068401C0E4908600E480068401CF4
:1028F0000C49086008460068B0F57A7F04D302F0FE
:1029000080FD00200749086001210448FFF748FBCB
:1029100010BD03480068704740420F0000040040AB
:10292000500000205400002010B586B0044601215C
:102930008803FDF78EFE01210420FDF78AFE4FF487
:102940000070ADF8140003208DF8160018208DF8E3
:10295000170005A91A48FDF74DFF4FF48060ADF848
:10296000140004208DF8170005A91548FDF742FF53
:1029700001940020ADF80800ADF80A00ADF80C0095
:10298000ADF810000C20ADF80E0001A90D48FEF7BF
:10299000EEF801210B48FEF780F906B010BD70B5C6
:1029A00004460D4600BF40210648FEF751FA0028B4
:1029B000F9D0E1B20348FEF7DDF9204670BD000012
:1029C000000801400038014000B585B06846FDF7B9
:1029D000C0FD6FF00400FDF794FC0098C0083F496B
:1029E000B0FBF1F03E4908700846007800EB40016A
:1029F000C1EBC0104FF6FF7101EAC00039490880F1
:102A0000374800786FF07F4191FBF0F0364908605D
:102A100005B000BD0146324A12784A434FF0E02328
:102A20005A6100229A611A46126942F001021A6143
:102A300000BF4FF0E022106900F001021AB100F46B
:102A40008032002AF5D04FF0E022126922F0010214
:102A50004FF0E0231A6100229A61704700BF00EB3B
:102A60004002C2EBC012204B1B68B3EBC20F05D271
:102A70001D4A12681A4B1B785A4302E0194A128801
:102A800042434FF0E0235A611A465269154B1B88A6
:102A9000B2FBF3F2821A90B200224FF0E0239A6167
:102AA0001A46126942F001021A6100BF4FF0E0229B
:102AB000116901F001021AB101F48032002AF5D047
:102AC0004FF0E022126922F001024FF0E0231A6178
:102AD00000229A610028C2DC7047000040420F00CB
:102AE000580000205A0000205C00002010B5FDF7BF
:102AF00027FC4FF48030FDF743FC00BF3120FDF789
:102B000062FC0028FAD00020FDF7AEFC0122164935
:102B100010041FF0D3FE0120FDF7A6FC00BF3920F2
:102B2000FDF751FC0028FAD00220FDF7A0FC0020A0
:102B3000FDF7ABFC4FF48060FDF7B0FC0020FDF723
:102B4000B6FC0120FDF7F8FC00BF6120FDF73BFC5F
:102B50000028FAD00120FDF778FC00BF2120FDF706
:102B600032FC0028FAD010BD0000281010B5044631
:102B700000BF082C02DD4FF0FF3010BD00BFA100E8
:102B8000491C4FF4807202EBC10010211FF07CFD44
:102B900000BFA100491C4FF4807202EBC1001FF07E
:102BA000ABFC0028F5D1A100491C4FF4007202EBE8
:102BB000C1001F211FF068FD0120A040F8490988CD
:102BC0008143F74801800120A040F64909888143EC
:102BD000F44801800020F44921F81400F349085515
:102BE00000BFA100491C4FF4407202EBC1001FF06E
:102BF00083FC0028F5D10120BFE7F8B504460E4656
:102C000017461D4600BF082C02DD4FF0FF30F8BD0F
:102C100000BF012E06D0022E10D0032E10D0042E9D
:102C20000FD10CE0042269464FF470601FF0B8FC2D
:102C3000009810B96FF00200E9E705E000BF00BF9F
:102C400002E06FF00400E2E700BF05F0040010B1FD
:102C50006FF00500DBE705B3012E02D0022E1AD17A
:102C600006E005F0210010B96FF00500CFE713E092
:102C700005F0200028B105F0800010B96FF00500C4
:102C8000C5E705F0100028B105F0800010B96FF01D
:102C90000500BCE700E000BF00BF2046FFF766FF6D
:102CA00005F0F00242EA0601A200521C002303EBE9
:102CB000C2001FF0E9FC7FB9BD4807880088401CAE
:102CC000BB490880084600884FF6F071884203D15E
:102CD0004FF44040B64908803912A200521C4FF40C
:102CE000806303EBC2001FF0CFFCF9B2A200521CBC
:102CF0004FF4806303EBC20202F580701FF0C4FC46
:102D0000A100491C4FF4807202EBC10001211FF0A9
:102D1000BBFC00BFA100491C4FF4807202EBC10054
:102D20001FF0EAFB0028F5D10120A0409C4909884A
:102D300081439B48018005F00100A0409849098823
:102D40000843974908800120A0409649098881439B
:102D5000944801800020944921F8140093490855B3
:102D600000BFA100491C4FF4407202EBC1001FF0EC
:102D7000C3FB0028F5D060B249E710B5044600BF98
:102D8000082C02DD4FF0FF3010BD00BF00BFA100D6
:102D9000491C002202EBC1001FF0AEFB00F00F0047
:102DA000012802D06FF00400EEE700BF00BFA100D1
:102DB000491C4FF4407202EBC1001FF09DFB132829
:102DC00002D06FF00200DFE700BFA100491C4FF402
:102DD000807202EBC10002211FF056FC00BFA1006F
:102DE000491C4FF4807202EBC1001FF085FB0028E4
:102DF000F5D105E02046FFF7B9FE6FF00300C3E709
:102E0000A100491C4FF4407202EBC1001FF074FB9B
:102E10001428EFD10120B7E770B504460D461646D9
:102E200000BF082C02DD4FF0FF3070BD00BF00BFB7
:102E3000A100491C002202EBC1001FF05DFB00F065
:102E40000F00012802D06FF00400EEE700BF00BFC2
:102E5000A100491C4FF4407202EBC1001FF04CFB73
:102E6000132802D06FF00200DFE700BF29786878EE
:102E700061F31F200146A87861F31F200146E8781E
:102E800061F31F200146481C00B111B96FF00B001F
:102E9000CBE716B96FF00A00C7E7A100491C4FF451
:102EA000406202EBC100042229461FF043FC3112AC
:102EB000A200521C4FF4805303EBC2001FF0E4FB4E
:102EC000F1B2A200521C4FF4805303EBC20202F590
:102ED00080701FF0D9FBA100491C4FF4807202EBF7
:102EE000C10004211FF0D0FB00BFA100491C4FF41A
:102EF000807202EBC1001FF0FFFA0028F5D101201B
:102F0000A04027490988084008B100208DE722E049
:102F1000A100491C4FF4007202EBC1001FF0ECFA53
:102F200000F0080058B1A100491C4FF4007202EBF8
:102F3000C10008211FF0A8FB6FF00C0075E7A1008D
:102F4000491C4FF4407202EBC1001FF0D5FA10B9D2
:102F50006FF0030069E7A100491C4FF4407202EBD7
:102F6000C1001FF0C9FA1728D2D101205DE710B5C2
:102F7000044600BF082C02DD4FF0FF3010BD00BF3B
:102F800000BFA100491C002202EBC1001FF0B4FAEF
:102F900000F00F0001280DD06FF00400EEE70000F4
:102FA000620000206400002060090020660000200C
:102FB0006000002000BFA100491C4FF4807202EBAA
:102FC000C10008211FF060FB00BFA100491C4FF4A5
:102FD000807202EBC1001FF08FFA0028F5D10120AA
:102FE000A040FE4909888143FC4801800120A0409F
:102FF000FB490988084008B10020BFE710E0A100A4
:10300000491C4FF4007202EBC1001FF075FA00F08A
:10301000080028B12046FFF7A9FD6FF00C00ADE7CE
:10302000A100491C4FF4407202EBC1001FF064FA8A
:103030000028E4D10120A1E72DE9F04104468846AB
:1030400015460026002700BF082C02DD701EBDE8D3
:10305000F08100BF00BFA100491C002202EBC100AB
:103060001FF04AFA00F00F00012802D06FF00400B0
:10307000EDE700BF00BF15B96FF00D00E7E700BF37
:10308000A100491C4FF4407202EBC1001FF034FA5A
:103090000646172E04D01C2E02D06FF00600D6E78D
:1030A0000120A040CD490988084040B3A100491C37
:1030B0004FF4007202EBC1001FF01EFA00F01F0671
:1030C00006F0100080B1A100491C4FF4007202EB21
:1030D000C10010211FF0D8FA0120A040BF49098883
:1030E0008143BE4801800AE006F0080028B120466E
:1030F000FFF73CFD6FF00C00A9E70020A7E7A10057
:10310000491C4FF4F85202EBC1001FF0F5F94FF6DD
:10311000FF7101EA8027BD4200DD3D4623E02046E5
:103120001FF02CFC0746A100491C4FF4407202EB33
:10313000C1001FF0E1F90646172E07D01C2E05D05E
:103140002046FFF713FD6FF0060080E70120A04046
:10315000A3490988084018B1BD4201DD002076E787
:10316000BD4200DC00E0DAE700BF2A4641462046C7
:103170001FF044FDA100491C4FF4807202EBC10016
:1031800020211FF081FA00BFA100491C4FF480727A
:1031900002EBC1001FF0B0F90028F5D10120A040DA
:1031A0008E49098808438D49088028464FE72DE954
:1031B000F0470446884616460027002500BF082C25
:1031C00002DD681EBDE8F08700BF00BFA100491CFA
:1031D000002202EBC1001FF08FF900F00F00012860
:1031E00002D06FF00400EDE700BF00BF16B96FF02A
:1031F0000D00E7E700BFA100491C4FF4F05202EBBD
:10320000C1001FF079F94FF6FF7101EA8025B54240
:1032100000DA2E4638E020461FF060FB0546A1008C
:10322000491C4FF4407202EBC1001FF065F90746DC
:10323000172F1ED01C2F16D105B126E020461FF0F7
:103240009DFB8146A100491C4FF4F85202EBC100DE
:103250001FF052F9B9EB802F0BD12046FFF786FC07
:103260006FF00600AEE72046FFF780FC6FF0060027
:10327000A8E70120A0405A490988084010B10DB9BB
:1032800000209FE705B100E0C5E700BFB54200DAC6
:103290002E463246414620461FF014FCA100491C30
:1032A0004FF4807202EBC10040211FF0EDF900BF26
:1032B000A100491C4FF4807202EBC1001FF01CF901
:1032C0000028F5D130467DE72DE9F05F04468B46B6
:1032D00015461E46DDF828A00027B84600BF082C7A
:1032E00002DD781EBDE8F09F00BFA100491C00224E
:1032F00002EBC1001FF000F900F00F00022804D01B
:10330000032804D0042803D100E000BF00BF02E07E
:103310006FF00400E6E700BF00BF15B96FF00D00C5
:10332000E0E700BF96F80090707869F31F208146AF
:10333000B07869F31F208146F07869F31F20814639
:10334000B9F1000F0DD1A100491C002202EBC10010
:103350001FF0D2F800F00400042802D06FF00B0038
:10336000C0E7BAF1000F0DD1A100491C002202EB09
:10337000C1001FF0C1F800F00400042802D06FF073
:103380000A00AFE7A100491C4FF4407202EBC100F4
:103390001FF0B2F80746422F06D0222F04D0322F5A
:1033A00002D06FF006009DE7A100491C4FF4406277
:1033B00002EBC100042231461FF0BCF94FEA2A217A
:1033C000A200521C4FF4805303EBC2001FF05CF9C3
:1033D0000AF0FF01A200521C04E00000640000207B
:1033E000620000204FF4805303EBC20202F58070AC
:1033F0001FF04AF9A100491C4FF4F85202EBC1003A
:103400001FF07AF84FF6FF7101EA8028454500DD8C
:1034100045461CE020461FF0B1FA8046A100491C39
:103420004FF4407202EBC1001FF066F810B96FF064
:10343000030057E70120A040F8490988084018B167
:10344000454501DD00204DE7454500DC00E0E1E7B2
:1034500000BF2A46594620461FF0D0FBA100491C58
:103460004FF4807202EBC10020211FF00DF900BF64
:10347000A100491C4FF4807202EBC1001FF03CF820
:103480000028F5D125E0A100491C4FF4007202EBA1
:10349000C1001FF031F800F01F0707F0100048B11D
:1034A000A100491C4FF4007202EBC10010211FF073
:1034B000EBF80FE007F0080058B1A100491C4FF4E9
:1034C000007202EBC10008211FF0DEF86FF00C0063
:1034D00008E7D8E700BF284604E72DE9FC47044683
:1034E0008A4616461D46DDF82880002700BF082CB6
:1034F00002DD781EBDE8FC8700BFA100491C002248
:1035000002EBC1001EF0F8FF814600F00F00022818
:1035100004D0032803D0042803D101E000BF00BF7A
:1035200002E06FF00400E5E700BF00BF16B96FF0DE
:103530000D00DFE700BFBA4830F81400E8B91AE020
:1035400020461FF0CBF90746A100491C4FF44072FA
:1035500002EBC1001EF0D0FF10B96FF00300C9E705
:103560000120A040AD490988084010B10FB90020E2
:10357000C0E707B100E0E3E700BF09F00700022859
:1035800004D003287ED004287DD158E0A44830F828
:103590001400E8BB0822694620461FF093FAA100F8
:1035A000491C4FF4807202EBC10040211FF06CF8FF
:1035B00000BFA100491C4FF4807202EBC1001EF055
:1035C0009BFF0028F5D19DF8000028709DF80100B0
:1035D00068709DF80200A8709DF80300E8709DF8DF
:1035E0000400A8F800009DF8050098F8001000EB12
:1035F0000120A8F800009DF80600894921F8140070
:103600009DF8070011F8141000EB0120844900E038
:1036100004E021F81400802082490855804830F8E1
:103620001400B04201DD374602E07D4830F81470E6
:103630003E463A46514620461FF044FAA1E07848FB
:1036400030F81400B8BB0222694620461FF03AFA4F
:10365000A100491C4FF4807202EBC10040211FF011
:1036600013F800BFA100491C4FF4807202EBC100A7
:103670001EF042FF0028F5D19DF80000684921F8AE
:10368000140001E02BE074E09DF8010011F8141023
:1036900000EB0120801E624921F81400084630F832
:1036A000140040F2EA51884206DD2046FFF75EFA38
:1036B0006FF47A701EE702E080205A490855584896
:1036C00030F81400B04201DD374602E0544830F8CB
:1036D00014703A46514620461FF0F4F951E0504824
:1036E00030F81400A8BB0622694620461FF0EAF90C
:1036F000A100491C4FF4807202EBC10040211EF072
:10370000C3FF00BFA100491C4FF4807202EBC1004F
:103710001EF0F2FE0028F5D19DF8000028709DF8FB
:10372000010068709DF80200A8709DF80300E87021
:103730009DF804003A4921F814009DF8050011F89D
:10374000141000EB0120364921F81400802035497F
:103750000855334830F81400B04201DD374602E026
:103760002F4830F814703A46514620461FF0AAF907
:1037700007E0394620461FF0F9F9294820F814706F
:1037800000BF00BFA100491C4FF4807202EBC100D2
:1037900040211EF079FF00BFA100491C4FF4807248
:1037A00002EBC1001EF0A8FE0028F5D11C4830F83D
:1037B0001400C01B1A4921F81400084630F8140000
:1037C00030B11848005D40F001001649085502E08C
:1037D00000201449085538468CE62DE9F04104468E
:1037E0000E461546002700BF082C02DD781EBDE8F6
:1037F000F08100BF082E77D2DFE806F004232A38D4
:10380000465864772F78012F0ED10120A04003493C
:10381000098808430149088012E000006200002086
:1038200060090020660000203FB90120A040FA494D
:1038300009888143F848018002E06FF00900D6E76B
:1038400062E0F5480088204100F0010028705BE04C
:10385000A100491C4FF4F85202EBC1001EF04CFECF
:103860004FF6FF7101EA802028804DE0A100491C3D
:103870004FF4F05202EBC1001EF03EFE4FF6FF7116
:1038800001EA802028803FE028781F2802DD6FF0C1
:103890000900ACE72A7802F01F01A200521C4FF485
:1038A000007303EBC2001EF0EFFE2DE0A100491CE7
:1038B0004FF4007202EBC1001EF01EFE00F01F006C
:1038C000287021E028781F2802DD6FF009008EE7BC
:1038D0002A7802F01F01A200521C4FF4305303EB70
:1038E000C2001EF0D1FE0FE00BE0A100491C4FF416
:1038F000305202EBC1001EF0FFFD00F01F002870E7
:1039000002E06FF0090072E700BF01206FE770B5B9
:1039100004460E46154600BF082C02DD4FF0FF306E
:1039200070BD00BF082E76D2DFE806F0B2040E1894
:103930002E394F982978A200521C4FF4B05303EB54
:10394000C2001EF0A1FEA6E02978A200521C4FF48E
:10395000A85303EBC2001EF097FE9CE02A881112C8
:10396000A200521C4FF4905303EBC2001EF08CFED9
:103970002978A200521C4FF4905303EBC20202F5C7
:1039800080701EF081FE86E0A100491C4FF4406269
:1039900002EBC100042229461EF0CCFE7BE02A88FF
:1039A0001112A200521C4FF4805303EBC2001EF010
:1039B0006BFE2978A200521C4FF4805303EBC20225
:1039C00002F580701EF060FE65E000BFA100491C9A
:1039D000002202EBC1001EF08FFD00F00F00012855
:1039E00002D06FF004009BE700BFA100491C4FF418
:1039F0003C5202EBC1001EF07FFD10B16FF00100E0
:103A00008EE7A100491C4FF4807202EBC100222115
:103A10001EF03AFE17E03BE0A100491C4FF4007293
:103A200002EBC1001EF068FD00F0080058B1A100D3
:103A3000491C4FF4007202EBC10008211EF024FE65
:103A40006FF00C006CE7A100491C4FF4807202EB90
:103A5000C1001EF051FD0028DED11CE000BFA10016
:103A6000491C002202EBC1001EF046FD00F00F00D1
:103A7000012802D06FF0040052E700BF2978A200AD
:103A8000521C4FF43C5303EBC2001EF0FDFD02E05C
:103A90006FF0090044E700BF012041E72DE9F04144
:103AA00004460E46154600BF082C03DD4FF0FF30DC
:103AB000BDE8F08100BF0D2E6FD2DFE806F00712DF
:103AC0001C263D48B55F7A7F848EA200A100491C68
:103AD000002202EBC1001EF00FFD00F0F000287084
:103AE000A5E0A100491C4FF4B05202EBC1001EF04A
:103AF00003FD28709BE0A100491C4FF4A85202EB83
:103B0000C1001EF0F9FC287091E0A100491C4FF49F
:103B1000905202EBC10101F580701EF0EDFC0746EA
:103B2000A100491C4FF4905202EBC1001EF0E4FCCE
:103B300007EB002028807AE0A100491C4FF4406286
:103B400002EBC100042229461EF02AFD6FE0A1000D
:103B5000491C4FF4805202EBC10101F580701EF048
:103B6000CBFC0746A100491C4FF4805202EBC10078
:103B70001EF0C2FC07EB0020288058E000BFA10027
:103B8000491C002202EBC1001EF0B6FC00F00F0041
:103B9000012803D06FF004008AE745E000BFA100D0
:103BA000491C4FF43C5202EBC1001EF0A5FC2880DA
:103BB0003DE020461EF0E2FE288038E020461EF060
:103BC0008DFE288033E0A100491C4FF4407202EBC7
:103BD000C1001EF091FC287029E0A100491C0022C0
:103BE00002EBC1001EF088FC00F0010020B120466D
:103BF0001EF074FE288003E0084830F81400288086
:103C000015E0A100491C002202EBC1001EF074FC6B
:103C1000012805D1801F4BE76200002060090020C9
:103C20000448005D287002E06FF0010040E700BF2B
:103C300001203DE7660000207047704770477047DD
:103C40000146087870470170704700207047704740
:103C50007047704700B141B9AFF22302FA4BDA6006
:103C6000AFF22903F84A136102E0F74AD06011610C
:103C7000704700B141B9AFF23B02F34B5A61AFF26A
:103C80004103F14A936102E0EF4A5061916170474C
:103C900000BFED4A128802F40072002AF9D000B188
:103CA00041B9AFF25902E84BDA61AFF25D03E64A7F
:103CB000136202E0E44AD0611162704700BFE24A39
:103CC000128802F40072002AF9D000B139B9AFF2BB
:103CD0007F03DD4A5362AFF28503936202E0DA4A62
:103CE00050629162704710B500244FF438501EF0B6
:103CF00003FC00F0010000B10124204610BD10B506
:103D000000244FF438501EF0F7FB00F03800302844
:103D100001D1012400E00024204610BD10B54FF46D
:103D200038501EF0E9FB044624F0800421464FF48D
:103D300038501EF0A9FC4FF438501EF0DDFB04464D
:103D400044F0800421464FF438501EF09DFC10BD15
:103D500070B5054600244FF438501EF0CDFB0446E4
:103D600004F0400010B94FF0FF3070BD24F038046B
:103D7000012D02D144F0300401E044F03804214622
:103D80004FF438501EF080FCFFF7C8FF4FF4385056
:103D90001EF0B2FB0446012D04D104F0300030B116
:103DA0000020E2E704F0380008B10020DDE74FF022
:103DB000FF30DAE770B5044600254FF438501EF0A6
:103DC0009BFB0546C5F38010207005F038002028C5
:103DD00002D0382803D100BF0120607002E000202B
:103DE000607000BF00BF05F03800102805D018280B
:103DF00002D0202804D100BF00BF0120A07002E043
:103E00000020A07000BF00BF05F03800082805D0D2
:103E1000182802D0202804D100BF00BF0120E07084
:103E200002E00020E07000BF00BF70BD70B5054625
:103E300000242878012802D144F0400401E024F055
:103E400040046878012802D144F0380412E0E87890
:103E5000012808D1A878012802D144F0180409E00B
:103E600044F0080406E0A878012802D144F01004C8
:103E700000E000BF21464FF438501EF005FCFFF76C
:103E80004DFF70BD70B50026002400254FF4B050E2
:103E90001EF032FB06464FF4C0501EF02DFB0446C8
:103EA000254606EB052085B2284670BD70B5044650
:103EB000E5B2261229464FF4B0501EF0E5FB31461C
:103EC0004FF4C0501EF0E0FB70BD70B5002600241A
:103ED00000254FF4A8501EF00FFB00F0F0064FF441
:103EE000B8501EF009FB0446254606EB052085B2B6
:103EF000284670BD70B50546ECB22E1204F0F001F4
:103F00004FF4A8501EF0C0FB00240EE00120A0409A
:103F1000304040B1A100491C4FF4007202EBC100D7
:103F20001F211EF0B1FB601CC4B2082CEEDB70BD7B
:103F300000B585B0062269464FF410601EF030FBD4
:103F4000042204A990011EF02BFB042203A94FF4C4
:103F5000A0601EF025FB042202A94FF470601EF041
:103F60001FFB802100201EF08FFB00201EF0C4FAF2
:103F7000062269464FF410601EF0DCFB042204A9FF
:103F800090011EF0D7FB042203A94FF4A0601EF09D
:103F9000D1FB042202A94FF470601EF0CBFB05B0E8
:103FA00000BD2DE9F04105460E460027FFF7C0FF92
:103FB000F5B100BF00240AE0285D384447B2102F55
:103FC00003DD4FF0FF30BDE8F081601C44B2082CE7
:103FD000F2DB00240AE0295DA200521C4FF4F853E2
:103FE00003EBC2001EF050FB601C44B2082CF2DB55
:103FF000EEB10027002409E0305D384447B2102FAD
:1040000002DD4FF0FF30DEE7601C44B2082CF3DB2A
:1040100000240AE0315DA200521C4FF4F05303EB80
:10402000C2001EF031FB601C44B2082CF2DB002001
:10403000C9E72DE9FC4106460C460025002000900A
:104040000190102E7FD201E070000020DFE806F022
:10405000080B1A161E2226323F54575B5F606470AD
:10406000FFF766FF72E01CB10094009808300190E1
:10407000DDE90001FFF795FFBDE8FC812088FFF72F
:1040800039FF63E0FFF721FF20805FE02088FFF722
:104090000DFF5BE0FFF7F6FE208057E0208801125D
:1040A0004FF498501EF0F0FA21784FF4A0501EF013
:1040B000EBFA4BE04FF4A0501EF01EFA07464FF407
:1040C00098501EF019FA07EB002020803EE084484B
:1040D000807820708248C078607081480079A07034
:1040E0007F484079E0707E48807920717C48C079B3
:1040F00060710020A07129E0FFF710FE26E0204645
:10410000FFF794FE22E02046FFF754FE1EE01DE07C
:104110002078FFF71DFEAFE7FFF7F1FDC5B268B2EB
:10412000401C18B94FF0FF30A6E70CE025700DE0F9
:10413000FFF7D9FDC5B268B2401C10B94FF0FF308F
:104140009AE7257002E04FF0FF3095E700BF0020AE
:1041500092E770B504464FF4D8501EF0CDF92070A8
:104160004FF4D0501EF0C8F905464FF4C8501EF069
:10417000C3F905EB0020608070BD10B504462178BE
:104180004FF4D8501EF080FA608801124FF4C850E6
:104190001EF07AFAA1784FF4D0501EF075FA10BDD7
:1041A00010B500201EF0A8F910BD70B5044600251A
:1041B00024F03A0008B1681E70BD00201EF09CF982
:1041C00005462543294600201EF05EFA0020F3E74D
:1041D00010B50446062221464FF410601EF0E0F9A7
:1041E000042204F10E0190011EF0DAF9042204F118
:1041F0000A014FF4A0601EF0D3F90422A11D4FF470
:1042000070601EF0CDF937480078A07435484178C9
:10421000E17481782175C178617533480078A075A3
:1042200010BD10B50446062221464FF410601EF062
:1042300081FA042204F10E0190011EF07BFA04229F
:1042400004F10A014FF4A0601EF074FA0422A11DCB
:104250004FF470601EF06EFAA07C22490870E07C7A
:104260004870207D8870607DC870A07D1E490870F0
:1042700010BD70B505460C46062D1CD2DFE805F0D2
:1042800003070B0F13172046FFF7CBFF16E020465E
:10429000FFF79EFF12E02078FFF787FF70BDFFF762
:1042A0007FFF20700AE02046FFF767FF06E0204608
:1042B000FFF74FFF02E04FF0FF30EFE700BF0020B5
:1042C000ECE770B504464FF438501EF015F905467A
:1042D000C5F38000E070C5F34000A07070BD000021
:1042E000700000209C000020A000002010B50422D7
:1042F000FE494FF470601EF01DFA0422FC494FF491
:10430000A0601EF017FA0422FA4990011EF012FA7A
:1043100010BD10B5802100201EF0B6F900201EF05F
:10432000EBF8FFF7E3FF0622F3494FF410601EF0AD
:1043300001FA10BD10B5802100201EF0A5F9002063
:104340001EF0DAF80622EC494FF410601EF0F2F984
:1043500010BD10B5AFF26B03E84C2360AFF24D0314
:10436000E74C2360AFF23303E64C236008B1E34B24
:10437000186009B1E24B19600AB1E24B1A6010BD36
:104380007CB5062269464FF410601EF009F9012041
:10439000DD4909680870DC49096848700620DA4977
:1043A000096888700020D8490968C870D648006834
:1043B000051DD6480068000E2870D4480068000C1F
:1043C0006870D2480088000AA870D0480078E87069
:1043D0000020CD4909680881CB48006800F10A0532
:1043E0008020287000206870C74909680873002180
:1043F000C54800684173C44800688173C2480068BA
:10440000C1730020C049096808740021BE480068D3
:104410004174BD4800688174BB480068C1740020C5
:10442000B949096808750021B74800684175B64860
:1044300000688175B4480068C1750020B2490968F8
:1044400008760021B04800684176AF480068817660
:10445000AD480068C176A8480078AB49096808777C
:10446000A5484178A84800684177A3488178A648C4
:1044700000688177A048C178A3480068C1779E484A
:104480000179A148006880F820109B4841799E4836
:10449000006880F82110062406E000219A48006890
:1044A0001C300155601CC4B2102CF6DB002406E061
:1044B0000021954800682C300155601CC4B2402C86
:1044C000F6DB002406E000218F4800686C300155BF
:1044D000601CC4B2802CF6DB63208B49096881F82C
:1044E000EC0082218848006880F8ED10532186484E
:1044F000006880F8EE1063218348006880F8EF10B0
:104500007CBD014601F00F01092903DC01F13000F7
:10451000C0B2704701F13700C0B2FAE77CB50024A1
:10452000FFF72EFF00207A49087048708870C87025
:104530007849087048708870C87004243522214674
:10454000641C71480068EC30425401222146641C0E
:104550006D480068EC3042542146641C6A4800688B
:10456000EC3042543D222146641C67480068EC3020
:10457000425407222146641C63480068EC304254D0
:1045800001222146641C60480068EC3042545A48BD
:1045900002782146641C5C480068EC30425456485E
:1045A00042782146641C58480068EC304254524816
:1045B00082782146641C54480068EC3042544E48CE
:1045C000C2782146641C50480068EC3042544A4886
:1045D00002792146641C4C480068EC30425446483D
:1045E00042792146641C48480068EC3042540C2251
:1045F0002146641C44480068EC30425400222046A6
:10460000611C8CB240490968EC310A5400250AE06B
:104610004148425D2046611C8CB23B490968EC313F
:104620000A54681C85B23C48405D0028F0D13249EC
:10463000C9780811FFF765FF2146621C94B2324A1F
:104640001268EC3250542C49C878FFF75AFF2146C3
:10465000621C94B22C4A1268EC32505426490979F3
:104660000811FFF74EFF2146621C94B2264A1268D9
:10467000EC32505420490879FFF743FF2146621C71
:1046800094B2214A1268EC3250541B4949790811FE
:10469000FFF737FF2146621C94B21B4A1268EC32C6
:1046A000505415494879FFF72CFF2146621C94B2FB
:1046B000154A1268EC325054A81DC1B2E81D221AE6
:1046C00011480068EC30815437222046611C8CB2BE
:1046D0000D490968EC310A5406222046611C8CB24F
:1046E00009490968EC310A54012217E0B1000020A1
:1046F000B9000020B5000020E0000020E800002004
:10470000EC000020F0000020D4000020D0000020A9
:10471000A5000020A9000020D80000202046611C30
:104720008CB2FE490968EC310A5403222046611C10
:104730008CB2FA490968EC310A5406222046611C01
:104740008CB2F6490968EC310A540F222046611CEC
:104750008CB2F2490968EC310A543A222046611CB5
:104760008CB2EE490968EC310A543B222046611CA8
:104770008CB2EA490968EC310A54FF222046611CD8
:104780008CB2E6490968EC310A54254606E000215E
:10479000E2480068EC304155681C85B2B5F59C7F55
:1047A000F5DBFF208DF804008DF805008DF806007C
:1047B0008DF80700432001AB4FF409720090D748F1
:1047C0000168D7480078FEF77FFD7CBD7CB50024EA
:1047D000FFF7D6FDD3480078032803D0D1480078EE
:1047E00004282CD10020CD49096888720021CB48CB
:1047F0000068C172CC480078C84909680873CA4883
:104800004178C64800684173C7488178C34800684A
:104810008173C548C178C1480068C173C348007836
:104820008DF80400C14840788DF80500BF488078B5
:104830008DF80600BD48C0788DF8070008E0FF201D
:104840008DF804008DF805008DF806008DF807003E
:10485000042435222146641CB0480068EC304254E0
:1048600001222146641CAD480068EC30425403220A
:104870002146641CA9480068EC3042543D22214680
:10488000641CA6480068EC30425407222146641C90
:10489000A2480068EC30425401222146641C9F4823
:1048A0000068EC304254A24802782146641C9B48C0
:1048B0000068EC3042549E4842782146641C974878
:1048C0000068EC3042549A4882782146641C934830
:1048D0000068EC3042549648C2782146641C8F48E8
:1048E0000068EC304254924802792146641C8B489F
:1048F0000068EC3042548E4842792146641C874857
:104900000068EC3042549DF80700FF2867D132223E
:104910002146601C84B281480068EC304254042275
:104920002146601C84B27D480068EC3042547E48C9
:1049300002782046611C8CB278490968EC310A542F
:10494000794842782046611C8CB274490968EC3180
:104950000A54754882782046611C8CB26F490968F8
:10496000EC310A547048C2782046611C8CB26B4905
:104970000968EC310A5436222146601C84B267482B
:104980000068EC30425404222046611C8CB263491A
:104990000968EC310A54654802782146601C84B2EB
:1049A0005E480068EC304254604842782046611C02
:1049B0008CB25A490968EC310A545C488278204626
:1049C000611C8CB255490968EC310A545748C278C9
:1049D0002046611C8CB251490968EC310A540C2202
:1049E0002046611C8CB24D490968EC310A54002202
:1049F0002046611C8CB249490968EC310A540025F3
:104A000009E04C48425D2046611C8CB2434909686C
:104A1000EC310A546D1C4748405D0028F1D14449EF
:104A2000C9780811FFF76DFD2146621C94B23B4A1C
:104A30001268EC3250543E49C878FFF762FD2146B7
:104A4000621C94B2354A1268EC32505438490979E4
:104A50000811FFF756FD2146621C94B22F4A1268D6
:104A6000EC32505432490879FFF74BFD2146621C65
:104A700094B22A4A1268EC3250542D4949790811EF
:104A8000FFF73FFD2146621C94B2244A1268EC32C3
:104A9000505427494879FFF734FD2146621C94B2EF
:104AA0001E4A1268EC325054A81DC1B2E81D221AE9
:104AB0001A480068EC30815437222046611C8CB2C1
:104AC00016490968EC310A5408222046611C8CB250
:104AD00012490968EC310A5401222046611C8CB24B
:104AE0000E490968EC310A5403222046611C8CB23D
:104AF0000A490968EC310A5406222046611C8CB22E
:104B000006490968EC310A540F222046611C8CB218
:104B100002490968EC310A543A220DE0D400002021
:104B2000A4000020C1000020B1000020A50000204A
:104B3000E0000020D80000202046611C8CB2F7491C
:104B40000968EC310A543B222046611C8CB2F349BF
:104B50000968EC310A541F222046611C8CB2EF49CF
:104B60000968EC310A5421222046611C8CB2EB49C1
:104B70000968EC310A54FF222046611C8CB2E749D7
:104B80000968EC310A54254605E00021E348006835
:104B9000EC3041556D1CB5F59C7FF6DB432001AB35
:104BA0004FF409720090DD480168DD480078FEF797
:104BB0008BFB7CBD7CB50024FFF7E2FB04240020C6
:104BC000D649096888720021D4480068C17235222C
:104BD0002146641CD1480068EC3042540122214631
:104BE000641CCE480068EC30425404222146641C08
:104BF000CA480068EC3042543D222146641CC74834
:104C00000068EC30425407222146641CC348006807
:104C1000EC30425401222146641CC0480068EC304C
:104C20004254C04802782146641CBC480068EC30FD
:104C30004254BC4842782146641CB8480068EC30B5
:104C40004254B84882782146641CB4480068EC306D
:104C50004254B448C2782146641CB0480068EC3025
:104C60004254B04802792146641CAC480068EC30DC
:104C70004254AC4842792146641CA8480068EC3094
:104C8000425432222146641CA4480068EC3042544D
:104C900004222046611C8CB2A0490968EC310A54F8
:104CA000A14802782046611C8CB29C490968EC310D
:104CB0000A549D4842782046611C8CB29749096885
:104CC000EC310A54984882782046611C8CB2934992
:104CD0000968EC310A549448C2782046611C8CB2B1
:104CE0008E490968EC310A5436222046611C8CB288
:104CF0008A490968EC310A5404222046611C8CB2AE
:104D000086490968EC310A54884802782046611CBB
:104D10008CB282490968EC310A54844842782046B2
:104D2000611C8CB27D490968EC310A547F48827855
:104D30002046611C8CB279490968EC310A547B48E1
:104D4000C2782046611C8CB274490968EC310A545F
:104D5000FF222046611C8CB270490968EC310A546C
:104D6000254605E000216D480068EC3041556D1C7A
:104D7000B5F59C7FF6DBFF208DF804008DF805006B
:104D80008DF806008DF80700432001AB4FF409723F
:104D900000906248016862480078FEF795FA7CBD91
:104DA0002DE9FF414FF000085D4800781DF096FDA9
:104DB000071E0BDD01A802AB3A4600905748016878
:104DC00057480078FEF789FB87B203E0002004B063
:104DD000BDE8F081BDF8040043286CD14F4800685D
:104DE000007F50490978884224D14C480068407FB0
:104DF0004C49497888421DD148480068807F49491C
:104E00008978884216D145480068C07F4549C978ED
:104E100088420FD14148006890F820004149097943
:104E2000884207D13D48006890F821003D49497902
:104E3000884201D00020CAE73C48007840B93B488E
:104E4000407828B93948807810B93848C07888B394
:104E50009DF8080035490978884211D19DF809006C
:104E60003249497888420BD19DF80A002F49897848
:104E7000884205D19DF80B002C49C97888421BD087
:104E80009DF808002A490978884211D19DF8090047
:104E90002749497888420BD19DF80A00244989782E
:104EA000884205D19DF80B002149C978884203D07A
:104EB00000208CE700E0AEE018480468F034A7F169
:104EC000F0000519A4E0207833285BD007DC70B12E
:104ED000012813D003282FD0062873D13FE03528AE
:104EE00007D0362870D0FF28F7D12C468FE0641CFD
:104EF0008DE0641C641C14F8018B88E0641C641C45
:104F000014F8010B0B49087014F8010B487014F8E1
:104F1000010B887014F8010BC87078E0D4000020F1
:104F2000A4000020E0000020B1000020A500002027
:104F3000A9000020B9000020641C14F8016B14F8CB
:104F4000010BFE49087014F8010B487014F8010BAE
:104F5000887014F8010BC870301F044457E0641CBB
:104F600014F8016B14F8010BF549087014F8010BE3
:104F7000487014F8010B887014F8010BC870301FCA
:104F8000044444E0641C14F8016B14F8010BED496F
:104F9000086014F8011BEB48006801EB0020E949A8
:104FA000086014F8011BE748006801EB0020E549A0
:104FB000086014F8011BE348006801EB0020E14998
:104FC000086024E01EE0FFE7641C14F8016B14F88D
:104FD000010BDD49087014F8010B487014F8010B3F
:104FE000887014F8010BC8709DF80800D749087044
:104FF0009DF8090048709DF80A0088709DF80B0024
:10500000C87004E0641C14F8016B344400BF00BF96
:10501000AC42FFF458AF4FFA88F0D8E60020CC49F4
:1050200008600A20CB4908600020CB49087070470F
:1050300010B50124C84890F90000022829DAC548B3
:105040000068C349096888423DD2C44890F900000D
:10505000012804D0022805D0042809D105E0FFF773
:105060005DFA06E0FFF7B2FB03E0FFF7AFFB00E0FD
:1050700000BF00BF0020B6490860084600680A303B
:10508000B4490860B4480078401C40B2B249087086
:1050900019E0B24890F90000012804D0022807D096
:1050A00004280CD105E00020AC490870002407E07A
:1050B00000BFFFF733FA0120A849087000E000BFE5
:1050C00000BFFFF7ABFF204610BD38B54FF4D850F6
:1050D0001DF012FA054603214FF4D8501DF0D4FA02
:1050E00041F288309E4B11229EA10090A248007888
:1050F000FEF7EAF8044629464FF4D8501DF0C4FAEA
:1051000004F10D0008B9012038BDFFF753FD9048A8
:10511000046800BF8E480068001B0228FAD30020F4
:10512000F2E770B58D480078062801D1052070BDE2
:10513000914909788900491C4FF4407202EBC10083
:105140001DF0DAF9222806D00023442202218A48E1
:105150000078FDF752FD0125FFF722FEC4B27F481B
:1051600090F90000052877D2DFE800F0030F2C4FFC
:10517000770000207A49087048708870C870FFF77F
:10518000CDF90120754908709CE0022C16D17B48AE
:105190000068007C7249087078480068407C48705C
:1051A00076480068807C887074480068C07CC8704D
:1051B000FFF70CFB02206949087002E0FFF738FF97
:1051C00005467FE0052C14D1FFF77FFF40B16C4806
:1051D00000688047FFF722FF03206049087013E052
:1051E000FFF71CFF67480068804700205B49087094
:1051F0000AE0062C05D1FFF711FF0120574908707E
:1052000002E0FFF715FF05465CE004254D48006805
:10521000401C00B34E4800684A490968B0EB510F82
:1052200019D900244E480078574908704C484078F6
:1052300048704B48807888704948C078C870534897
:105240000068401C51490860FFF7C0FAFFF7E6FE0E
:1052500004204249087035E033E00425052C24D1B0
:1052600000203D490870484800783D490978884247
:1052700011D1454840783A49497888420BD1424893
:10528000807837498978884205D13F48C0783449C9
:10529000C978884203D003253D4800688047FFF75E
:1052A000BDFE03202D4908700AE0062C05D1FFF74A
:1052B000B5FE01202949087002E0FFF7B9FE054656
:1052C00000E000BF00BF284631E710B52A4800784B
:1052D000FDF74CFC06202149087010BD38B5044686
:1052E0000D460020009006222A494FF410601DF060
:1052F00057F928480078274949780843254989788B
:1053000008432449C97808432249097908432149B7
:105310004979084378B900201E4908700820487070
:10532000DC2088700020C8700871487106224FF494
:1053300010601DF0FFF9104804702DE0B50000204A
:10534000BD000020C4000020A5000020A90000200E
:10535000C8000020CC000020C2000020C1000020B6
:10536000B1000020434845434B5F49505F434F4ED7
:10537000464C494354000000A4000020D400002003
:10538000E8000020F0000020AD000020D000002048
:10539000EC000020E000002038480560384839491A
:1053A00008603948C07809680844364908603648BA
:1053B000007909680844334908603348407909682E
:1053C0000844304908603048C0782F49097948407E
:1053D0002D49497948402B49096808442949086002
:1053E000042269464FF470601DF0A4F90422694656
:1053F00090011DF09FF9FFF711FE0020234908706E
:1054000038BD23480068401C214908607047214985
:10541000097801701F49497841701E498978817067
:105420001C49C978C17070471B49097801701A4935
:10543000497841701849897881701749C978C170D5
:105440007047164909780170144949784170134929
:10545000897881701149C978C170704710490978FD
:1054600001700F49497841700D49897881700C4964
:10547000C978C17070470B4800687047D40000209D
:1054800078563412D0000020E0000020C100002037
:10549000C8000020B1000020B5000020B9000020A5
:1054A000BD000020C400002030B503461868081A6B
:1054B000012802DA6FF05F0030BD1868007800F054
:1054C000800028B91C68601C18602078106024E0F7
:1054D0001868007800F07F040CB1042C02DD6FF036
:1054E0006300E9E71868081AA04202DC6FF05F0069
:1054F000E2E7002010601868401C186008E0186897
:105500000078156840EA052010601868401C186093
:10551000201EA4F10104F2D100BF10681C680C1B0E
:10552000A04202D96FF05F00C6E70020C4E7F0B5E3
:1055300004460D4617461E462068281A012802DA3E
:105540006FF05F00F0BD20680078B04202D06FF0CD
:105550006100F7E72068401C20603A462946204653
:10556000FFF7A2FFEEE7F8B504460E4615466FF0CA
:105570006D0701236A4631462046FFF7D8FF071E14
:1055800001D03846F8BD0098012802D06FF06300C2
:10559000F8E72068007808B1012000E000202860CA
:1055A0002068401C20600020ECE72DE9F84104460B
:1055B0000F4616461D466FF06D0833466A4639465B
:1055C0002046FFF7B4FFB0F1000802D04046BDE826
:1055D000F881009810B96FF06300F8E72068007850
:1055E00000F0800010B16FF06300F0E705E0206884
:1055F000401C20600098401E0090009818B1206860
:1056000000780028F3D00098042802D96FF06300D6
:10561000DDE70098042807D12068007800F08000BA
:1056200010B16FF06300D2E70020286008E0206826
:105630000078296840EA012028602068401C20602A
:105640000099481E00900029F1D10020BFE770B5F5
:1056500005460E4614462346022231462846FFF7E9
:10566000A4FF70BD70B505460E46144623460A22B7
:1056700031462846FFF799FF70BDF8B504460E463F
:1056800015466FF06D0702236A4631462046FFF744
:105690004EFF071E01D03846F8BD21682846009A03
:1056A00001F085FF074620680099084420603846CD
:1056B000F2E7F0B504460E4615466FF06D0703237A
:1056C0002A4631462046FFF732FF071E01D03846F2
:1056D000F0BD286810B96FF05F00F9E72868401E38
:1056E00028602068007828712879072802DD6FF08B
:1056F0006300EDE72068401C20602068A8602068F7
:105700002968084420602068B04202D06FF065002C
:10571000DEE70020DCE72DE9F84F04460D4617468A
:105720009846DDF828B0DDF8309030236A462946E7
:105730002046FFF7FCFEB0F1000A02D05046BDE85B
:10574000F88F206800990844A84202D06FF06500E5
:10575000F5E72CE02168481C20600E7806EA070077
:10576000404502D06FF06100E9E76A4629462046CD
:10577000FFF79AFEB0F1000A01D05046DFE706EAD3
:105780000B000B9988420DD1B9F1000F0AD02268A5
:105790003146009B0D98C8478246BAF1000F01D0F0
:1057A0005046CCE7206800990844206000BF20687C
:1057B000A842CFD30020C2E7F0B504460E461546F6
:1057C0006FF06D0703232A4631462046FFF7AFFEF0
:1057D000071E01D03846F0BD286810B96FF0670089
:1057E000F9E72868401E28602068007810B16FF043
:1057F0006700F0E72068401C20600020EBE770B5F0
:10580000044605E0E56820461DF07EFE2C4600BFFC
:10581000002CF7D170BD2DE9F04705460E4617461E
:105820009846A946D9F80440A06858B11021012033
:105830001CF0EAFBE060E06818B96FF06900BDE8B1
:10584000F087E468A760C4F804802660C9F80440C3
:105850000020F4E7F0B587B006460F4614461D4613
:1058600005950694002020606060A060E06005A8B7
:10587000644900220092EBB2CDE901210390FF229E
:1058800039463046FFF747FF07B0F0BD2DE9F84332
:1058900004460F4616461D466FF06D0830236A46D3
:1058A00039462046FFF743FEB0F1000802D04046DB
:1058B000BDE8F8832068381A012802DA6FF05F002B
:1058C000F6E72068007830602068009947180623C2
:1058D000321D39462046FFF72AFEB0F1000801D0FC
:1058E0004046E5E72068B0602068716808442060A1
:1058F0002068B84205D10C2128460CF0DBFB0020C3
:10590000D6E72068007828602068401C20602A1DA7
:1059100039462046FFF7C8FDB0F1000801D04046E7
:10592000C6E72068A860206869680844206020688D
:10593000B84202D06FF06500BAE70020B8E7FEB5C4
:1059400004460D4616466FF06D070020009001904A
:1059500002906B46324629462046FFF797FF071E06
:1059600001D03846FEBD0098052801D0009808B93E
:10597000019810B16FF06700F4E70020F2E710B56E
:10598000044604B910BDA0681DF0BEFD60691DF09D
:10599000BBFD202120460CF08DFB00BFF2E770B567
:1059A00005460AE0A0692860A0681DF0ADFD6069A9
:1059B0001DF0AAFD20461DF0A7FD2C68002CF1D19A
:1059C00070BD70B5044604E0A56920461DF09CFD3D
:1059D0002C46002CF8D170BD70B504460E46154615
:1059E0000AE06068A84206D12A463146A0681CF049
:1059F000FEFA00B902E0A469002CF2D100BF2046F3
:105A000070BD00001758000830B503460C46012150
:105A1000802A05D3104601E0491C000A0028FBD16A
:105A20001868001B884202DA6FF06B0030BD00BFBF
:105A30001868401E18600270120A002AF8D1012965
:105A400006DD01F17F00C5B21868401E18600570C0
:105A50000846EBE703461868401A012802DA6FF09F
:105A60006B0070471868401E186002700120F8E74C
:105A70002DE9F0410746884614461E466FF06D0535
:105A800000BF224641463846FFF7BEFF051E02DA38
:105A90002846BDE8F0812C4400BF00BF3246414695
:105AA0003846FFF7D7FF051E01DA2846F1E72C44F8
:105AB00000BF2046EDE72DE9F04104460E46904632
:105AC0001D4600272068B04203D32068801BA842EF
:105AD00003D26FF06B00BDE8F0812F462068C01B39
:105AE00020603A46414620681CF012FA3846F2E738
:105AF0002DE9F04104460E4617466FF06D0800256B
:105B0000384600F072FE054605B901252068B0420E
:105B100003D32068801BA84203D26FF06B00BDE85E
:105B2000F0812068401B206000BF2A46384621686B
:105B300001F071FDB0F1000800D01DE000BFB88891
:105B4000012811D12068007800F0800060B1206841
:105B5000801B012802DA6FF06B00E0E7002120686B
:105B6000401E206001706D1C02232A4631462046EB
:105B7000FFF77EFF804600BF4046D0E770B5044681
:105B80000D460523002229462046FFF771FF70BD10
:105B90002DE9F04706460F46904699466FF06D0492
:105BA000002500BF4B46424639463046FFF783FF8B
:105BB000041E02DA2046BDE8F087254400BF062314
:105BC0002A4639463046FFF753FFF4E72DE9F05FE8
:105BD0000746884691469A46DDE90A6B6FF06D05E7
:105BE0000024BBF1000F0DD05EB900BF414638461E
:105BF000FFF7C4FF051E02DA2846BDE8F09F2C44DB
:105C000000E0344400BF53464A4641463846FFF759
:105C1000BFFF051E01DA2846EFE72C4400BF302302
:105C2000224641463846FFF723FFE6E72DE9FC41CF
:105C300004460D4616461F46DDF8208001203B46EF
:105C400032462946CDE900802046FFF7BFFFBDE878
:105C5000FC812DE9F04104460D46164600272068D8
:105C6000401B012803DA6FF06B00BDE8F0810EB134
:105C7000FF2100E000212068401E206001707F1C91
:105C800001233A4629462046FFF7F2FEEDE72DE9CB
:105C9000F04104460E4615469846002700BF20688E
:105CA000801B012803DA6FF06B00BDE8F0817F1CD8
:105CB0002068401E206005702D12002DEFDC20684A
:105CC000007800F0800060B12068801B012802DAB3
:105CD0006FF06B00E9E700212068401E2060017032
:105CE0007F1C08F0FF033A4631462046FFF7C0FE0E
:105CF000DBE770B504460D461646022332462946B8
:105D00002046FFF7C4FF70BD70B504460D46164629
:105D10000A23324629462046FFF7B9FF70BD2DE918
:105D2000F0478046894614461D46DDF820A06FF0F6
:105D30006D06002700BF53462A4649464046FFF7F6
:105D4000BAFE061E02DA3046BDE8F087374400BFCF
:105D5000E3B23A4649464046FFF78AFEF4E7F8B513
:105D600006460F4614461D4623460C223946304649
:105D70000095FFF7D4FFF8BDF8B506460F46144668
:105D80001D4623461322394630460095FFF7C7FFCC
:105D9000F8BDF8B506460F4614461D4623461622A2
:105DA000394630460095FFF7BAFFF8BD2DE9F047B8
:105DB00004460E46174698464FF0000A08F10700C1
:105DC000C508C8EBC5092068B04204D32068811B10
:105DD000681C814203D26FF06B00BDE8F08705F1CB
:105DE000010A95B16D1E795D012000FA09F0401E8F
:105DF00081432068401E206001702068401B2060A5
:105E00002A46394620681CF083F82068401E20602E
:105E100080F800900323524631462046FFF728FEC3
:105E2000DBE72DE9FF5F824690461C46E01DC50872
:105E3000C4EBC50BCCB108EB0500461E307840FA28
:105E40000BF700BF07F001097F10B9F1000F00D078
:105E50000AE0641E04B907E004F007000028F1D14D
:105E6000701E06460778EDE700BF234642465046BF
:105E70000199FFF79BFF04B0BDE8F09F2DE9F047C3
:105E800006460F46904699466FF06D04002500BF08
:105E90004B46424639463046FFF70DFE041E02DAF5
:105EA0002046BDE8F087254400BF04232A46394632
:105EB0003046FFF7DDFDF4E72DE9F04706468A4658
:105EC00017469846089D3A4651463068FFF784FDCC
:105ED000041E2FD1202101201CF096F8044614B98D
:105EE0000020BDE8F0876760394601201CF08CF87F
:105EF000A060A06820B920461DF006FB0020F0E756
:105F00003A465146A0681CF003F8256175B1294650
:105F100001201CF079F86061606938B9A0681DF053
:105F2000F3FA20461DF0F0FA0020DAE73068A061AD
:105F300034601AE02DB960691DF0E6FA0021616154
:105F400013E02069A84210D0294601201CF05CF81B
:105F50008146B9F1000F01D10020C2E760691DF050
:105F6000D3FAC4F81490256100BFB8F1000F05D032
:105F700025B12A46414660691BF0CAFF2046B0E7BA
:105F80002DE9F05F04460D4616461F46304600F0E8
:105F9000C8F900F0FF08384600F0C3F900F0FF0927
:105FA000A8EB04004FEA102AA5EB08004FEA102BDB
:105FB0004AEA0B0129EA0100BDE8F09F70B50546E9
:105FC000002405F14100C3B22A4619210020FFF741
:105FD000D7FF044305F14700C3B22A4633211A20F4
:105FE000FFF7CEFF0443281FC3B22A463D213420C9
:105FF000FFF7C6FF04432B232A463E210846FFF73E
:10600000BFFF04432F232A463F210846FFF7B8FF6E
:106010000443204670BD70B504460025A4F140003D
:10602000C3B222465A214120FFF7AAFF0543A4F13B
:106030004600C3B222467A216120FFF7A1FF054343
:10604000601DC3B2224639213020FFF799FF054376
:1060500004F11400C3B222462B210846FFF790FF3B
:10606000054304F11100C3B222462F210846FFF771
:1060700087FF0543681E40B270BD2DE9FF4F81B018
:1060800091461D460E9E2EB90020C9F8000005B0AD
:10609000BDE8F08F0320B6FBF0F00321B6FBF1F270
:1060A00001FB126109B1012100E0002100EB0108B0
:1060B000B8F1804F06D34FF0FF30C9F800006FF001
:1060C0002900E4E74FEA880808F1010102988842B4
:1060D00001D3019830B908F10100C9F800006FF050
:1060E0002900D4E70320B6FBF0F000EB40080027BE
:1060F000019C29E015F801AB15F801BB15F8010B5F
:1061000000904FEA9A00FFF759FF04F8010B4FEA9D
:106110000A1101EB2B1101F03F00FFF74FFF04F8CC
:10612000010B4FEA8B02009902EBA11101F03F0035
:10613000FFF744FF04F8010B009901F03F00FFF75F
:106140003DFF04F8010BFF1C4745D3D3B7422AD2C9
:1061500015F801AB781CB04202D215F8010B00E033
:1061600000208346CAF38500FFF728FF04F8010BDF
:106170004FEA0A1101EB2B1101F03F00FFF71EFF60
:1061800004F8010B781CB04207D23F2101EA8B00D2
:10619000FFF714FF04F8010B02E03D2004F8010BA7
:1061A0003D2004F8010B0198201AC9F800000020D6
:1061B000207000BF6BE72DE9FF4F83B08246934606
:1061C0001D4600200290814601900746044648E0A3
:1061D0000020019002E0641C01200190109884428C
:1061E00002D2285D2028F6D01098844200D13BE0EE
:1061F0001098001B022807D3285D0D2804D1601CCD
:10620000285C0A2800D12BE0285D0A2800D127E06D
:10621000019820B16FF02B0007B0BDE8F08F285D2A
:106220007F2802DD6FF02B00F6E7285D3D2807D1BF
:1062300009F101008146022810D96FF02B00EBE72D
:10624000B9F1000F02D06FF02B00E5E7285DFFF7F2
:10625000E2FE002802DA6FF02B00DDE77F1C00BFB2
:10626000641C10988442B3D300BF1FB90020CBF840
:106270000000D1E7F80800EB4000410007F00700FC
:1062800000EB40004000C01D01EBD007A7EB090761
:10629000BAF1000F02D00498B84204D2CBF80070D3
:1062A0006FF02900B8E74FF00009C846564630E0C5
:1062B00028780D2805D028780A2802D028782028A8
:1062C00000D124E04FEA881828783D2802D109F14E
:1062D000010904E02878FFF79EFE40EA08080298CA
:1062E000401C0290042811D1002002904FEA18406F
:1062F00006F8010BB9F1010F03D84FEA182006F890
:10630000010BB9F1000F01D106F8018B00BF641E2B
:106310006D1C002CCCD1A6EB0A00CBF800000020AD
:106320007AE7014601480068484070470C010020A8
:1063300070B50646304602F055F804466008404203
:10634000614240EA0105ED0F684270BD2DE9F0475A
:1063500004460F4690467E1C08F1010500BF20460A
:1063600002F040F86FEA000904EA060009EA0501B4
:10637000084300BF401E00B2BDE8F0872DE9F04F92
:1063800087B006460F469346F088F988884204D0C5
:106390006FF0030007B0BDE8F08F3179C1F3400022
:1063A000FFF7C6FF04463979C1F34000FFF7C0FF8D
:1063B000804600BF84EA080500BF2146284602F057
:1063C00016F881463068059038680690012004EA86
:1063D000000A00BFF2888AF001030DF1140C5CF88A
:1063E000231005AB53F82A0002F0B9F80490CDF859
:1063F0000890E8430190049901F0F9FF0390DDE96A
:10640000029049EA000081464846012100EA010263
:10641000CBF800200020BDE770B504460D4642F2DF
:106420001070854202D96FF00F0070BDE088A8425D
:1064300017D2042128461BF0E7FD061E02D16FF09B
:106440000F00F2E7206850B1E088820030462168F2
:106450001BF05EFDE288910020680BF036FEE580BF
:1064600026600020E1E72DE9F04704460D469046FE
:106470004FF0000900BFE9882046FFF7CDFFB0F1DB
:10648000000900D024E000BF4046FFF751FF064658
:10649000B4F90420B5F904103046FFF757FFA08087
:1064A000EA8829683346206802F098F83046C143EC
:1064B0000F46E88808E0226852F8201007EA010237
:1064C000216841F82020401CE1888142F3D800BFB8
:1064D0004846BDE8F0872DE9F04704460D461746CB
:1064E0004FF00008AC4202D10020BDE8F0873846EA
:1064F000FFF71EFF814600BFE9882046FFF78CFFAB
:10650000B0F1000800D022E000BF00BFE1882846BB
:10651000FFF782FFB0F1000800D018E000BFB4F927
:106520000460B4F90420B5F904104846FFF70EFFE3
:10653000A080B5F9042031464846FFF707FFA88040
:10654000E28829684B46206802F062F800BF4046A6
:10655000CBE7012181800021C1800160704710B527
:10656000044604B910BD206820B1E288910020687B
:106570000BF0ABFD0120A0800020E080206000BF78
:10658000F0E72DE9F04104460E4642F210708642D3
:1065900003D96FF00F00BDE8F081E088B04204D865
:1065A00031462046FFF738FFF5E7E088451E05E055
:1065B000206850F8250000B102E06D1E002DF7D1D3
:1065C00000BF6D1CB54200D23546042128461BF0A1
:1065D0001BFD071E02D16FF00F00DCE7206848B1F9
:1065E000AA00384621681BF093FCE28891002068DD
:1065F0000BF06BFDE58027600020CCE770B504460A
:106600000D4625B92046FFF7AAFF002070BDE0889F
:10661000A84207D1A90020681BF0A1FC0120A0809E
:106620000020F3E72046FFF79AFF29462046FFF7B0
:10663000F3FEEBE72DE9F04104460E460027B44295
:1066400002D10020BDE8F081F08850B9E08830B177
:106650000120A080E288910020681BF080FC0020CF
:10666000F0E7F088451E05E0306850F8250000B1DD
:1066700002E06D1E002DF7D100BF6D1CB088A08018
:10668000E088A84208D200BF29462046FFF7C4FE92
:10669000071E00D00EE007E0226802EB8500E288CA
:1066A000521B91001BF05BFCAA00316820681BF0B4
:1066B0002FFC00BF3846C5E70CB5D0E90023CDE973
:1066C0000023D1E90023C0E90023DDE90023C1E96B
:1066D00000230CBD70B504460D466FF06D0600BF7B
:1066E00001212046FFF798FE061E00D011E000BFF2
:1066F000E288910020681BF032FC284601F07BFE06
:1067000021680860E80F4042012101EB4000A080B1
:1067100000BF304670BD0246D088B1EB401F01D3A8
:10672000002070474B09106850F8230001F01F0348
:10673000D84000F00100F4E72DE9F04704460F4689
:1067400015464FF000097E0907F01F082DB1012DF5
:1067500003D06FF00300BDE8F087E088B7EB401F7F
:106760000CD30DB90020F6E700BF711C2046FFF7DF
:1067700053FEB0F1000900D014E000BF206850F8CB
:106780002600012101FA08F18843216841F826001A
:10679000206850F8260005FA08F10843216841F8FE
:1067A000260000BF4846D6E710B501460024002267
:1067B0000FE000230AE0086850F82200D84000F0FB
:1067C000010008B1204610BD5B1C641C202BF2D3D5
:1067D000521CC8889042ECD80020F4E710B504465B
:1067E000E188206801F05BFE10BD10B5044620462C
:1067F000FFF7F4FFC01DC00810BD0346FF2018605E
:10680000302A04DB392A02DCA2F130001860412A68
:1068100004DB462A02DCA2F137001860612A04DB9F
:10682000662A02DCA2F1570018601868884202D379
:106830006FF0050070470020FCE72DE9F0470546A2
:10684000894617466FF06D0ABD4203D14846A946F6
:10685000074600BF4D4509D000BF49462846FFF70F
:10686000E9FEB0F1000A00D047E000BF0120A88097
:10687000FC8806E0601E396851F8200000B102E093
:10688000641E002CF6D100BF14B90020BDE8F087CB
:1068900000BF21462846FFF7BFFDB0F1000A00D037
:1068A0002BE000BF2E682346314630463A6802F09E
:1068B00021F8804606EB84061BE0E888A0420CD84D
:1068C00000BF611C2846FFF7A7FDB0F1000A00D009
:1068D00013E000BF286800EB840630684044306055
:1068E0003068404501D2012000E000208046641C51
:1068F000361DB8F1000FE0D100BF5046C6E72DE9C4
:10690000F04705460E4690466FF06D09B8F8064010
:1069100007E0601ED8F8001051F8200000B102E036
:10692000641E002CF5D100BFF088A04202D26FF0A7
:10693000090941E000BFF1882846FFF76DFDB0F17D
:10694000000900D038E000BFF088A0420CD9AE4268
:106950000AD0336803EB84012B6803EB8400F388CF
:106960001B1B9A001BF0D4FAE888F188884208DDE6
:10697000EA88F388D21A91002A6802EB83001BF0A0
:10698000EEFAD8F8002031682346286802F002F8B1
:10699000074677B12A6802EB840102EB8400EA889B
:1069A000131B3A4602F09AFB074617B16FF009092C
:1069B00002E00120A88000BF4846BDE8F08770B51E
:1069C00003460C46D98806E0481E1D6855F820008D
:1069D00000B102E0491E0029F6D100BFE28806E0BE
:1069E000501E256855F8200000B102E0521E002A12
:1069F000F6D100BF914201D9012070BD8A4202D96F
:106A00004FF0FF30F9E717E0481E1D6855F8205099
:106A1000266856F82000854201D90120EDE7481E7E
:106A20001D6855F82050266856F82000854202D28D
:106A30004FF0FF30E1E7491E0029E5D10020DCE7F7
:106A40002DE9F04705460C4616461F46B4F904806A
:106A5000B4F90400B6F904104843784300282BDA4F
:106A600031462046FFF7ABFF8146B9F1000F13DB3B
:106A700000BF324621462846FFF741FFB0F1000A29
:106A800000D028E000BFB9F1000F01D1012000E0E3
:106A9000404600B2A8800EE000BF2246314628469C
:106AA000FFF72DFFB0F1000A00D014E000BFC8F1DD
:106AB000000000B2A8800DE000BF32462146284603
:106AC000FFF7BBFEB0F1000A00D004E000BF0FFAF0
:106AD00088F0A88000BF5046BDE8F08770B5044636
:106AE0000D4616460123324629462046FFF7A8FFE9
:106AF00070BDFEB505460E461446204601F07BFCEF
:106B00000090E00F4042012101EB4000ADF8080089
:106B10000120ADF80A00CDF804D001AA314628467C
:106B2000FFF7DCFFFEBD2DE9F84306460D4617468C
:106B3000EC8800E0641E2CB1601E296851F820002A
:106B40000028F7D007B12CB900213046FFF7C2FD6D
:106B5000BDE8F8836FF06D0800BF611C3046FFF799
:106B60005BFCB0F1000800D013E000BF00BF294675
:106B70003046FFF75FFDB0F1000800D009E000BF2C
:106B8000781E0090F1882A682346306801F02CFFB7
:106B900000BF4046DCE72DE9FF5F07468846154603
:106BA0006FF06D0003904FF0010BB8F1020F02DBA4
:106BB000B8F1100F04DD6FF0030004B0BDE8F09FE2
:106BC0006846FFF7C6FC287820B93846FFF7C7FCAF
:106BD0000020F2E728782D2802D16D1C4FF0FF3BF2
:106BE00028461BF0EFF90646B8F1100F47D1B6F171
:106BF000804F02D36FF00300DFE71F2000EA86001A
:106C000008B1012000E00020C6F3DA0100EB010A20
:106C100000BF51463846FFF7FFFB039000B165E027
:106C200000BF00BF00213846FFF754FD039000B1BC
:106C30005CE000BF34464FF000091DE000BF601E5D
:106C40002A5C414602A8FFF7D8FD039000B14DE051
:106C500000BF4FEAD901386850F821004FEA497166
:106C6000CA0E0299914008434FEAD902396841F8A7
:106C70002200641E09F10109002CDFD12BE000BFC6
:106C800000213846FFF726FD039000B12EE000BF3B
:106C900000241EE000BF2A5D414602A8FFF7ADFDBB
:106CA000039000B122E000BF00BF4246394668466B
:106CB000FFF739FF039000B118E000BF00BF69463D
:106CC0003846029AFFF715FF039000B10EE000BFAF
:106CD000641CB442DED3BBF1000F06DA3846FFF77E
:106CE0007DFD10B14FF0FF30B88000BF6846FFF760
:106CF00036FC039861E770B502460B46D18806E082
:106D0000481E156855F8200000B102E0491E002910
:106D1000F6D100BFDC8806E0601E1D6855F8200033
:106D200000B102E0641E002CF6D100BF11B90CB90D
:106D3000002070BDA14202D9B2F90400F9E78C42EB
:106D400003D9B3F904004042F3E7B2F90400002884
:106D500005DDB3F90400002801DA0120E9E7B3F901
:106D60000400002806DDB2F90400002802DA4FF022
:106D7000FF30DEE719E0481E156855F820501E6800
:106D800056F82000854202D9B2F90400D1E7481E26
:106D9000156855F820501E6856F82000854203D229
:106DA000B2F904004042C4E7491E0029E3D10020A3
:106DB000BFE73EB505460C46204601F01CFB00909F
:106DC000E00F4042012101EB4000ADF80800012036
:106DD000ADF80A00CDF804D001A92846FFF78BFFD3
:106DE0003EBD70B504460D46E08820B1E1882A46D4
:106DF000206801F0F4FC002070BD2DE9F04104464C
:106E00000D466FF06D072046FFF7E8FC4619E08855
:106E1000B6EB401F0FD900BF06F01F0008B10120DC
:106E200000E0002000EB56112046FFF7F5FA071EA0
:106E300000D007E000BF0027E1882A46206801F063
:106E40001AFD00BF3846BDE8F08170B504460D4616
:106E500016464FF0FF33324629462046FFF7F0FD35
:106E600070BD2DE9F05F06468B4691469A46B9F112
:106E7000000F01D04E450AD3BAF1000F03D04FF0F6
:106E8000FF30CAF800004FF0FF30BDE8F09F002748
:106E9000B046464647EA0B074A4600233846414675
:106EA0001AF0FAFF04460D460022D4F1FF30AA4141
:106EB00001D24FF0FF34BAF1000F04D0A4FB090156
:106EC000381ACAF800002046DFE72DE9F04F8FB0EE
:106ED0008146884616469A466FF06D000E90002156
:106EE0005046FFF766FF20B96FF00B000FB0BDE80A
:106EF000F08F0CA8FFF72DFB0AA8FFF72AFB08A8C4
:106F0000FFF727FB06A8FFF724FB0120ADF81400CC
:106F10000320ADF8160001A8049051463046FFF753
:106F20004EFD002819DAB9F1000F08D000BF00218A
:106F30004846FFF7CFFB0E9000B19CE100BFB8F1CF
:106F4000000F08D000BF31464046FFF773FB0E909C
:106F500000B190E100BF0020C8E700BF31460CA897
:106F6000FFF768FB0E9000B185E100BF00BF5146FE
:106F70000AA8FFF75FFB0E9000B17CE100BF012083
:106F8000ADF82C00ADF8340000BFF088811C08A8D3
:106F9000FFF742FA0E9000B16DE100BF00BF002183
:106FA00008A8FFF797FB0E9000B164E100BF00BF97
:106FB000F088811C06A8FFF72FFA0E9000B15AE165
:106FC00000BF0AA8FFF70AFC00F01F0BBBF11F0F60
:106FD00013D2CBF11F0B00BF59460CA8FFF70DFFD2
:106FE0000E9000B147E100BF00BF59460AA8FFF765
:106FF00004FF0E9000B13EE101E04FF0000BBDF840
:107000003600471EBDF82E00451E00BF781B41010B
:107010000AA8FFF7F2FE0E9000B12CE100BF12E0CB
:10702000791B089850F82100401C7A1B089941F8F8
:10703000220000BF0AAA0CA90CA8FFF706FF0E90B9
:1070400000B118E100BF0AA90CA8FFF754FE002800
:10705000E6DA00BF781B41010AA8FFF7C2FE0E90D6
:1070600000B108E100BF3C46CEE00C9850F8240087
:107070000A9951F82510884207D34FF0FF31601B61
:10708000401E089A42F8201011E00A9B53F8252070
:10709000631EDDF830C05CF823105CF82400002388
:1070A000FFF7DFFE611B491E089A42F82100022CFF
:1070B00001D2002003E0A01E0C9951F82000049991
:1070C00008600CB9002003E0601E0C9951F8200004
:1070D000049948600C9850F8240004998860601B5B
:1070E000401E089951F82000401C0A46611B491EA9
:1070F00042F8210000BF601B401E089951F8200093
:10710000401E0A46611B491E42F8210000BF0021B3
:1071100006A8FFF7DFFA0E9000B1ACE000BF0DB992
:10712000002003E0681E0A9951F8200006990860C3
:107130000A9850F825000699486000BF601B401E61
:10714000089951F8202006A906A8FFF7ECFC0E903C
:1071500000B190E000BF04A906A8FFF7CCFD00280D
:10716000C9DC00BF601B401E089951F820200AA905
:1071700006A8FFF7D8FC0E9000B17CE000BF00BF6E
:10718000601B401E410106A8FFF737FE0E9000B1BC
:1071900071E000BF00BF06AA0CA90CA8FFF755FEBE
:1071A0000E9000B167E000BF00210CA8FFF701FEC0
:1071B000002828DA00BF0AA906A8FFF73BFA0E90BC
:1071C00000B158E000BF00BF601B401E410106A88F
:1071D000FFF713FE0E9000B14DE000BF00BF06AAFE
:1071E0000CA90CA8FFF77AFC0E9000B143E000BF99
:1071F000601B401E089951F82000401E0A46611B82
:10720000491E42F82100641EAC423FF62EAFB9F190
:10721000000F0FD000BF08A94846FFF70BFA0E90E9
:1072200000B128E000BFB088BAF80410484300B2AB
:10723000A9F80400B8F1000F1CD000BF59460CA8F3
:10724000FFF7CFFD0E9000B115E000BFB088ADF89C
:10725000340000BF0CA94046FFF7ECF90E9000B1D6
:1072600009E000BF00214046FFF7A3FD10B901204F
:10727000A8F8040000BF0CA8FFF771F90AA8FFF7EF
:107280006EF908A8FFF76BF906A8FFF768F90C215B
:1072900001A80AF00FFF0E9828E6FEB505460E4637
:1072A00017461C46204601F0A6F80090E00F404229
:1072B000012101EB4000ADF808000120ADF80A0003
:1072C000CDF804D001AB3A4631462846FFF7FDFD24
:1072D000FEBDF0B504460B4612B96FF00B00F0BDD1
:1072E000002A02DA6FF00900F9E7012A01D0D888F4
:1072F00010B900202060F2E7022A06D11868007851
:1073000000F0010020600020E9E7DD88002114E0A2
:10731000681ED3F800C05CF82060080440EA1641FB
:10732000B1FBF2F707FB12113604080440EA1641DC
:10733000B1FBF2F707FB12116D1E002DE8D1B3F976
:107340000400002801DA01B1511A21600020C6E7CB
:107350002DE9F84F06460F46144698466FF06D0A21
:107360000025206800EB080900BF454503D36FF0F6
:107370000700BDE8F88F00BF3A4631466846FFF780
:10738000A8FFB0F1000A00D02EE000BF00BF3B46CE
:10739000324600213046FFF780FFB0F1000A00D0EE
:1073A00022E000BF00980A2807D200983030C1B20E
:1073B000A9F101008146017006E000983730C1B2A2
:1073C000A9F10100814601706D1C00213046FFF7D4
:1073D000F0FC0028C9D12A46494620681AF098FDD9
:1073E00020682844206000BF5046C2E72DE9FE4FC8
:1073F00006460D4617469846DDF830904FF0000AD5
:10740000022D01DB102D03DD6FF00300BDE8FE8FC0
:107410003046FFF7E3F90446042D00DB6408102D25
:1074200000DB6408641C641C641C04F00100044458
:10743000A04504D2C9F800406FF00700E6E70297C4
:107440006846FFF786F8B6F90400401C40B92D20C5
:10745000029908700298401C0290A8F10100804631
:10746000102D4ED1F1884FF0000C47E0042242E08D
:107470004B1ED6F800B05BF82330A2F1010B4FEAA7
:10748000CB0B23FA0BF3D8B230B9BCF1000F03D108
:107490008B18022B00D02DE003464FEAE07B00EB77
:1074A0001B7B4FEA2B1B0FF6546E1EF80BB0DDF85A
:1074B00008E08EF800B0DDF808B00BF1010BCDF854
:1074C00008B04FEAE07B00EB1B7B4FEA2B1BA0EBE5
:1074D0000B1B0FF6286E1EF80BB0DDF808E08EF8D7
:1074E00000B0DDF808B00BF1010BCDF808B04FF09B
:1074F000010C00BF521E002ABAD1491E0029B5D185
:107500001CE000BF31466846FFF794F8B0F1000A6E
:1075100000D01EE000BFBDF90400401C10B90120DE
:10752000ADF8040000BF434602AA29466846FFF7AB
:107530000FFFB0F1000A00D00BE000BF002002995D
:1075400008700298401C02900298C01BC9F8000005
:1075500000BF6846FFF703F8504657E72DE9F041B2
:1075600005460E4614466FF06D0804F0030008B19E
:10757000012000E0002000EB940700BF39462846B8
:10758000FFF73CF8B0F1000800D00DE000BF00BFED
:10759000E98823463246286801F05EF8B0F1000819
:1075A00000D001E000BF00BF4046BDE8F0812DE9FA
:1075B000F04105460E4614466FF06D0804F00300D6
:1075C00008B1012000E0002000EB940700BF39461D
:1075D0002846FFF713F8B0F1000800D00DE000BF17
:1075E00000BFE98823463246286801F060F8B0F110
:1075F000000800D001E000BF00BF4046BDE8F081B8
:1076000070B504460D461646E18833462A46206882
:1076100001F079F870BD70B504460D461646E18854
:1076200033462A46206801F0A2F870BDFEB5054633
:107630000E461446204600F0DEFE0090E00F404269
:10764000012101EB4000ADF808000120ADF80A006F
:10765000CDF804D001AA31462846FFF7F6FBFEBD5F
:107660002DE9F04786B00746884614466FF06D094D
:107670004FF0000A04A8FEF76CFF02A8FEF769FFAE
:1076800047450BD100BF414604A8FEF7D3FFB0F138
:10769000000900D058E000BF0DF11008A7420AD140
:1076A00000BF214602A8FEF7C5FFB0F1000900D0D7
:1076B0004AE000BF02ACB8F8065007E0681ED8F8F0
:1076C000001051F8200000B102E06D1E002DF5D130
:1076D00000BF0DB94FF0010AE68806E0701E216870
:1076E00051F8200000B102E0761E002EF6D100BF56
:1076F0000EB94FF0010A00BFA9193846FEF78CFEFB
:10770000B0F1000900D01FE000BF00BF00213846E3
:10771000FEF7E0FFB0F1000900D015E000BF0096D1
:107720002368D8F800102A46386801F09CFABAF1AC
:10773000000F02D00120B88005E0B8F80400A1884D
:10774000484300B2B88000BF02A8FEF708FF04A8B3
:10775000FEF705FF484606B0BDE8F0872DE9F04189
:1077600005460E4614466FF06D0700212046FFF7D0
:1077700020FB002803DA6FF00900BDE8F08100BFAC
:107780002346324629460020FFF79FFB071E00D004
:1077900023E000BF09E000BF224629462846FFF744
:1077A0009DF9071E00D018E000BF00212846FFF712
:1077B00000FB0028EFDB09E000BF224629462846EF
:1077C000FFF743FB071E00D007E000BF2146284615
:1077D000FFF791FA0028EFDA00BF3846CDE72DE930
:1077E000F04F87B005468A4617461C46109E6FF03C
:1077F0006D00069000212046FFF7DBFA002804DD2B
:107800002068007800F0010020B96FF0030007B095
:10781000BDE8F08F00213846FFF7CBFA002802DAE6
:107820006FF00300F3E73846FEF7D8FFB0F5005FCE
:1078300005D82046FEF7D2FFB0F5005F02D96FF001
:107840000300E4E7F88830B901212846FEF742FF3B
:1078500006900698DBE7F988E08801F06CFB81462A
:10786000042148461AF0D0FB8046B8F1000F02D13F
:107870006FF00F00CBE704A8FEF76BFE0EB1306887
:1078800070B900BF214604A801F069FA069000B162
:107890007BE000BF8EB1DDE90401C6E900010CE028
:1078A00000BFE1883046FEF7B7FD069000B16CE0FE
:1078B00000BFD6E90001CDE9040100BF51462846CA
:1078C000FEF7B8FE069000B15FE000BF0120A8807F
:1078D00021462846FFF70FFA002809DB00BF2246A1
:1078E00029462846FFF73AFF069000B14DE000BF59
:1078F00000BFE1882846FEF78FFD069000B144E006
:1079000000BF206801F0CEF983460498CDE900B0AD
:10791000CDF80880E38822682968084601F005FC54
:10792000F98804983A68CDE90208CDE90021E38896
:1079300022682968084601F051FBCDE900B8E388C8
:1079400022682968084601F004FCBAF90400401CCA
:10795000D0B93868007800F00100A8B1E98828683B
:1079600001F0D0FB83460122911E5846FEF7EEFC43
:10797000A88000BF2A4621462846FFF7AFF80690A8
:1079800000B102E000BF00BF00BF4FEA89014046DE
:107990000AF09BFB0EB1306810B904A8FEF7DFFDBA
:1079A000069834E72DE9FF470746884616466FF0EC
:1079B0006D0902A8FEF7CDFD6846FEF7CAFD00BFBF
:1079C000414602A8FEF736FEB0F1000900D08EE075
:1079D00000BF00BF31466846FEF72CFEB0F100093B
:1079E00000D084E000BF02A8FEF7DEFE0546684630
:1079F000FEF7DAFE044654B900216846FEF78BFE16
:107A000028B941463846FEF715FE81466FE0AC4284
:107A100000D225460120ADF80400ADF80C004BE083
:107A200000BF02A8FEF7C0FE8246514602A8FFF73B
:107A3000D8F9B0F1000900D059E000BF00BF684696
:107A4000FEF7B2FE824651466846FFF7CAF9B0F12A
:107A5000000900D04BE000BF694602A8FFF74BF9D0
:107A6000002814DB00BF6A4602A902A8FEF747FF00
:107A7000B0F1000900D03AE000BF00BF012102A828
:107A8000FFF7AFF9B0F1000900D030E014E000BF1B
:107A900002AA69466846FEF732FFB0F1000900D03D
:107AA00025E000BF00BF01216846FFF79AF9B0F159
:107AB000000900D01BE000BF002102A8FFF779F900
:107AC0000028ADD100BF29466846FFF796F9B0F10E
:107AD000000900D00BE000BF00BF69463846FEF742
:107AE000A9FDB0F1000900D001E000BF00BF02A86D
:107AF000FEF735FD6846FEF732FD484604B0BDE8A6
:107B0000F0872DE9F84305460C4616461F466FF0F0
:107B10006D0904F0030008B1012000E0002000EB33
:107B2000940800BF41462846FEF768FDB0F1000901
:107B300000D00DE000BF14B90020BDE8F883009725
:107B4000E98833462246286801F05EF9814600BF85
:107B50004846F2E72DE9FC4705460F46144698468D
:107B6000DDF82890002F03DA6FF00300BDE8FC87F2
:107B700039462046FFF71DF9002802DC6FF00300AC
:107B8000F4E7E1882846FEF739FD06460EB1304697
:107B9000ECE7CDE90089EB8822683946286801F0D6
:107BA00069F9E3E7F0B593B005460E4614466FF069
:107BB0006D0701212046FFF7FCF8002802DC781150
:107BC00013B0F0BD0FA8FEF7C4FC0DA8FEF7C1FC72
:107BD0000BA8FEF7BEFC09A8FEF7BBFC11A8FEF738
:107BE000B8FC07A8FEF7B5FC05A8FEF7B2FC03A891
:107BF000FEF7AFFC01A8FEF7ACFC00BF2246314601
:107C000011A8FFF7CFFE071E00D047E100BF0121FA
:107C100011A8FFF7CEF810B16FF00D073EE100BFDD
:107C2000224631460FA8FFF799FD071E00D035E127
:107C300000BF00BF0FA90DA8FEF7FCFC071E00D077
:107C40002CE100BF00BF214607A8FEF7F3FC071E8A
:107C500000D023E100BF00BF214605A8FEF7EAFCE3
:107C6000071E00D01AE100BF00BF01210BA8FEF7DC
:107C700031FD071E00D011E100BF00BF002109A89F
:107C8000FEF728FD071E00D008E100BF00BF00215D
:107C900003A8FEF71FFD071E00D0FFE000BF00BFD6
:107CA000012101A8FEF716FD071E00D0F6E000BF77
:107CB00000BF38E000BF01210DA8FFF792F8071EB2
:107CC00000D0EBE000BF0B98007800F0010020B975
:107CD0000998007800F0010098B100BF07AA0BA92D
:107CE0000BA8FEF7FBFE071E00D0D7E000BF00BFC9
:107CF0000FAA09A909A8FFF7A8F8071E00D0CDE030
:107D000000BF00BF01210BA8FFF76BF8071E00D0D2
:107D1000C4E000BF00BF012109A8FFF762F8071EF9
:107D200000D0BBE000BF0D98007800F001000028F3
:107D3000C0D038E000BF012105A8FFF752F8071EA8
:107D400000D0ABE000BF0398007800F0010020B93C
:107D50000198007800F0010098B100BF07AA03A9BC
:107D600003A8FEF7BBFE071E00D097E000BF00BFD0
:107D70000FAA01A901A8FFF768F8071E00D08DE03F
:107D800000BF00BF012103A8FFF72BF8071E00D09A
:107D900084E000BF00BF012101A8FFF722F8071E01
:107DA00000D07BE000BF0598007800F001000028BB
:107DB000C0D005A90DA8FEF79EFF00281DDB00BF5F
:107DC00005AA0DA90DA8FFF740F8071E00D065E031
:107DD00000BF00BF03AA0BA90BA8FFF736F8071EC8
:107DE00000D05BE000BF00BF01AA09A909A8FFF706
:107DF0002CF8071E00D051E01DE000BF0DAA05A918
:107E000005A8FFF722F8071E00D047E000BF00BF1B
:107E10000BAA03A903A8FFF718F8071E00D03DE03E
:107E200000BF00BF09AA01A901A8FFF70EF8071EAD
:107E300000D033E000BF00210DA8FEF7BAFF0028F4
:107E40007FF437AF09E000BF224603A903A8FEF77D
:107E500045FE071E00D021E000BF002103A8FEF769
:107E6000A8FF0028EFDB09E000BF224603A903A812
:107E7000FEF7EBFF071E00D010E000BF214603A86D
:107E8000FEF739FF0028EFDA00BF03A92846FEF706
:107E9000D1FB071E00D001E000BF00BF0FA8FEF716
:107EA0005EFB0DA8FEF75BFB0BA8FEF758FB09A8CD
:107EB000FEF755FB11A8FEF752FB07A8FEF74FFB94
:107EC00005A8FEF74CFB03A8FEF749FB01A8FEF747
:107ED00046FB384674E6F8B50546002703262868B1
:107EE000007800F0010010B96FF00D00F8BD00241B
:107EF00019E000BF324629466846FFF7EAF9071E37
:107F000000D013E000BF009848B931462846FEF77C
:107F100050FF08B90120E9E76FF00D00E6E7FC48E3
:107F2000005D0644641CA72CE3D300BF3846DDE7A0
:107F30002DE9FF4F8DB00446894693460AA8FEF707
:107F400008FB08A8FEF705FB06A8FEF702FB04A83D
:107F5000FEF7FFFA02A8FEF7FCFA00BF0122214655
:107F60000AA8FFF763FBB0F1000A00D0B6E000BF3B
:107F70000AA8FEF719FC064600BF0AA908A8FEF7E2
:107F800059FBB0F1000A00D0A8E000BF00BF3146A5
:107F900008A8FEF726FFB0F1000A00D09EE000BF5F
:107FA000002796E000200C9000BF00BFE088810011
:107FB0005A4604A8109BFFF7A4FDB0F1000A00D0B8
:107FC0008CE000BF04A8FEF709FC80460AA8FEF773
:107FD00005FC0546A84516D9BDF81600401E0499B3
:107FE00051F82010BDF81600401EA5EB4010401EB1
:107FF000012202FA00F0401E0140BDF81600401EAA
:10800000049A42F820100C98411C0C911E2802DDA5
:108010006FF00D0A62E00AA904A8FEF76CFE0028C2
:10802000C3DA012104A8FEF7C4FE0028BDDD00BFAD
:1080300002A8234608AA04A9009004A8FFF7CFFBD2
:10804000B0F1000A00D049E000BF0AA904A8FEF779
:1080500052FE20B1012104A8FEF7ABFE00B937E0C3
:108060004FF001081DE000BF04AA04A906A8FFF70D
:10807000F7FAB0F1000A00D030E000BF00BF22469E
:1080800006A904A8FFF76AFBB0F1000A00D025E0BA
:1080900000BF012104A8FEF78CFE00B909E008F139
:1080A0000108B04505D20AA904A8FEF724FE00285D
:1080B000D9D100BF0AA904A8FEF71DFE20B90121ED
:1080C00004A8FEF776FE10B96FF00D0A04E000BFB9
:1080D0007F1C4F45FFF466AF00BF00BF0AA8FEF744
:1080E0003EFA08A8FEF73BFA06A8FEF738FA04A8FD
:1080F000FEF735FA02A8FEF732FA504611B0BDE895
:10810000F08F2DE9FC4104460E46174698466FF065
:108110006D050120ADF80400E088ADF80600206888
:10812000009000216846FEF744FE20B10121684618
:10813000FEF73FFE18B96FF00D00BDE8FC8102218B
:108140006846FEF736FE08B90020F6E76846FFF7F6
:10815000C2FE051E05D0012D01D10020EDE7284605
:10816000EBE743463A4631466846FFF7E1FEE4E76F
:108170002DE9FF5F05460C4617469A46DDF838B0F4
:108180006FF00D08032C02D3B4F5005F04D96FF033
:10819000030004B0BDE8F09F6846FEF7DAF904F08A
:1081A0001F0008B1012000E0002000EB541607F08A
:1081B000020008BB40F21450844201D3022019E0AF
:1081C00040F25230844201D3032013E040F28A206F
:1081D000844201D304200DE0B4F5AF7F01D3082021
:1081E00008E0FA2C01D30C2004E0962C01D31220D5
:1081F00000E01B2003902BE040F2AA50844201D300
:10820000042024E040F27E40844201D305201EE099
:10821000B4F57A7F01D3062019E040F2523084424F
:1082200001D3072013E040F2EE20844201D308205E
:108230000DE0B4F5FA7F01D30D2008E0FA2C01D34C
:108240001C2004E0962C01D3282000E0332003906A
:10825000C2E000BFB1005B4652462846FFF751FC22
:10826000B0F1000800D0B8E000BF701E296851F8D6
:1082700020002849884200D2AEE04FEA4619A145C5
:108280000AD900BFA9EB04012846FEF7AAFDB0F108
:10829000000800D0A1E000BF2868006840F001009D
:1082A0002968086007F0010058B95B465246284625
:1082B0000399FFF726FF804608F10E0000286ED0D4
:1082C0008BE02868006840F002002968086000BF61
:1082D0000322294602A8FEF7FCFFB0F1000800D0F7
:1082E0007BE000BF0298C0B900BF0822294628469B
:1082F000FEF7FFFBB0F100080ED06EE030313233F4
:108300003435363738394142434445460000000091
:10831000C435020834F304B50DE0029801280AD1EF
:1083200000BF042229462846FEF7E3FBB0F100080F
:1083300000D052E000BF00BF29466846FEF77AF938
:10834000B0F1000800D048E000BF00BF012168463E
:10835000FEF747FDB0F1000800D03EE000BF39E075
:108360002846FFF7B8FDB0F1000819D16846FFF7BD
:10837000B2FDB0F1000813D15B465246284603997E
:10838000FFF7D6FDB0F100080AD15B4652466846B9
:108390000399FFF7CDFDB0F1000801D11DE01AE00F
:1083A00008F10E0000B118E000BF0C222946284653
:1083B000FEF79FFBB0F1000800D00EE000BF00BF49
:1083C000062269466846FEF794FBB0F1000800D02B
:1083D00003E000BFC4E700BF3BE76846FEF7BFF815
:1083E0004046D6E6014607480068484070470246C6
:1083F00002EA010070470146002901DB0846704788
:108400004842FCE70C01002070B50646304600F0FB
:10841000B6FE044660084042614240EA0105ED0FA5
:10842000684270BD2DE9F04104460D4616462046CF
:1084300000F0A5FEC74304EA050007EA0601084369
:10844000BDE8F0812DE9F04780460D46404600F03A
:1084500096FE0646284600F092FE044686EA04018F
:10846000C80FFFF7D1FF8146321B21464846FFF770
:10847000D9FF0746FF0F3846FFF7C6FFBDE8F08774
:1084800002464FF00041002005E002EA010303B17B
:1084900003E04908401C2028F7D300BF7047F0B51F
:1084A00005460E46741E0CE055F8240040B155F800
:1084B0002400FFF7E5FFC0F1200707EB4410F0BDF3
:1084C000641E002CF0DA0020F9E70146FC48007831
:1084D000012801D10846704708BAFCE72DE9F041B0
:1084E00006460F460FB9BDE8F0813446781E06EB0C
:1084F00080050BE02068FFF7E8FF80462868FFF75B
:10850000E4FF2060C5F80080241D2D1FAC42F1D986
:1085100000BFE8E72DE9F04704460D4617462E68F0
:1085200021463046FFF78EFFC0438046002000F012
:1085300026FE814601260AE055F82600FFF764FF73
:1085400082465146484600F02DFE8146761CBE42CA
:10855000F2D34146484600F025FEBDE8F0872DE9FC
:10856000F84F05460E469046002000F008FE814672
:10857000002000F004FE0090002000F000FE0746FE
:10858000444626E0621E55F8221056F82200FFF7F6
:1085900059FF00903846009900F004FE0746621E1D
:1085A00056F8221055F82200FFF74CFF009038468D
:1085B000C1438B46009800F0F1FD82465146484683
:1085C00000F0F0FD81463846009900F0EBFD0746CB
:1085D000641E002CD6D14846BDE8F88F2DE9F04145
:1085E00005460E4617469846B54201D1BDE8F081D2
:1085F000002409E055F8242056F82410404600F0E5
:10860000C3FD45F82400641CBC42F3D300BFEDE772
:108610002DE9F04705460E4617469846B54201D16A
:10862000BDE8F087002413E055F8249055F8242085
:1086300056F82410404600F0A7FD45F8240056F8EF
:1086400024204946404600F09FFD46F82400641C63
:10865000BC42E9D300BFE3E72DE9F04104460E46F2
:1086600017461D4605F0030008B1012000E0002078
:1086700000EB9508464503D26FF00700BDE8F08196
:108680009CB1B100204619F06AFC00200BE0820783
:10869000D10E820854F822203B5C8B401A43830899
:1086A00044F82320401CA842F1D30020E6E72DE93E
:1086B000F04706460C4617461D4605F0030008B174
:1086C000012000E0002000EB9508444503D26FF044
:1086D0000700BDE8F0870CB90020FAE7A10030469A
:1086E00019F03DFC4DB1C5EB8409B2460AEB090017
:1086F0002A46394619F00CFC00BF21463046FFF7E8
:10870000EDFE0020E5E72DE9F04707468946904653
:108710001C464FEA8905A54201D22E4611E02646A5
:1087200031460CE0880857F820008A07D20ED04066
:10873000C0B218B16FF00700BDE8F087491CA9422C
:10874000F0D3002008E0810857F821108207D20EEC
:10875000D14008F80010401CB042F4D3A54204D226
:10876000611B08EB050019F0FAFB0020E4E72DE996
:10877000F04780468A4617461D464FEA8A06AE42B3
:1087800008D234467819A0EB0409291B384619F0A1
:10879000E6FB12E02C46B94621460CE0880858F862
:1087A00020008A07D20ED040C0B218B16FF0070087
:1087B000BDE8F087491CB142F0D300200BE08108EE
:1087C00058F821108207D20ED140CAB2211A491E90
:1087D00009F80120401CA042F1D30020E8E72DE970
:1087E000F05F05460E4691464FF0000B4FEA5917D1
:1087F00009F01F08B74204D8B74208D1B8F1000FFA
:1088000005D0B100284619F0AAFBBDE8F09F8FB152
:10881000002405E0E01955F8200045F82400641C08
:10882000F01BA042F6D803E0002045F82400641CA9
:10883000B442F9D3B8F1000F1BD0344617E0601EE4
:1088400055F82000C8F1200100FA01FA601E55F821
:10885000200020FA08F0611E45F82100601E55F83E
:10886000200040EA0B0045F82100D346641E002C8E
:10887000E5D100BFC9E72DE9F04103460C460027CA
:10888000510902F01F05C1B120460AE0A0EB010C1E
:10889000ACF1010C53F82C80A0F1010C43F82C80B2
:1088A000401E8842F2D806E04FF00008A0F1010C0B
:1088B00043F82C80401E0028F6D1CDB1084615E0C3
:1088C0006C36020853F820C0C5F120082CFA08F6CF
:1088D00053F820C00CFA05FC43F820C053F820C020
:1088E0004CEA070C43F820C03746401CA042E9D3AD
:1088F000BDE8F081F0B505460C461E460023002079
:1089000018E054F82070F91854F820708F4201D9FB
:10891000012700E000273B4652F82070394452F806
:1089200020708F4201D9012700E000273B4445F821
:108930002010401CB042E4D31846F0BD2DE9F047AA
:1089400004460F469046994600254846FFF75CFDD1
:108950000646002019E057F8203006EA030C62466C
:1089600054F82030591954F820308B4201D9012392
:1089700000E000231D461144914201D2012300E092
:1089800000231D4444F82010401C4045E3D32846F2
:10899000BDE8F087F0B505461E46002300201FE025
:1089A00051F820C09C4502D24FF0010C01E04FF07D
:1089B000000C674651F820C0ACEB030452F820C00D
:1089C000A44502D94FF0010C01E04FF0000C0CEB74
:1089D000070352F820C0A4EB0C0C45F820C0401C43
:1089E000B042DDD31846F0BD2DE9FE4F044688465F
:1089F00016469C460C9F0025E04500D2C446A8EBD5
:108A00000C094FEADC0A0CF007000290F1E056F87E
:108A100004BBABFB071E7246084613462844A84217
:108A200002D24FF0010B01E04FF0000B5B44D4F891
:108A300000B05844D4F800B0834502D94FF0010B80
:108A400001E04FF0000B5B441D4601C456F804BB27
:108A5000ABFB0712084613462844A84202D24FF047
:108A6000010B01E04FF0000B5B44D4F800B0584418
:108A7000D4F800B0834502D94FF0010B01E04FF06C
:108A8000000B5B441D4601C456F804BBABFB071248
:108A9000084613462844A84202D24FF0010B01E0D9
:108AA0004FF0000B5B44D4F800B05844D4F800B049
:108AB000834502D94FF0010B01E04FF0000B5B44FE
:108AC0001D4601C456F804BBABFB0712084613460B
:108AD0002844A84202D24FF0010B01E04FF0000BF6
:108AE0005B44D4F800B05844D4F800B0834502D9B0
:108AF0004FF0010B01E04FF0000B5B441D4601C439
:108B000056F804BBABFB0712084613462844A8429C
:108B100002D24FF0010B01E04FF0000B5B44D4F8A0
:108B200000B05844D4F800B0834502D94FF0010B8F
:108B300001E04FF0000B5B441D4601C456F804BB36
:108B4000ABFB0712084613462844A84202D24FF056
:108B5000010B01E04FF0000B5B44D4F800B0584427
:108B6000D4F800B0834502D94FF0010B01E04FF07B
:108B7000000B5B441D4601C456F804BBABFB071257
:108B8000084613462844A84202D24FF0010B01E0E8
:108B90004FF0000B5B44D4F800B05844D4F800B058
:108BA000834502D94FF0010B01E04FF0000B5B440D
:108BB0001D4601C456F804BBABFB0712084613461A
:108BC0002844A84202D24FF0010B01E04FF0000B05
:108BD0005B44D4F800B05844D4F800B0834502D9BF
:108BE0004FF0010B01E04FF0000B5B441D4601C448
:108BF00000BFBAF10000AAF1010A7FF408AF19E042
:108C000008CEA3FB0723CDE900230098019928444F
:108C1000A84201D2012200E000221144226810443F
:108C20002268824201D9012200E0002211440D464F
:108C300001C400BF0298411E02910028E0D10AE061
:108C40002068284420602068A84201D2012000E06A
:108C500000200546241DB9F10000A9F10109EFD15A
:108C60002846BDE8FE8F2DE9F84306460F46144618
:108C70009846DDF8209004EB09008100304619F099
:108C80006EF900250AE058F82500009006EB8500F3
:108C900023463A46611CFFF7A7FE6D1C4D45F2D3F3
:108CA000BDE8F88301460A680878801C00F00400DB
:108CB00002EB4002202005E00B685343C3F102039E
:108CC0005A4340080828F7D2D043401C70472DE98A
:108CD000FF4F83B0074688469146139D119C600064
:108CE000401C8100284619F03AF900261BE058F88C
:108CF00026B02868D9F800100BFB010012994843F0
:108D00000190CDF800B04A46A11C2846069BFFF70B
:108D10006BFE019823460090A11C2846109AFFF78D
:108D200063FE2D1D761CA642E1D355F824A02346F0
:108D300029463846109AFFF72DFE029002998AEADA
:108D40000100FFF761FB0646A00000232A463946D2
:108D50000090304601F030F807B0BDE8F08F70B5F4
:108D600005460C466FF06D0600BF01212846FDF751
:108D7000B1FC061E00D01EE000BF00BFE0888101EC
:108D80002846FEF73AF8061E00D014E000BF00BFE8
:108D9000224629462846FEF7E1FC061E00D00AE0DE
:108DA00000BF00BFE1882846FDF7EBFB061E00D0A0
:108DB00001E000BF00BF304670BD2DE9FF4F81B01C
:108DC0000F46904699460E9C002518E02E4600BF9F
:108DD000304600F0D4F98246204600F0D0F98AEA05
:108DE000000B5846FFF710FBC0430090424639463F
:108DF000DDE90030FFF7F2FB6D1C07EB88074D45FE
:108E0000E4D305B0BDE8F08F2DE9F05F06460F46CC
:108E100015469946DDF828A06FF06D0B05F00300AC
:108E200008B1012000E0002000EB9504C5EB8408A8
:108E3000A74203D26FF00300BDE8F09F41463046E1
:108E400019F08DF83A1B910006EB840019F087F8B1
:108E500000BF06EB08012A465046C847B0F1000B98
:108E600000D005E000BF21463046FFF737FB00BFCA
:108E70005846E1E72DE9F04F85B00746884614468D
:108E80001D46DDF83CA04FF0FF3000F078F904906B
:108E9000002000F074F9039029462046FFF7FFFAFE
:108EA000814609F10700C6086FF06D000290042E9C
:108EB00001D91E2000E0FA20019000BF00BFCDF8CC
:108EC00000A03246294638460E9BFFF79DFF0290D0
:108ED00000B125E000BFC9EBC60229463846FFF7BE
:108EE0007EFC0198401E019018B96FF00D000290B1
:108EF00016E02A4639464046FFF70CFB04902A4606
:108F000021463846FFF72BFB0390DDE9031000F004
:108F100045F98346002000F032F98345CED000BFEA
:108F2000029805B0BDE8F08F01464F2901D9032012
:108F300070470120FCE72DE9F04704460D46680123
:108F4000FFF7F2FF0746012000FA07F808FB04F9D3
:108F50002646600000F1010A09EB06005044BDE816
:108F6000F0872DE9F04F87B081460E4614461F4624
:108F7000DDE9125AA100284618F0F1FF012028600F
:108F80002346CDE9027ACDE9006429462846109AA5
:108F9000FFF79DFE05EB8408A2004946404618F005
:108FA000B7FFC3460220069011E00BEB840005904A
:108FB000234642465946CDE9027ACDE90064059838
:108FC000FFF785FEDDF814B00698401C0690119955
:108FD00006988842E9D307B0BDE8F08F2DE9FF4F2E
:108FE0008DB0804615461C46DDF874901B994801EB
:108FF000FFF79AFF0C9001210C9881400B910B9880
:1090000060430A900994CDF82090DDF820900A98EA
:1090100009EB80000790099C079800EB84000690FC
:109020002846FFF73FFE8246DDF820900B9A1C99F8
:10903000069853468DE806020390224629460E986C
:10904000FFF78FFFA2004046089918F061FF1B9FB1
:10905000002600200590834600BF0698234642461E
:109060004146CDE9014A009503904046FFF72FFEA7
:1090700016B97F1E1F2600E0761E0598401C05903D
:109080004FEA4B0B1A9850F82700F04000F001000F
:1090900040EA0B0B0C990598884201D0BEB9B7B9CC
:1090A000CDF800B022460B9BDDE90701FFF785FEF6
:1090B00006982346CDE9014A009503904146404673
:1090C000079AFFF704FE4FF0000B00200590002EDA
:1090D000C3D1002FC1D111B0BDE8F08FF0B5044667
:1090E00000200BE051F82050AE1AAE4201D9012702
:1090F00000E000273A4644F82060401C9842F1D333
:109100001046F0BD2DE9F04104460D4627460026E5
:10911000002003E057F820100E43401CA842F9D36A
:109120003046FFF771F9BDE8F0812DE9FF470646AB
:109130000F4614461D46DDE90D9ADDF830802B46BA
:109140004A46394630468DE83005FFF7C0FDBDE898
:10915000FF872DE9F04385B006460F4614461D46AD
:10916000DDE90C8901200490012304AA3946304628
:109170008DE83003FFF7ABFD05B0BDE8F083014695
:109180000A4800684840704770B504460D461646C8
:10919000324629462046FFF745F970BD024602EAED
:1091A00001007047024642EA010070470C010020AE
:1091B000FE48006860B9FE4AFE4902E012F8080B5A
:1091C00001C110780028F9D108600120F74B186020
:1091D000F84870470246F64905E00878904201D108
:1091E00048687047083148680028F6D100BFF8E7A2
:1091F00070B505460DB9002070BDED4C08E0616802
:109200000868294618F0E5FE08B96068F4E70834F4
:1092100060680028F3D100BFEEE72DE9F041054674
:109220000E461746E24C14E0606800F028FC007817
:10923000A8420DD1606800F00FFCB04208D1606810
:109240008088C0F30330B84202D16068BDE8F08185
:10925000083460680028E7D100BFF7E710B504467E
:109260004021204618F07BFE10BD70B5044604B9BD
:1092700070BDE06B30B1206800F001FC8669E56BE1
:109280002846B0474021204608F014FF00BFEFE712
:1092900070B504460D460DB9C74870BD4021204643
:1092A00018F05DFE284600F0EAFB406950B1284600
:1092B00000F0E5FB4669B047E063E06B10B9BE48DB
:1092C0008038EAE725600020E7E72DE9F04704460B
:1092D0000F4616461D46012D03D015B1B648BDE810
:1092E000F087206808B9B448F9E720684068000EA4
:1092F00000F0020030B9206800F0AEFBB04201D0AF
:10930000AD48ECE766602572012D11D02068808899
:10931000C0F3033003280BD020688088C0F30330EB
:10932000042805D020688088C0F3033005280DD1BB
:10933000206800F0A4FBD0F80CA0D4F804804246CA
:109340003946D4F83C904846D047C8E76DB9206804
:1093500000F095FBD0F810A0D4F8048042463946BE
:10936000D4F83C904846D047B9E79348B7E72DE991
:10937000F04104460F461546206810B98E48BDE8F6
:10938000F081102D02D98C488030F8E720684068C1
:10939000C0F3006008B12E460CE0206808B9002137
:1093A00003E00179C1F3421189000E46AE4201D9B2
:1093B0008148E4E720688088C0F30330062807D19D
:1093C00094F908102B463A46E06B04F0D4FBD6E73C
:1093D00036B13246394604F1280018F099FDA663EB
:1093E0000020CCE70146086808B9734870470020A0
:1093F000486200BFFAE770B504460D46164620687D
:1094000008B96D4870BD20688088C0F30330062815
:1094100005D132462946E06B04F03AFCF2E7664893
:109420008030EFE72DE9F04F85B0044689461546B8
:109430009A460E9F6FF06D000490206818B95E4840
:1094400005B0BDE8F08F00203860204600F00DFB2D
:1094500006460EB95948F3E720688088C0F3033008
:1094600001281AD1B54201D05548E9E73D6020688E
:1094700000F005FB4068039094F9088053464A4683
:109480004146D4F83CB05846DDF80CC0E0470490A3
:1094900008B10498D4E70020D2E720688088C0F3A0
:1094A0000330062808D1CDE9005753462A464946DD
:1094B000E06B04F0CBFCC3E7D14508D1606A20B96A
:1094C000B5FBF6F006FB105008B13B48B8E7206842
:1094D0008088C0F30330022867D14FF00008207A5B
:1094E00028B9E06818B1606A301AA8420ED2207A12
:1094F00028B9E06818B9606A301AA84206D8207AFC
:10950000012810D1606A301AA8420CD904F1140164
:10951000626A50182A46494618F0FAFC606A2844E4
:10952000606200208CE7606A50B3606AA6EB0008B6
:1095300004F11401626A50184246494618F0E8FCEA
:1095400004F11400CDE9000A206800F098FAD0F880
:1095500008B094F908000390E06B04F12803324648
:1095600002900399D847049008B1049868E73868D6
:1095700030443860B24400206062C144A5EB080565
:109580003DB3B5FBF6F006FB1058B8F1000F04D15F
:10959000207A10B9E06800B1B046A5EB080000EBF6
:1095A0000901424604F114000CE02DE0F400002013
:1095B0007437020870090020009FFFFF809CFFFFA6
:1095C000809DFFFF18F0A4FC606A40446062A5EB38
:1095D0000805BDB1CDE9009A206800F050FAD0F836
:1095E00008B094F908000390E06B04F128032A46C0
:1095F00002900399D847049008B1049820E738688E
:109600002844386000201BE7FD4819E7034603B1F2
:1096100012B9FB488038704711600020FBE72DE944
:10962000FC5F04460D461646206818B9F448803899
:10963000BDE8FC9F0020306020688088C0F30330C4
:10964000022804D1206910B9ED488038F0E720687D
:109650008088C0F30330032823D020688088C0F3BB
:10966000033004281DD020688088C0F3033005280B
:1096700017D020688088C0F30330062811D02068F6
:109680008088C0F3033009280BD020688088C0F39D
:1096900003300A2805D020688088C0F303300728EB
:1096A00001D10020C4E720684068C0F307404C287F
:1096B00005D020684068C0F307404D2801D1002044
:1096C000B6E720688088C0F30330012805D1606ABE
:1096D00008B1CC48ACE70020AAE720688088C0F336
:1096E000033002285CD10027207A01281DD1E068D0
:1096F00028B9606A08B1C3489AE7002098E700BF1C
:10970000206808B9002008E0A06B08B1A06B04E055
:1097100020680079C0F3421080008046414604F181
:109720001400E368626A98470DE0204600F09DF956
:10973000616A884207D0E06818B9606A08B90020F9
:1097400076E7B04874E7204600F08FF9834604F1CD
:109750001400CDE90005206800F091F994F9088023
:10976000D0F808A004F128035A464146D4F83C90AA
:109770004846D047071E01D0384659E7207A48B9F5
:10978000204600F072F98046324641462846236959
:1097900098474DE7204600F068F93060002047E721
:1097A000974845E70246106828B110688088C0F3E2
:1097B0000330022802D0924880387047042904D12F
:1097C0000020D0609048106101E08D48F5E700BFAF
:1097D0000020F2E7FEB504460D461646206810B993
:1097E00087488038FEBD207A012802D0844880381E
:1097F000F8E720688088C0F30330062808D1CDE957
:10980000005602AB00221146E06B04F0FBFBE9E7D7
:109810007B48E7E7F0B587B004460E4615466FF083
:109820006D07206818B97648803807B0F0BD207AF7
:1098300010B173488038F8E7714F20688088C0F312
:10984000033006281BD1102D02D96D488038ECE773
:1098500003A8CDE9000502AB00221146E06B04F03D
:10986000D1FB071E01D03846DFE72A4603A9304660
:1098700000F03EFA10B1634F803F01E000BF00BF2F
:10988000294603A808F016FC3846CEE72DE9FC5F10
:109890000746884691461D46DDE90CA60E9C6FF0F2
:1098A0006D0B4A4641463846FFF761FDB0F1000BAB
:1098B00002D05846BDE8FC9F3846FFF793FDB0F153
:1098C000000B01D05846F5E7334652462946384644
:1098D0000094FFF7A7FDB0F1000B01D05846E9E76F
:1098E0002068811901AA3846FFF799FEB0F1000BF4
:1098F00001D05846DEE72068019908442060002026
:10990000D8E72DE9F04F87B004460D4616461F46AE
:10991000DDE9128BDDE9109A20688088C0F30330FE
:10992000062811D11498C0F80080DDE915018DE8F2
:10993000C00ECDE905102B4642460121E06B04F034
:1099400020FC07B0BDE8F08F2D48FAE72DE9F04F75
:1099500087B004460D4616461F46DDE9128BDDF83A
:1099600044A020688088C0F3033006281FD16FF020
:109970006D091498C0F80080DDE91501CDE904AB4C
:10998000CDE902011098CDE9007033462A464146E0
:10999000E06B04F035FC814609F1120018B9DFF8DC
:1099A0006490A9F18009484607B0BDE8F08F1448DB
:1099B000FAE72DE9FF4F87B08146DDE9177BDDE946
:1099C00015A4DDE91956A019584504D90C4880386A
:1099D0000BB0BDE8F08F3819CDE90375CDE9050668
:1099E0001498CDE901A40090484608A90EC9FFF7D4
:1099F00088FF80462868304428604046E8E7000039
:109A0000809FFFFF809DFFFF0D9600082DE9FF4F0F
:109A100087B007468846DDE917ABDDE91496169D49
:109A20001A9CA54202D3281B584503D918480BB0ED
:109A3000BDE8F08F7019001B1999CDE903A1CDE99C
:109A40000504281BCDE90096029041463846DDE921
:109A50000923FFF77BFFEAE7014609B900207047B9
:109A60008888C0F303208001F9E70146086808B937
:109A7000002070470868007900F01F00F9E70146F0
:109A80004868C0F38460034A52F820007047000021
:109A9000009FFFFFF800002010B54FF4C4710120B3
:109AA00018F0B2FA044614B1204603F0FDFD20463A
:109AB00010BD10B50446204604F0D8FB204619F02E
:109AC00023FD10BD2DE9F04104460D4616461F4604
:109AD0003B4632462946204616F04FF8BDE8F08155
:109AE0002DE9FC4704460D4616461F46DDE90A8966
:109AF0003B46324629462046CDE9008916F085F8D6
:109B0000BDE8FC8770B504460D4616463246294628
:109B1000204616F025F870BD70B504460D46164671
:109B200032462946204616F00DF870BD10B52821A2
:109B3000012018F069FA04460CB9002010BD204637
:109B400015F0F2FF2046F9E710B50446204615F05F
:109B5000F2FF204619F0D8FC10BD70B506460C4641
:109B600015462B4622460221304603F0DDFE70BD2D
:109B70002DE9F04106460F4614461D462A46214669
:109B8000304616F0C7F8BDE8F0812DE9F0410646F1
:109B90000F4614461D462A462146304616F049F91E
:109BA000BDE8F0812DE9FC4704460D4616461F46E8
:109BB000DDE90A893B46324629462046CDE900893F
:109BC00016F0CEF8BDE8FC872DE9FC4704460D46AB
:109BD00016461F46DDE90A893B463246294620469D
:109BE000CDE9008916F04BF9BDE8FC8770B5044655
:109BF0000D4616462946204616F083F870BD70B50E
:109C000004460D4616462946204616F071F870BDEA
:109C100070B504460D4616462946204616F085F9CD
:109C200070BD70B504460D4616462946204616F00E
:109C300069F970BD70B504460D46164629462046A2
:109C400016F0EBF870BD70B504460D461646294671
:109C5000204616F0D6F870BD10B51021012018F07E
:109C6000D3F904460CB9002010BD204616F034F894
:109C70002046F9E710B50446204616F033F8204692
:109C800019F042FC10BD10B52021012018F0BCF9DC
:109C900004460CB9002010BD204616F0A4F820465A
:109CA000F9E710B50446204616F0A4F8204619F04E
:109CB0002BFC10BD70B50646304600F0D1F80446C6
:109CC00060084042614240EA0105ED0F684270BD04
:109CD0002DE9F04104460D461646204600F0C0F836
:109CE000C74304EA050007EA06010843BDE8F0811E
:109CF0002DE9F04103460C46154600211E46274635
:109D0000002207E016F801C0785C8CEA000848EAF7
:109D10000202491CA942F5D390B240EA1240BDE8C4
:109D2000F0812DE9F74F82B00C46029E00253EE0FF
:109D30000498A4EB000800BF284600F091F8824682
:109D4000404600F08DF881468AEA0901C80FFFF706
:109D5000B1FF0190AAEB090249460198FFF7B8FF4D
:109D600083464FEADB7B5846FFF7A4FF00BF074658
:109D70004FF0000811E016F808B008F10100305C5F
:109D80000190D946DDF804A0524649463846FFF70F
:109D90009FFF06F8080008F10108601E4045EAD858
:109DA000611E705C07EA0001601E31546D1CA54203
:109DB000BED305B0BDE8F08F2DE9F05F07460D4634
:109DC00090461E46DDF82890BA46384600F048F81E
:109DD0006FEA000B06B92E46002409E018F80400CB
:109DE00000EA0A00315D01EA0B0108432855641CB2
:109DF0004C45F3D3BDE8F09F2DE9FC5F074688464C
:109E0000154699464C4619E0264600BF304600F0FC
:109E100027F88246284600F023F88AEA000B5846C5
:109E2000FFF748FFC04301900D9808EB04020023A0
:109E3000394600900198FFF7BFFF641C0C988442DC
:109E4000E2D9BDE8FC9F70B50346DD430C46002017
:109E500003E0265C2E402654401C9042F9D370BD8E
:109E60000146024800684840704700000C0100208D
:109E700070B50446002004E00D5C165C7540255466
:109E8000401C9842F8D370BD70B50546032400BF4E
:109E9000F7480078012804D105EB840000F0A6FA09
:109EA00004E005EB840000F0A1FA00BA0646761C37
:109EB000EF480078012805D105EB8400314600F019
:109EC00098FA04E005EB840031BA00F092FA06B982
:109ED00004B901E0641EDBE700BF70BD10B50446A5
:109EE0005021204618F03BF804F1200015F01CFE2C
:109EF0004FF0FF30206142F21070E06110BD10B5EC
:109F0000044604B910BD04F1200015F014FE5021E0
:109F1000204608F0CFF842F21070E0614FF0FF30B9
:109F2000206100BFEEE741617047816170470246E2
:109F3000906C10B16FF033007047B1F5C07F02D95B
:109F40006FF03700F8E7B1F1004F02D36FF0370040
:109F5000F2E711610020EFE7C16170472DE9F74F8B
:109F6000ADF50C7D8246154600200B90B5F5C07FFF
:109F700005D96FF037000DF50F7DBDE8F08F4FF478
:109F8000D07124A817F0EBFF28ACB948007801285D
:109F900004D12946204600F02CFA03E029BA2046D5
:109FA00000F027FAE41D302004F8010B2A46204671
:109FB0008D9917F0ADFF8020605505F1190B002732
:109FC00002E010A9CF557F1C202FFADB01A815F065
:109FD000ABFD4FF4807210A901A815F0B3FD0B90F2
:109FE00000B154E000262FE024AC00200C900D902E
:109FF0000E900F90D94617E0102322460CA90CA80A
:10A00000FFF736FF1034B9F1100F01D3102000E034
:10A010004846A9EB00090CAB0CAA012101A815F0D8
:10A02000ACFD0B9000B132E0B9F1000FE4D118A9FA
:10A03000881910220CA917F06BFF9DF89300401CA3
:10A04000C0B28DF893001036302ECDDB4FF4807205
:10A0500018A901A815F076FD0B9000B117E00DF1DD
:10A060008008544600260FE043464246012101A8DD
:10A0700015F083FD0B9000B109E010224146204607
:10A0800017F046FF10341036302EEDDB00BF01A86C
:10A0900015F051FD4FF4D07124A808F00BF83021D1
:10A0A00018A808F007F8202110A808F003F81021DC
:10A0B0000CA807F0FFFF0B9818B13021504607F0AD
:10A0C000F9FF0B9857E72DE9F0418CB004460D4697
:10A0D0006E464FF000083021684617F040FF002719
:10A0E0000FE02046FFF7D0FE33462246012104F15F
:10A0F000200015F042FDB0F1000800D019E0103644
:10A100001037302FEDDB30232A4669466846FFF7CB
:10A11000AFFE4FF48072694604F1200015F012FD85
:10A12000B0F1000800D004E008A80FC884E80F00D0
:10A1300000BF3021684607F0BDFF40460CB0BDE8C7
:10A14000F081F0B58DB005460E4614466FF06D07F0
:10A1500014B900200DB0F0BD2246314601A8FFF72A
:10A16000FDFE071E00D007E001A92846FFF7ABFF60
:10A17000071E00D000E000BF302101A807F09AFFC1
:10A180003846E7E72DE9F043E1B004468846174634
:10A190001D4600266FF06D09A069B0F5C07F04D997
:10A1A0006FF0370061B0BDE8F083A069C0F5C07002
:10A1B000A84202D26FF03700F4E7A069C0F5C07082
:10A1C000401BB84202D26FF03700EBE74FF4C0718A
:10A1D00001A817F0C4FE01A9D4E91230A26998477A
:10A1E00010B16FF03300DDE7A069064455B101AA54
:10A1F00091192A46D4E91230984710B16FF0330014
:10A20000D0E72E44B8F1000F07D037B101A9881963
:10A210003A46414617F07CFE3E44324601A901A869
:10A22000FFF79CFEB0F1000900D00AE001A920462A
:10A23000FFF749FFB0F1000900D002E001202061E2
:10A2400000BF4FF4C07101A807F034FF4846A9E7EA
:10A2500070B504460D461646002332462946204670
:10A26000FFF790FF70BD0146302903D300207047EF
:10A27000F4370208481C4008F9E72DE9F04788B098
:10A2800004460D4616461F46DDF840806FF06D0906
:10A290002021684617F063FEA564E664A06908B94A
:10A2A0002020A0612069002801DB206902E0A0696C
:10A2B000FFF7D9FF82464FF48072694604F120000F
:10A2C00015F040FCB0F1000903D0484608B0BDE8E5
:10A2D000F0875346424639462046FFF753FFB0F118
:10A2E000000901D04846F1E70020EFE72DE9F04FE3
:10A2F00091B08046894615469A461A9E00201090D5
:10A300004446CB46B5F5806F04D96FF0350011B0E7
:10A31000BDE8F08FB6F5807F02D96FF03700F6E721
:10A320003021684617F01BFEE1692069884201DC94
:10A33000606948B1324651462046FFF789FF1090C8
:10A3400008B11098E3E7002676B1324651466846D8
:10A35000FFF704FE109000B12EE069462046FFF79B
:10A36000B2FE109000B127E019E02046FFF78CFD07
:10A370000CAB2246012104F1200015F0FEFB1090E9
:10A3800000B119E0102D01D9102000E02846074641
:10A390003A460CA9584617F0BBFDBB44ED1B002DF7
:10A3A000E3D169462046FFF78EFE109000B103E02E
:10A3B0002069401C206100BF4021684607F07AFEFA
:10A3C0001098A4E72DE9F84304460D4616466FF0B1
:10A3D0006D07A046002003463246294600904046BD
:10A3E000FFF784FF07463846BDE8F8830146086852
:10A3F00070470160704700002DE9F04780460C4629
:10A4000016462068301A022802DAF748BDE8F087BD
:10A41000F6480078012803D1206800F05EFC08E0CF
:10A42000206800F05AFC05462806000C40EA15207A
:10A4300000BF07462068801C20602068301AB842A0
:10A4400001D2E948E2E73A4640462168FDF7AFF815
:10A45000B0F1000907D03B23E5A24946E248803825
:10A4600000F042FCD2E72068384420600020CDE7AD
:10A470007CB504460D4600266846FCF76AF800BF26
:10A48000022229466846FDF7D1F8061E00D00EE0EC
:10A4900000BF02212046FCF78CFC002805DB694642
:10A4A0002046FCF728FC002800DDCF4E00BF6846A0
:10A4B000FCF755F830467CBD10B5044650212046C7
:10A4C00017F04DFD10BD10B504462046FCF786F987
:10A4D00010BD10B504462046FCF787F910BD2DE9E4
:10A4E000F04104460D4616460027062D15D2DFE83A
:10A4F00005F00305080B0E11274611E004F10807CB
:10A500000EE004F110070BE004F1180708E004F175
:10A51000200705E004F1280702E0B348BDE8F08118
:10A5200000BF39463046FCF785F8F7E72DE9F041E2
:10A5300004460D4616466FF06D0732462946204602
:10A54000FFF75AFF071E0FD13246294604F10800D3
:10A55000FFF752FF071E07D13246294604F12000BB
:10A56000FFF74AFF071E02D03846BDE8F0812146BA
:10A5700004F12000FFF77CFF071E01D03846F4E706
:10A580000020F2E72DE9F84304460D4616461F4623
:10A5900000BF33462A46032120460097FDF7DAFA2A
:10A5A000B0F1000800D00CE000BF00BF012221463E
:10A5B0002046FDF73BF8B0F1000800D001E000BFF5
:10A5C00000BF4046BDE8F8832DE9F84304460D4638
:10A5D00017469846002600212046FCF7EAFB10B9F2
:10A5E0008148BDE8F883002D01DA7F48F9E720466D
:10A5F000FCF7FBF8A8420BD900BF43463A46294670
:10A6000004F11000FDF77DFA061E00D02AE00FE0ED
:10A6100043463A46214604F11000FFF7B3FF0646D1
:10A6200006F10E0008B97948DBE70EB13046D8E7ED
:10A6300000BF04F13000234604F1100204F10801C8
:10A6400000901838FDF7CBF8061E00D00AE000BFD6
:10A65000214604F11800FFF70BFF061E01D030461B
:10A66000BFE700BF3046BCE72DE9FF5F06469246D4
:10A670009B463046DDE90E230199FFF7A5FF07460B
:10A6800007B14DE03046FCF7B0F8804606F108000F
:10A69000FCF7ABF8814606F11800FCF7A6F8054672
:10A6A000544600BF00BF4246A11C3046FCF7B3FF32
:10A6B000071E00D034E000BF4FEA182004F8010B59
:10A6C00004F8018B444400BF00BF00BF4A46A11CF0
:10A6D00006F10800FCF79FFF071E00D020E000BF36
:10A6E0004FEA192004F8010B04F8019B4C4400BF09
:10A6F00000BF00BF2A46A11C06F11800FCF78BFF23
:10A70000071E00D00CE000BF280A04F8010B04F873
:10A71000015B2C4400BFA4EB0A00CBF8000000BF93
:10A7200057B117F1800F07DD4FF4847330A239461B
:10A73000364800F0D9FA0746384604B0BDE8F09F25
:10A740002DE9F04104460E4615466FF06D0731467F
:10A750002046FBF76FFF071E06D1294604F10800CB
:10A76000FBF768FF071E08D04FF48C7320A2394610
:10A77000274800F0B9FABDE8F0810020FBE72DE999
:10A78000F04105460E4614466FF06D0724B1284689
:10A79000FFF79FFEA04202D21348BDE8F081224697
:10A7A000314605F12000FCF702FF071E08D040F2F9
:10A7B0002B130FA239461548803800F095FAECE7C4
:10A7C0000020EAE72DE9F0470646884617461D4671
:10A7D000DDE9089A25B13046FFF77BFEA84219D281
:10A7E0000148BDE8F087000080CFFFFFF637020880
:10A7F0002E2E5C6D626564746C735C6C6962726150
:10A8000072795C64686D2E630000000080CEFFFFEB
:10A8100080CAFFFF53464A4641463046FFF7D4FE02
:10A82000044614F5465F02D1FE48BDE8F08704B146
:10A830000BE000BF2A46394606F11800FCF7EBFE94
:10A84000041E00D001E000BF00BF5CB114F1800F16
:10A8500008DD40F24B13AFF268022146F14800F0E8
:10A8600043FA04462046E0E7FEB504460E46174686
:10A8700001A8FBF76EFE04F1480104F11000FCF79B
:10A880003AFA00B300BF04F1100104F14800FBF7ED
:10A89000D1FE051E00D0AAE000BF00BF012104F1D7
:10A8A0003800FBF717FF051E00D0A0E000BF00BF77
:10A8B000012104F14000FBF70DFF051E00D096E0DA
:10A8C00000BF0020FEBD012104F13800FCF771FA41
:10A8D00068B300BF04F1380211460846FCF7C0FE19
:10A8E000051E00D083E000BF00BF224604F13801FE
:10A8F0000846FCF733FF051E00D078E000BF00BF1C
:10A9000004F1400211460846FCF7AAFE051E00D0DD
:10A910006DE000BF00BF224604F140010846FCF78D
:10A920001DFF051E00D062E000BF0020CAE700BF87
:10A930003B463246214604F13800FFF723FE051E50
:10A9400000D054E000BF00BF3B463246214601A87C
:10A95000FFF718FE051E00D049E000BF00BF01AAA6
:10A9600004F1380104F14000FCF77AFE051E00D026
:10A970003DE000BF00BF224604F140010846FCF75D
:10A98000EDFE051E00D032E000BF00BF224604F1FC
:10A9900040010846FDF706F9051E00D027E000BF7C
:10A9A00000BF01AA04F140010846FCF759FE051E4C
:10A9B00000D01CE000BF00BF224604F14001084661
:10A9C000FCF7CCFE051E00D011E000BF00BF04F173
:10A9D0003000234604F1100204F1400100901030D1
:10A9E000FCF7FDFE051E00D001E000BF00BF01A87E
:10A9F000FBF7B5FD284665E72DE9FE4F044689467D
:10AA000017461D46DDE90C8A6FF06D06B8F1000FA0
:10AA100002D18548BDE8FE8F2046FFF75AFDB842B7
:10AA200001D98148F6E7214604F12000FFF720FD17
:10AA3000061E01D03046EDE701A8FBF78AFD00BFF6
:10AA4000524641462046FFF70FFF061E00D04DE05C
:10AA500000BF00BF04F1380204F1200101A8FCF797
:10AA6000FFFD061E00D041E000BF00BF224601A945
:10AA700001A8FCF773FE061E00D037E000BF00BF40
:10AA800004F13000234604F1100201A900900838B7
:10AA9000FCF7A5FE061E00D028E000BF00BF04F1B1
:10AAA000400204F128010846FCF7DAFD061E00D03A
:10AAB0001CE000BF00BF224604F128010846FCF755
:10AAC0004DFE061E00D011E000BF04F12800FBF788
:10AAD0008CFE286000BF494604F128002A68FCF774
:10AAE0009AFD061E00D001E000BF00BF01A8FBF7E1
:10AAF00036FD4EB140F2C113AFF20C323146494837
:10AB0000803800F0F1F885E7002083E710B50446AF
:10AB100004B910BD04F14800FBF721FD04F1400029
:10AB2000FBF71DFD04F13800FBF719FD04F13000BF
:10AB3000FBF715FD04F12800FBF711FD04F12000DF
:10AB4000FBF70DFD04F11800FBF709FD04F11000FF
:10AB5000FBF705FD04F10800FBF701FD2046FBF7BC
:10AB6000FEFC5021204607F0A5FA00BFD1E7F7B55B
:10AB700088B007460E466FF06D0403A805F0D2FAC0
:10AB80000A9818B10A98401E305C08B1274C0BE0B7
:10AB90000AA800210091334625A2CDE901102BA17E
:10ABA00003A805F04FFC044614B904980A9003E08A
:10ABB00014F5845F00D086E00CB9039800E03046BD
:10ABC00006900A9906984518302307AA294606A830
:10ABD000FAF7ADFC041E09D040F21123AFF2F032B7
:10ABE0002146224800F080F804466CE0DDE90601C9
:10ABF00045183A46294606A8FAF73FFD041E07D134
:10AC000007F10802294606A8FAF737FD041E2FD0DF
:10AC100040F21923AFF228422146144800F064F8AC
:10AC2000044650E080CDFFFF80CFFFFF80EFFFFFA5
:10AC30002D2D2D2D2D454E4420444820504152416C
:10AC40004D45544552532D2D2D2D2D002D2D2D2D9F
:10AC50002D424547494E20444820504152414D45E0
:10AC6000544552532D2D2D2D2D00000080CCFFFF7B
:10AC70000698A84225D001A8FBF76BFC01AA29463B
:10AC800006A8FAF7FAFC044601A8FBF768FC4CB1E9
:10AC900040F22523AFF2A8422146154800F024F8DF
:10ACA000044610E00698A8420AD040F22923AFF2E9
:10ACB000C0426FF065010E4800F016F8044602E04D
:10ACC00000BF002400BF03A805F06FFD14B1384693
:10ACD000FFF71CFF20460BB0F0BD08B50146088801
:10ACE0000090BDF8000008BD10B50446601810BD06
:10ACF00080CCFFFF0146487870470146012070472D
:10AD00002DE9FE4F05460E4617461C46DDE90C8927
:10AD10006FF06D0A4FF0000BBBF1000F0BD100BFBD
:10AD2000434622463146284602F0B2F9B0F1000A05
:10AD300000D010E000BF00BF05F11C0332463946C9
:10AD400028468DE8100302F061F8B0F1000A00D047
:10AD500001E000BF00BF5046BDE8FE8F2DE9FC4179
:10AD600004460D4616461F46DDF8208000203B466F
:10AD700032462946CDE900802046FFF7C1FFBDE8F5
:10AD8000FC812DE9F04F89B007460C4615461E465A
:10AD9000DDE9139ADDF848806FF06D0B03A800F031
:10ADA000D8FA00BF2B46324603A938468DE8000783
:10ADB00002F02CF8B0F1000B00D012E000BF03A8A5
:10ADC00000F0B9FB10B1DFF888B40AE000BF03A9B6
:10ADD0002046FBF72FFCB0F1000B00D001E000BFD4
:10ADE00000BF03A800F0F3FA584609B0BDE8F08FA1
:10ADF0002DE9FE4304460D4616461F46DDE90A8945
:10AE000000203B4632462946CDE900890290204683
:10AE1000FFF7B7FFBDE8FE8310B50446204600F0FB
:10AE2000A6FA04F16000FBF794FB04F1680000F05F
:10AE300090FA04F1800000F08CFA04F19800FBF71E
:10AE400088FB10BD01464878704710B50446A42120
:10AE5000204617F084F80020A070207010BD70B557
:10AE600004460D466FF06D062946204602F059FB58
:10AE700006460EB1F74870BD0020FCE770B50446E9
:10AE80000D4600BF002020700120A0706570201DBD
:10AE9000FFF7C2FF2946201DFFF7E1FF70BD10B587
:10AEA0000446204600F0ADFA04F16000FBF757FBC2
:10AEB00004F1680000F08BFA04F1800000F087FADA
:10AEC00004F19800FBF74BFB10BD10B5044604B924
:10AED00010BDA078012803D1201DFFF7E0FF00E09E
:10AEE00000BF00BF00202070A070607000BFEFE7BF
:10AEF0002DE9FF5F04460F4690461D46DDE90F9A97
:10AF00000E9E6FF06D0BE06B18B9D14804B0BDE830
:10AF1000F09F4B4604F1680204F160012046CDF831
:10AF200000A0FFF71BFFB0F1000B01D05846EDE782
:10AF300033462A4603A9204600F011FEB0F1000B6B
:10AF400001D05846E2E7039805440398361A02AB4D
:10AF5000424604F168012046CDE9005600F08EFD1E
:10AF6000B0F1000B01D05846D0E7DDE902100844EB
:10AF700038600020CAE72DE9FF4704460F46154612
:10AF80001E46DDE90C894FF0000AA07801280AD19D
:10AF90008DE8400722782B463946201DFFF7A8FF91
:10AFA00004B0BDE8F087AA48FAE770B505460C463C
:10AFB00016462068331A224605F18001284600F023
:10AFC0003AFD70BDF8B504460D4616466FF06D07A4
:10AFD0002868321A2946684600F07DFD071E01D018
:10AFE0003846F8BD9DF800102046FFF747FF071EC2
:10AFF00001D03846F5E7A078012805D13246294628
:10B00000201DFFF7D2FFECE79148EAE72DE9F04178
:10B0100004460D4616466FF06D07012E07D105F167
:10B02000680104F1800000F033FABDE8F0810EB150
:10B030008748FAE705F1680104F1680000F028FA92
:10B04000071E07D105F1600104F16000FBF7F2FA79
:10B05000071E01D03846E8E70020E6E72DE9F04179
:10B0600004460D4616466FF06D0726B1012E02D03C
:10B070007748BDE8F0812046FFF73CFE38B92978D3
:10B080002046FFF7FBFE071E09D03846F1E72046B1
:10B09000FFF730FE2978884201D06D48E9E7A078B3
:10B0A000012805D132462946201DFFF7AFFFE0E712
:10B0B0006748DEE72DE9FC5F04460D4617461E464D
:10B0C000DDE90D9ADDF830806FF06D0BE06B10B9A3
:10B0D0005F48BDE8FC9F4B4604F1680204F1600143
:10B0E0002046CDF800A0FFF739FEB0F1000B01D0EB
:10B0F0005846EEE72B463A4604F168012046CDE972
:10B10000006800F0BBFCE4E72DE9FF4704460F466A
:10B1100015461E46DDE90C894FF0000AA07801288B
:10B120000AD18DE8400722782B463946201DFFF7CB
:10B13000C1FF04B0BDE8F0874548FAE7F8B5064618
:10B140000C4615466FF06D0700942B466A4606F1D3
:10B150008001304600F06FFC071E01D03846F8BD74
:10B160000098001BA84201D03948F8E70020F6E714
:10B1700070B504460D461646A078012805D1324622
:10B180002946201DFFF7DAFF70BD3148FCE72DE9A5
:10B19000FC5F04460D4616461F46DDE90D9BDDF8B3
:10B1A00030806FF06D0A0CB1E06B10B92848BDE833
:10B1B000FC9F04F1600304F1800204F19801204631
:10B1C000CDE90089FFF714FEB0F1000A01D0504626
:10B1D000EDE704F19800FBF708FBB84201D91C48E1
:10B1E000E5E794F83C0000F0070008B1012000E01A
:10B1F0000020E16B00EBD1002860204600F09EF8B3
:10B20000022806D1314604F198002A68FCF7F8F9C3
:10B21000CDE7314604F198002A68FCF7FCF9C6E74F
:10B220002DE9FE4F04460D4616461F46DDE90C8902
:10B230004FF0000AA07801280ED13B46324629463D
:10B24000201D8DE80007FFF7A2FFBDE8FE8F00007C
:10B2500080B0FFFF80B1FFFF0048F6E780B0FFFF3E
:10B2600070B504460D4603E020460834FBF771F93B
:10B27000281EA5F10105F7D170BD70B504460D4635
:10B2800003E020460834FBF76AF9281EA5F1010502
:10B29000F7D170BDFA48704710B5FA48006898B900
:10B2A0000022FFF7F7FF014605E00C781046521C1C
:10B2B000F54B1C540C3108780028F6D1F24B985409
:10B2C0000120F04B186000BFEF4810BD00B50246EA
:10B2D000FFF7E0FF014605E00878904201D10846FB
:10B2E00000BD0C3108780028F6D100BFF8E700B5A2
:10B2F0000246FFF7CFFF014605E04888904201D1A2
:10B30000084600BD0C3108780028F6D100BFF8E7E8
:10B3100070B505460DB9002070BDFFF7BBFF0446B0
:10B3200007E02946A06816F054FE08B92046F3E766
:10B330000C3420780028F4D100BFEDE70146C8693D
:10B3400008B900207047486A08B90220FAE70120CE
:10B35000F8E710B504462046FBF7FBF804F10800B7
:10B36000FBF7F7F804F11000FBF7F3F810BD10B588
:10B37000044600202070201DFBF7EBF804F10C00C0
:10B38000FBF7E7F804F11400FBF7E3F804F11C0005
:10B39000FFF7DFFF04F13400FBF7DBF80020E06388
:10B3A00020646064A064E06420656065A065E06579
:10B3B00010BD10B504462046FFF7D9FF04F1600028
:10B3C000FBF7C7F804F16800FFF7C3FF10BD10B525
:10B3D000044604B910BD2046FBF7C1F804F108008B
:10B3E000FBF7BDF804F11000FBF7B9F800BFF1E777
:10B3F0000146886D18B1C86D08B90120704700205A
:10B40000FCE770B5044604B970BD606C012812D029
:10B4100004F10C00FBF7A3F804F11400FBF79FF80C
:10B4200004F11C00FFF7D3FF04F13400FBF797F899
:10B43000201DFBF794F82046FFF7DAFF88B9A06DCE
:10B4400078B1002507E005EB4502A16D01EBC200D4
:10B45000FFF7BDFF6D1CE06DA842F4D8A06D18F099
:10B4600053F86021204606F025FE00BFCCE710B55A
:10B47000044604B910BD2046FFF7C3FF04F1600085
:10B48000FBF76DF804F16800FFF7A1FF00BFF1E7DB
:10B4900070B504460D466FF06D0600BF2946204684
:10B4A000FBF7C8F8061E00D017E000BF00BF05F18B
:10B4B000080104F10800FBF7BDF8061E00D00CE0FF
:10B4C00000BF00BF05F1100104F11000FBF7B2F856
:10B4D000061E00D001E000BF00BF304670BD70B551
:10B4E00005460C462178284602F01BF870BD70B561
:10B4F00004466FF06D0500BF01212046FBF7EAF816
:10B50000051E00D015E000BF00BF012104F10800B6
:10B51000FBF7E0F8051E00D00BE000BF00BF0021E4
:10B5200004F11000FBF7D6F8051E00D001E000BFC3
:10B5300000BF284670BD10B50446002104F110007C
:10B54000FBF737FC08B9012010BD0020FCE770B5FF
:10B5500005460C4621462846FBF7CDFB78B904F199
:10B56000080105F10800FBF7C6FB40B904F1100122
:10B5700005F11000FBF7BFFB08B9002070BD434880
:10B58000FCE72DE9F04104460E4617461D466FF0D4
:10B590006D0800BF3A4631462046FBF7FCFAB0F191
:10B5A000000800D018E000BF00BF2A46314604F171
:10B5B0000800FBF7F0FAB0F1000800D00CE000BF83
:10B5C00000BF012104F11000FBF784F8B0F100087E
:10B5D00000D001E000BF00BF4046BDE8F0812DE98A
:10B5E000F05F82460E4617461C46DDE90A59DFF831
:10B5F000A0B027B1012F02D02448BDE8F09F0AF186
:10B600000400FBF7F2F880465046FFF797FE01284A
:10B610005ED1002106F11000FBF7CBFB58B9B9F160
:10B62000000F02D119488030E7E700202870012080
:10B6300020600020E1E76FBB4FEA4800401C20601B
:10B640002068484502D911488030D6E70420287088
:10B6500000BF4246691C3046FBF7DDFFB0F1000B2E
:10B6600000D036E000BF00BF681C00EB0801424676
:10B6700006F10800FBF7CFFFB0F1000B0BD028E07C
:10B68000FC370208140100201001002080B0FFFFE9
:10B6900080B1FFFF00E01BE0012F19D108F101008C
:10B6A00020602068484501D9FD48A6E7002106F141
:10B6B0000800FBF730F8801C287000BF4246691C68
:10B6C0003046FBF7A8FFB0F1000B00D001E000BF4F
:10B6D00000BF584691E72DE9F04104460D46164655
:10B6E0001F466FF06D0800BF3A4631462846FBF70B
:10B6F000F5F9B0F1000800D013E000BF0AE000BF88
:10B70000221D29462846FBF7FAF8B0F1000800D0C0
:10B7100007E000BF211D2846FBF7EDFA0028EEDA0E
:10B7200000BF4046BDE8F08170B505460C466FF09D
:10B730006D06A06C28B9221D29462846FCF70EF894
:10B7400070BDB5F90400002804DA00212846FBF793
:10B7500030FB30B92846FBF741F8E16B49008842DD
:10B7600002D9CF488038EBE700BF2846A16C884754
:10B77000061E00D027E000BF09E000BF221D2946B9
:10B780002846FBF7ABF9061E00D01CE000BFB5F958
:10B790000400002805DA00212846FBF70AFB0028F0
:10B7A000EBD109E000BF221D29462846FBF7A7F888
:10B7B000061E00D007E000BF211D2846FBF79BFABC
:10B7C0000028EFDA00BF3046BAE72DE9F041044621
:10B7D0000D4616461F466FF06D0800BF3A463146CB
:10B7E0002846FBF73DFFB0F1000800D00DE000BF98
:10B7F00000BF00BF21462846FFF796FFB0F10008C2
:10B8000000D002E000BF00BF00BF4046BDE8F081AD
:10B810002DE9F04104460D46164600BF3346324638
:10B8200029462046FFF7D1FF071E00D033E000BFB6
:10B83000204601F0F5FD50B100BF03232A462946FA
:10B84000204601F0F4FD071E00D024E00BE000BF0D
:10B8500004F10C032A4629462046FFF73CFF071E49
:10B8600000D018E000BF00BF33462A4629462046D4
:10B87000FFF7ABFF071E00D00DE000BF00BF04F1D3
:10B8800014032A4629462046FFF725FF071E00D04D
:10B8900001E000BF00BF3846BDE8F0812DE9FE435E
:10B8A00004460E4615461F460021201DFAF733FFB9
:10B8B000012805D10121201DFAF72DFF012803D011
:10B8C00077488030BDE8FE8301A8FAF742FE00BF4A
:10B8D000324629462046FFF79BFFB0F1000800D012
:10B8E00035E000BF00BF0122211D01A8FBF701F9CF
:10B8F000B0F1000800D02AE000BF00BF022101A87B
:10B90000FBF76FFAB0F1000800D020E000BF00BFE5
:10B910000020231D01AA294600902846FBF75FFF5F
:10B92000B0F1000800D012E000BF00212846FAF76D
:10B93000F2FEB8420AD000BF2A46211D2846FBF776
:10B9400084FAB0F1000800D001E000BF00BF01A8F8
:10B95000FAF705FE4046B5E72DE9F04780460F4669
:10B9600014461E46DFF8389109F180091EB94C488B
:10B970008038BDE8F08708F10400FAF736FF054685
:10B980004046FFF7DBFC012852D1207840B9012E58
:10B9900003D13846FFF7ABFDEBE741488038E8E7D5
:10B9A000681CB04202D93E488038E2E700BF2A4610
:10B9B000611C3846FBF7FBFDB0F1000900D038E010
:10B9C00000BF00BF012107F11000FAF783FEB0F1BC
:10B9D000000900D02DE000BF207804280FD10120FD
:10B9E00000EB4500B04202D02D488038C1E7601C12
:10B9F00041192A4607F10800FBF7D9FDB9E720787D
:10BA0000022802D0207803280FD1681CB04202D04F
:10BA100023488038ADE7207800F0010307F10802E1
:10BA200039464046FFF73AFFA3E71D488038A0E7B4
:10BA300000BF48469DE72DE9F047804689461446F9
:10BA40001E46022E03D216488038BDE8F0872168D2
:10BA5000481C20600D78012D02DB701EA84202D226
:10BA60000F488038F1E727682068284420602B467B
:10BA70003A4649464046FFF76FFFE6E72DE9FC47A7
:10BA80008046894615461C46DDE90A676FF06D0A57
:10BA900045B1012D06D002488038BDE8FC87000082
:10BAA00000B1FFFF0FB9F848F7E7781E711C234675
:10BAB0002A46CDE9001049464046FFF790FDB0F117
:10BAC000000A01D05046E8E7207830702068401C1A
:10BAD00020600020E1E72DE9F04706460C461746B6
:10BAE000032F02D2E848BDE8F0872168481C206097
:10BAF0000878032801D0E448F5E7E44800780128F5
:10BB000003D1206801F07AFC05E0206801F076FCA2
:10BB1000814601F07FFC80462068801C2060404602
:10BB2000FFF7E5FB051E01D1D948DCE72878307026
:10BB30000020D8E7F8B504460D4616466FF06D07AD
:10BB4000324629466846FFF7C6FF071E01D0384631
:10BB5000F8BD9DF80010204601F0E3FCF8E72DE960
:10BB6000F04706460D4614461F463078FFF7AEFBF9
:10BB7000B0F1000802D1C448BDE8F0870320286076
:10BB80002868B84202D9C0488030F5E7032004F89D
:10BB9000010BBE480078012805D1B8F802102046F4
:10BBA00001F033FC08E0B8F8020001F033FC8146F4
:10BBB0004946204601F029FC0020DDE72DE9F0414F
:10BBC00005460C4616461F466FF06D0800BF3A4604
:10BBD00031462046FBF739F9B0F1000800D019E0F2
:10BBE00000BF00BF0AE000BF2A1D21462046FAF729
:10BBF00075FFB0F1000800D00CE000BFB4F90400FC
:10BC0000002805DA00212046FBF7D3F80028EAD106
:10BC100000BF00BF4046BDE8F0812DE9F041044679
:10BC20000D4616461F466FF06D0800BF3A46314676
:10BC30002846FAF778FFB0F1000800D013E000BF03
:10BC40000AE000BF221D29462846FAF758FEB0F147
:10BC5000000800D007E000BF211D2846FBF74BF885
:10BC60000028EEDA00BF4046BDE8F0812DE9F04142
:10BC700004460D4616466FF06D0700BF3146284654
:10BC8000FBF7BBF8071E00D012E000BF09E000BFC1
:10BC9000221D29462846FAF732FE071E00D007E08B
:10BCA00000BF211D2846FBF726F80028EFDA00BF69
:10BCB0003846BDE8F0817CB505460C46002104F10C
:10BCC0001000FBF776F808B900207CBD6FF06D0618
:10BCD0006846FAF73EFC00BF2A1D04F110016846D1
:10BCE000FBF760FF061E00D039E000BF00BF6B46C7
:10BCF00004F1080211462846FFF767FD061E00D032
:10BD00002DE000BF00BF6B466A4669462846FFF734
:10BD10005CFD061E00D022E000BF00BF6B4622463D
:10BD200021462846FFF751FD061E00D017E000BF50
:10BD300000BF6B4604F1080211462846FFF745FD97
:10BD4000061E00D00BE000BF00BF012104F110006F
:10BD5000FAF7C0FC061E00D001E000BF00BF684635
:10BD6000FAF7FDFB3046B0E72DE9FC4780460D466B
:10BD70001746022F05D240462968FFF79CFFBDE811
:10BD8000FC876FF06D090821384616F03DF9061E54
:10BD900001D14048F3E76846FAF7DBFB3946304605
:10BDA000FFF75EFA00BF286800F110013046FAF78D
:10BDB00041FCB0F1000900D0C8E000BF012412E04E
:10BDC00000BF55F8240000F11003601E06EBC0020E
:10BDD00006EBC4014046FFF7F8FCB0F1000900D0C3
:10BDE000B4E000BF641CBC42EAD300BF7A1E06EB7D
:10BDF000C20106EBC20008F10402FBF7D3FEB0F16A
:10BE0000000900D0A2E000BF7C1E00BF04B300BF49
:10BE1000601E06EBC00306EBC40269464046FFF70E
:10BE2000D4FCB0F1000900D090E000BF00BF55F88D
:10BE3000240000F1100306EBC402601E06EBC001F3
:10BE40004046FFF7C2FCB0F1000900D07EE009E0F7
:10BE500000BF31466846FAF7EDFBB0F1000900D0AB
:10BE600074E000BF00BF55F8240000F1080255F847
:10BE7000240000F108016B464046FFF7A6FCB0F134
:10BE8000000909D062E0000080B0FFFFF837020827
:10BE900080B1FFFF80B2FFFF00BF00BF6B466A4664
:10BEA00069464046FFF791FCB0F1000900D04DE033
:10BEB00000BF00BF55F8242055F824106B464046BB
:10BEC000FFF783FCB0F1000900D03FE000BF00BFE6
:10BED00055F8240000F1080255F8240000F108018B
:10BEE0006B464046FFF771FCB0F1000900D02DE031
:10BEF00000BF00BFB8F80A1055F82400FAF741FB5C
:10BF0000B0F1000900D021E000BF00BFB8F80A106E
:10BF100055F8242002F10800FAF733FBB0F10009CC
:10BF200000D013E000BF00BF55F8241001F110004D
:10BF30000121FAF7CFFBB0F1000900D006E000BF05
:10BF400004B901E0641E61E700BF00BF6846FAF76C
:10BF500006FB39463046FFF790F9304617F0D4FA21
:10BF600048460CE72DE9FC4105460C4616466FF0A5
:10BF70006D076846FAF7EDFA00BF002104F10800EA
:10BF8000FAF717FF08B1012000E00020804600BF4B
:10BF900004F10802291D6846FAF757FF071E00D072
:10BFA0000EE000BF00BF08EA0602694604F108007F
:10BFB000FAF759FA071E00D002E000BF00BF00BF29
:10BFC0006846FAF7CCFA3846BDE8FC812DE9F04125
:10BFD00007460E4615461C466FF06D08384601F0C0
:10BFE0001FFA002845D000BF05F110031A4604F1DE
:10BFF00008013846FFF7E9FBB0F1000800D070E116
:10C0000000BF00BF04F108032A4604F110013846BE
:10C01000FFF761FBB0F1000800D062E100BF00BF94
:10C0200004F108032A4604F118013846FFF7C6FD5B
:10C03000B0F1000800D054E100BF00BF04F11803C4
:10C0400004F1100204F108013846FFF7BEFBB0F11D
:10C05000000800D045E100BF00BF032304F108023F
:10C0600021463846FFF7D9FDB0F1000800D038E18D
:10C0700058E000BF2B462A4604F108013846FFF776
:10C08000A4FBB0F1000800D02BE100BF00BF0323E8
:10C0900004F1080221463846FFF7BFFDB0F1000861
:10C0A00000D01EE100BF002107F10C00FAF781FE6D
:10C0B000B0B300BF05F110031A4604F10801384679
:10C0C000FFF783FBB0F1000800D00AE100BF00BF1A
:10C0D00004F108031A4604F110013846FFF775FB16
:10C0E000B0F1000800D0FCE000BF00BF07F10C0376
:10C0F00004F1100204F108013846FFF766FBB0F1C5
:10C10000000800D0EDE000BF00BF04F108032246A4
:10C1100021463846FFF7DFFAB0F1000801D0E0E031
:10C1200000E000BF00BF05F108031A4604F110014A
:10C130003846FFF74AFBB0F1000800D0D1E000BF5D
:10C1400000BF012204F110013846FFF78FFDB0F166
:10C15000000800D0C5E000BF00BF04F110032A466C
:10C1600004F108013846FFF730FBB0F1000800D0B9
:10C17000B7E000BF00BF012204F108013846FFF715
:10C1800075FDB0F1000800D0ABE000BF00BF04F1C6
:10C1900010031A4604F118013846FFF716FBB0F1F8
:10C1A000000800D09DE000BF00BF012204F118018B
:10C1B0003846FFF75BFDB0F1000800D091E000BF0A
:10C1C00000BF2346224604F110013846FFF7FDFA6E
:10C1D000B0F1000800D084E000BF00BF04F1080304
:10C1E00004F1100211463846FFF7E8FCB0F10008F0
:10C1F00000D076E000BF00BF04F1080304F1100294
:10C2000011463846FFF7DAFCB0F1000800D068E0CC
:10C2100000BF00BF04F1100304F1080211463846C4
:10C22000FFF7CCFCB0F1000800D05AE000BF00BF1F
:10C23000234604F1080211463846FFF7C6FAB0F16A
:10C24000000800D04DE000BF00BF04F1180304F166
:10C25000080211463846FFF7B1FCB0F1000800D0E3
:10C260003FE000BF00BF05F1100305F1080204F133
:10C2700018013846FFF7A9FAB0F1000800D030E005
:10C2800000BF00BF012204F118013846FFF7EEFCA1
:10C29000B0F1000800D024E000BF00BF04F110019D
:10C2A0003046FAF7C7F9B0F1000800D019E000BF36
:10C2B00000BF04F1080106F10800FAF7BBF9B0F17C
:10C2C000000800D00DE000BF00BF04F1180106F126
:10C2D0001000FAF7AFF9B0F1000800D001E000BF9C
:10C2E00000BF4046BDE8F0812DE9F84F81460F467A
:10C2F00015461E460A9C6FF06D0AB84607F1080BFA
:10C3000007F110000090306910B9FE48BDE8F88FC1
:10C31000002105F11000FAF74CFD20B931463846EE
:10C32000FFF7B6F8F2E7002106F11000FAF741FD39
:10C3300020B929463846FFF7ABF8E7E7012106F1B7
:10C340001000FAF736FD08B1EE48DFE700BF05F14F
:10C3500010031A4621464846FFF737FAB0F1000AA3
:10C3600000D003E100BF00BF05F11003224604F135
:10C3700008014846FFF729FAB0F1000A00D0F5E0BD
:10C3800000BF00BF3346224621464846FFF71DFA4C
:10C39000B0F1000A00D0E9E000BF00BF06F10803D9
:10C3A00004F1080211464846FFF70FFAB0F1000AFF
:10C3B00000D0DBE000BF00BF2B46224621464846A6
:10C3C000FFF7FCFBB0F1000A00D0CFE000BF00BFD8
:10C3D00005F1080304F1080211464846FFF7EEFB99
:10C3E000B0F1000A00D0C1E000BF00212046FAF7FA
:10C3F000E0FC90B9002104F10800FAF7DAFC38B942
:10C4000023462A4639464846FFF7E0FD8246ADE01E
:10C410003846FFF76CF88246A8E000BF234605F1D6
:10C42000100248460099FFF7D0F9B0F1000A00D099
:10C430009CE000BF00BF2346224604F1100148469D
:10C44000FFF7C3F9B0F1000A00D08FE000BF00BFD2
:10C45000234604F1100204F118014846FFF7B5F92C
:10C46000B0F1000A00D081E000BF00BF2B4604F10C
:10C47000100211464846FFF7A8F9B0F1000A00D0B3
:10C4800074E000BF00BF04F110012046FAF7D2F8B3
:10C49000B0F1000A00D069E000BF00BF01222146D0
:10C4A0004846FFF7E3FBB0F1000A00D05EE000BFB2
:10C4B00000BF04F108031A4641464846FFF785F9D4
:10C4C000B0F1000A00D051E000BF00BF2346424651
:10C4D00041464846FFF772FBB0F1000A00D045E044
:10C4E00000BF00BF04F11803424641464846FFF72B
:10C4F00065FBB0F1000A00D038E000BF00BF434642
:10C5000004F1100211464846FFF758FBB0F1000A4B
:10C5100000D02BE000BF00BF04F1080304F11002BB
:10C5200011464846FFF751F9B0F1000A00D01DE06E
:10C5300000BF00BF05F1080304F118021146484688
:10C54000FFF743F9B0F1000A00D00FE000BF00BFD1
:10C5500004F1180304F1100259464846FFF72EFB78
:10C56000B0F1000A00D001E000BF00BF5046CDE6A8
:10C570002DE9FE4305460C4616461F466FF06D0832
:10C5800001A8F9F7E6FF00BF33462A1D022101A8E2
:10C590000097FBF7DFFAB0F1000800D040E000BFE1
:10C5A00000BF01AB04F1100211462846FFF70DF958
:10C5B000B0F1000800D033E000BF00BF01AB04F1D0
:10C5C000080211462846FFF700F9B0F1000800D034
:10C5D00026E000BF00BF01AB01AA01A92846FFF772
:10C5E000F4F8B0F1000800D01AE000BF00BF01ABC2
:10C5F000224621462846FFF7E8F8B0F1000800D0AF
:10C600000EE000BF00BF01AB04F10802114628464E
:10C61000FFF7DBF8B0F1000800D001E000BF00BF79
:10C6200001A8F9F79CFF08F10E0008B9DFF8D880DF
:10C630004046BDE8FE832DE9FF5F05460E46934662
:10C64000711C284615F08BFC00240EE0002709E041
:10C6500006FB07410398FAF75EF8B840295D0843E6
:10C6600028557F1C5F45F3D3641CB442EED34FF0D2
:10C670000008012422E0285D00EA080A285D80EA1B
:10C6800008002855D046285D00F00100C0F10109DE
:10C69000285D611E695C01FB09F1084040EA080859
:10C6A000285D611E695C01FB09F148402855601E48
:10C6B000285C40EAC910611E6854641CB442DAD98F
:10C6C000BDE8FF9F2DE9FF4F91B00E469346994676
:10C6D000DDF878A06FF06D0010900025A9F1010041
:10C6E00001218140CFB21C2109A815F038FC04219A
:10C6F00001A8FEF7B5FD00BF59463046FEF7C8FE5B
:10C70000109003E080B0FFFF00B3FFFF00B193E0A3
:10C7100000BF002526E0B5FBFAF101208840C4B235
:10C7200004EB440006EBC008B5FBFAF00AFB10501E
:10C7300060B900BF601000EB400006EBC00140464E
:10C74000FEF7A6FE109000B176E000BF00BF01AB7F
:10C75000424641461198FFF739FC109000B16BE05A
:10C7600000BF6D1CA9F1010000FB0AF0A842D2D85D
:10C77000002501240AE004EB440006EBC002284631
:10C780006D1C09A941F820206006040EBC42F2DBB2
:10C7900000BF2A4609A91198FFF7E6FA109000B1E8
:10C7A0004AE000BF01241EE0254616E000BF01A8B4
:10C7B000009004EB440006EBC00305EB450006EBDC
:10C7C000C002601900EB400006EBC0011198FFF7B2
:10C7D0008BFD109000B12FE000BF281EA5F10105D0
:10C7E000E4D16006040EBC42DEDB002508E005EB68
:10C7F000450006EBC000183009A941F825006D1C62
:10C80000681CB842F3D300BF2A4609A91198FFF764
:10C81000ABFA109000B10FE000BF002409E004EB78
:10C82000440106EBC10101F11000F9F798FE601C0C
:10C83000C4B2BC42F3DB00BF042101A8FEF71DFD1A
:10C84000109815B0BDE8F08F2DE9F05F82460D46D7
:10C8500016461F46DDF828806FF06D0BC8F34509BA
:10C8600000242AE000BF4C4501D1012000E0002057
:10C87000024604EB440006EBC0012846F9F7F3FD3D
:10C88000B0F1000B00D032E000BF00BF4C4501D139
:10C89000012000E00020024604EB440006EBC0004B
:10C8A00000F1080105F10800F9F7DDFDB0F1000B1A
:10C8B00000D01CE000BF601CC4B2BC42D2DB00BF91
:10C8C0004FEAE81229465046FFF74CFBB0F1000B47
:10C8D00000D00CE000BF00BF012105F11000F9F706
:10C8E000F9FEB0F1000B00D001E000BF00BF5846D8
:10C8F000BDE8F09F2DE9F04F91B080460D4691467E
:10C900009A46DDE91BB71A9E6FF06D0010900AA8D9
:10C91000FEF71FFD042102A8FEF7A2FC5C4600BF43
:10C92000305D53464A46294600904046FFF78CFF4B
:10C93000109000B136E000BF57B100BF3A4629461B
:10C9400040461D9BFFF714FE109000B12AE000BF87
:10C9500025E0641E00BF02AB2A4629464046FFF789
:10C9600035FB109000B11DE000BF00BF305D5346A5
:10C970004A460AA900904046FFF766FF109000B1B2
:10C9800010E000BF00BF02A80AAB2A46294600906B
:10C990004046FFF7A9FC109000B103E000BF002C57
:10C9A000D7D100BF0AA8FEF712FD042102A8FEF7A6
:10C9B00064FC109811B0BDE8F08F2DE9FF470446E4
:10C9C0000D4616461F46DDE90C986FF06D0A02A869
:10C9D000F9F7BFFD6846F9F7BCFD002104F134000A
:10C9E000F9F799FE012803D0F84804B0BDE8F087B4
:10C9F00000212846F9F78FFE08B9012000E0002049
:10CA000088F8000000BF294602A8F9F713FEB0F12C
:10CA1000000A00D01FE000BF00BF2A4604F1340125
:10CA20006846FAF712FAB0F1000A00D013E000BF2E
:10CA300000BF98F80020694602A8F9F714FDB0F18C
:10CA4000000A00D007E000BF02AB4A463946304634
:10CA5000FFF7F1FD00BF6846F9F781FD02A8F9F77D
:10CA60007EFD5046C1E72DE9F04FB9B082460D4634
:10CA700016461F46DDF808B1DDF81891DDF8108183
:10CA8000459C6FF06D003890059500BF37A943981D
:10CA9000434606AACDE9000131465046FFF78DFF17
:10CAA000389000B134E000BF00BF4798CDE902499B
:10CAB000CDF80480049006A85B463A4600905046A4
:10CAC0000599FFF717FF389000B121E000BF00BFC4
:10CAD0009DF8DC2050460599FFF744FA389000B1E4
:10CAE00016E000BF54B100BF4B46224650460599A0
:10CAF000FFF73EFD389000B10AE000BF00BF50468E
:10CB00000599FFF7D8F8389000B101E000BF00BFE9
:10CB1000389839B0BDE8F08F70B505460E46286CE0
:10CB2000B0F5C07F01D3052000E0042004460EB11B
:10CB3000601CC4B21EB12846FEF75AFC10B9042C82
:10CB400000DD0424286CA04200D80224204670BDD9
:10CB50002DE9FF4F89B0044699466FF06D000890AB
:10CB60004FF0000800200790002504F1240109F18E
:10CB70000800FAF7C0F838B904F11C014846FAF782
:10CB8000BAF808B9012000E000208246514620464C
:10CB9000FFF7C2FF0646701E0121814001F0FF0829
:10CBA000216C3144491EB1FBF6FBBAF1000F05D0F0
:10CBB000A06D18B1A56D0120079016E01821404620
:10CBC00015F022FA054615B98148089039E000278A
:10CBD00007E007EB470105EBC100FEF7BAFB781C45
:10CBE000C7B24745F5DB00200790079898B900BF0A
:10CBF000189833464A462946CDE900B02046FFF74B
:10CC000061FD089000B11CE000BFBAF1000F02D036
:10CC1000A565C4F85C8000BFDDE9162118982B4695
:10CC2000CDE9016BCDF80080CDE9032105902046C8
:10CC3000DDE90A12FFF717FF089000B101E000BF1D
:10CC400000BFA06DA84200D1002575B1002707E004
:10CC500007EB470105EBC100FEF7B9FB781CC7B233
:10CC60004745F5DB284616F04FFC089808B101202F
:10CC700000E000200690069810B10A98FEF7A7FB86
:10CC800008980DB0BDE8F08F7FB505460C466FF0F3
:10CC90006D0600212046FAF78CF8002813DB0021EE
:10CCA00004F10800FAF785F800280CDB291D20465E
:10CCB000FAF721F8002806DA291D04F10800FAF72E
:10CCC0001AF8002802DB434804B070BD02A8F9F747
:10CCD00040FC6846F9F73DFC00BF04F108031A4622
:10CCE00002A92846FEF771FD061E00D011E000BF24
:10CCF00000BF224669462846FEF78AFD061E00D080
:10CD000007E000BF694602A8F9F7F5FF00B1314E10
:10CD100000BF02A8F9F723FC6846F9F720FC30466B
:10CD2000D2E770B505460C46012104F11000FAF770
:10CD300040F808B1274870BD2846FEF7FFFA0128E1
:10CD400004D121462846FFF79FFFF4E71F48F2E78A
:10CD500070B505460C462846FEF7F0FA012810D1BA
:10CD600001212046FAF725F8002806DB05F13401F9
:10CD70002046F9F7C0FF002801DB164870BD0020EF
:10CD8000FCE71248FAE72DE9FF5F06460F46144616
:10CD90001D46DDE90F9ADDF838800C4803904FF00E
:10CDA000000BBBF1000F18D100BF21463046FFF742
:10CDB000CFFF039000B125E000BF00BF29463046F9
:10CDC000FFF7AFFF039038B11CE0000080B0FFFF19
:10CDD00080B2FFFF80B3FFFF00BFFA4803903046E8
:10CDE000FEF7ACFA01280CD100BF2B46224639468B
:10CDF00030468DE80007FFF7ABFE039000B101E07D
:10CE000000BF00BF039804B0BDE8F09F2DE9FE4FBE
:10CE100005460E4617469846DDE90D9A0C9C14B956
:10CE2000E848BDE8FE8F43463A46314628468DE83D
:10CE30001006FFF7A8FFF4E72DE9FE4304460D4670
:10CE400016461F46DDE90A8900203B463246294640
:10CE5000CDE9008902902046FFF7D8FFBDE8FE83A8
:10CE60002DE9F04786B005460C4616461F46DDF80C
:10CE700038806FF06D0904A8F9F76BFB002130468C
:10CE8000F9F797FF90B900BF39462846FFF749FFE9
:10CE9000B0F1000900D073E000BF00BF2046FEF7EC
:10CEA00026FBB0F1000900D06AE068E001213046BD
:10CEB000F9F77FFF98B900BF39462846FFF731FFE1
:10CEC000B0F1000900D05BE000BF00BF394620464A
:10CED000FEF7DEFAB0F1000900D051E04FE04FF06C
:10CEE000FF313046F9F765FFB0BB00BF3946284631
:10CEF000FFF717FFB0F1000900D041E000BF00BF0D
:10CF000039462046FEF7C4FAB0F1000900D037E0F8
:10CF100000BF00BF002104F10800F9F74AFF08B183
:10CF2000012000E00020824600BF04F10802291D14
:10CF300004A8F9F78AFFB0F1000900D020E000BF93
:10CF400000BF0AF0010204A904F10800F9F78BFA06
:10CF5000B0F1000901D013E001E000BF0FE000BF15
:10CF6000002000903B4632462146CDE90108284684
:10CF7000FFF709FFB0F1000900D001E000BF00BFDA
:10CF800004A8F9F7ECFA484606B0BDE8F0872DE9A9
:10CF9000F04F91B080460C4691469A46DDF868B055
:10CFA0001C9D6FF06D0010900AAE27464046FEF7BC
:10CFB000C5F9012803D0844811B0BDE8F08F0AA854
:10CFC000FEF7C7F9042102A8FEF74AF900BF53464D
:10CFD0004A46314640460095FFF742FF109000B1A7
:10CFE00023E000BF00BF00955A46394640461B9BD0
:10CFF000FFF736FF109000B117E000BF00BF02A896
:10D000003B463246394600904046FFF76DF9109096
:10D0100000B10AE000BF00BF39464046FEF74BFEB4
:10D02000109000B101E000BF00BF042102A8FEF78C
:10D0300024F90AA8FEF7CBF91098BDE72DE9FE43C5
:10D0400004460D4616461F46DDE90A8900203B4688
:10D0500032462946CDE9008902902046FFF797FF26
:10D06000BDE8FE832DE9F84304460D4616461F46EB
:10D0700033462246012128460097FAF76BFD804689
:10D0800018F10E0F02D15148BDE8F8834046FBE786
:10D090002DE9F04104460D4616461F462046FEF790
:10D0A0004DF9012808D13B463246294604F13400A7
:10D0B000FFF7D8FFBDE8F0814248FBE72DE9FC47C8
:10D0C00081460C4615461E46DDE90A786FF06D0A6A
:10D0D00000BF43463A4629464846FFF7D9FFB0F11C
:10D0E000000A00D00FE000BF00BF23462A463146A9
:10D0F0004846CDE90078FFF79FFEB0F1000A00D066
:10D1000001E000BF00BF5046BDE8FC872DE9FC41AF
:10D1100004460D4616461F46DDF8208033462A4653
:10D1200004F11C012046CDE90078FFF7C7FFBDE8F8
:10D13000FC812DE9F84305460C4616461F466FF064
:10D140006D082946204600F0ECF9B0F1000802D045
:10D150004046BDE8F883334604F1680204F16001FB
:10D1600020460097FFF7D2FFF3E72DE9F04105468F
:10D170000C4616466FF06D07207840B929462046C8
:10D1800000F0CFF9071E07D03846BDE8F0812078BF
:10D19000A84201D00B48F8E7314604F16800FEF7D9
:10D1A00077F9F2E72DE9F04106460C461746984616
:10D1B00000253146204600F0B4F9051E08D0284667
:10D1C000BDE8F08180B0FFFF80B1FFFF00B3FFFF3B
:10D1D000AE4D2046FEF7B2F801280AD100BF424604
:10D1E000394604F16000FAF7E2F9051E00D00CE0C0
:10D1F00000BF4DB900BF04F160012046FFF7A8FD54
:10D20000051E00D001E000BF00BF1DB104F16000A9
:10D21000F9F7A5F92846D3E72DE9F04104460D4674
:10D2200016466FF06D072046FEF788F801280AD1F0
:10D2300000BF3246294604F16000FAF7ECF9071EF8
:10D2400000D001E000BF00BF3846BDE8F0812DE905
:10D25000F04104460D4617469846206CC01DC6088E
:10D26000464505D90020286088488038BDE8F0810F
:10D270002E606620005B08B98548F7E72046FEF778
:10D280005DF8012806D13246394604F16000FAF70C
:10D29000C2F9EBE76FF06D00E8E72DE9FC410446C9
:10D2A0000D4616461F46DDF8208033462A4604F117
:10D2B00068012046CDE90078FEF791F9BDE8FC81D0
:10D2C0002DE9F041A0B005460C4616461F466FF00A
:10D2D0006D082878C0B128782178884214D104F1EB
:10D2E000680105F16800F9F706FD68B904F17001FD
:10D2F00005F17000F9F7FFFC30B904F1780105F190
:10D300007800F9F7F8FC18B1614820B0BDE8F08169
:10D310001AA8FEF71EF802A8FEF729F8214602A86F
:10D32000FEF7DDF800BF04F11C0304F160021AA946
:10D3300002A8CDE90067FFF77FFDB0F1000800D03B
:10D3400016E000BF04F168011AA8F9F7D4FC58B937
:10D3500004F170011CA8F9F7CEFC28B904F178019A
:10D360001EA8F9F7C8FC10B1DFF8248100E000BF67
:10D370001AA8FEF72CF802A8FEF743F84046C4E7C7
:10D380007CB504460D46164604F11C0304F1600208
:10D3900004F168012046CDE90056FFF74DFD7CBD44
:10D3A0000146087870472DE9F04104460D461646BF
:10D3B0001F466FF06D084DB121462846FEF78FF8E5
:10D3C000B0F1000802D04046BDE8F0814EB104F152
:10D3D00060013046F9F72EF9B0F1000801D040465F
:10D3E000F2E74FB104F168013846FEF751F8B0F1A9
:10D3F000000801D04046E7E70020E5E708B5014610
:10D4000008880090BDF8000008BD03B5BDF8041001
:10D4100001800CBD01460806000C40EA112070474F
:10D420000146C86808B9012070470020FCE72DE9D3
:10D43000F04105460C4616461F466FF06D0800BFCA
:10D440003A4631462046FAF7F1F8B0F1000800D02C
:10D4500019E000BF00BF0AE000BF2A1D2146204698
:10D46000F9F73CFBB0F1000800D00CE000BFB4F9C4
:10D470000400002805DA00212046F9F79AFC00286C
:10D48000EAD100BF00BF4046BDE8F08180B1FFFF98
:10D4900080B0FFFF2DE9F05F04460E4617461D469B
:10D4A000DDE90CABDDE90A893A463146201D00F082
:10D4B0007DF82DB14246294604F10C0000F076F8C3
:10D4C0005246494604F1140000F070F804F13400AB
:10D4D000DDE9111200F06AF8594604F11C000E9AB9
:10D4E00000F064F804F12400DDE90F1200F05EF8AA
:10D4F00004F12C0001218180C1803049016000BF0E
:10D50000201DF9F76BF9E06304F13400F9F766F9CF
:10D510002064012060641398A0650020E065BDE8E8
:10D52000F09F30B58BB004460D462046FDF769FFED
:10D530002046FDF71CFF2570032D02D0042D31D1AC
:10D5400018E01F4820211F4ACDE90612CDE9081036
:10D550001D481E4ACDE90212CDE904101C480021E5
:10D560000B462022CDE900101A492046FFF792FF12
:10D570000BB030BD18483021184ACDE90612CDE96C
:10D5800008101748174ACDE90212CDE904101648D1
:10D5900000210B463022CDE9001014492046FFF748
:10D5A00079FFE5E7002020701148E1E7012383803F
:10D5B000C2F38F03C3800160704700002038020867
:10D5C000C43C0208A43802088438020864380208FF
:10D5D0004438020824380208344B0208043F020889
:10D5E000D43E0208A43E0208743E0208443E0208EB
:10D5F00080B1FFFFF0B502460B46140600214FF440
:10D600007F401040094344EA00204FF47F0502EABE
:10D61000050600252C0644EA162441EA066120434B
:10D620004FF07F4502EA050600252C0244EA166405
:10D63000054641EA062045EA0401DDB22E063446DD
:10D640002E0A0D4640EA040145EA06004FF47F46E3
:10D6500003EA06052E02314340EA15604FF47F04C9
:10D660001C40250A044641EA050021464FF07F444C
:10D670001C4040EA1460F0BD70B50446002004E090
:10D680000D5C165C75402554401C9842F8D370BD63
:10D6900070B50446002004E00D5C165C754025540E
:10D6A000401C9842F8D370BD10B504464FF4C471C5
:10D6B000204614F054FC10BD2DE9FC5F81460C4659
:10D6C000CA46A346FE480078012818D1FC480078D5
:10D6D000012804D104F1080000F0DBFD06E004F1AC
:10D6E000080000F0D6FD0746FFF784FF4B084FEA1D
:10D6F00030052A4609F1080000F0D4FD1DE0F0488D
:10D700000078012804D104F1080000F0C2FD07E010
:10D7100004F1080000F0BDFDCDE90001FFF76AFF4C
:10D7200049084FEA30073846FFF764FF05462A46A6
:10D730000B4609F1080000F0B5FD9AF808009BF8C7
:10D74000071001F0010140EAC1108AF80800DC4826
:10D750000078012815D1DA480078012803D1204645
:10D7600000F097FD05E0204600F093FD0746FFF727
:10D7700041FF4B084FEA30052A46484600F092FD2B
:10D780001AE0CF480078012803D1204600F081FD3F
:10D7900006E0204600F07DFDCDE90001FFF72AFFFD
:10D7A00049084FEA30073846FFF724FF05462A4666
:10D7B0000B46484600F076FD9AF800009BF80F10E3
:10D7C00001F0010109B1E12100E0002148408AF89F
:10D7D0000000BDE8FC9F2DE9F04786B0054600201B
:10D7E00002900390049005900DF10808019001A8A3
:10D7F00043461022414600902846FBF713FE074699
:10D800001FB1384606B0BDE8F08700BF002085F89C
:10D81000810100BF05F1C001DDE90220C1E900205E
:10D8200005F1C000DDE90421C0E9022100BF0020AC
:10D83000286468640022AA64EA64042408E005F10C
:10D84000400202EB441102EB0410FFF735FF6410B5
:10D85000002CF4DC08244AE09948007801280DD116
:10D8600005F1400101EB0411D1E9009305F14001FC
:10D8700001EB04104A4600F015FD11E005F14000EF
:10D8800000EB0410D0E900211046FFF7B3FE8146FB
:10D890000B4605F1400101EB04104A4600F002FD81
:10D8A0008748007801280DD105F1400101EB0412F1
:10D8B00001EB041101F10800D2E902934A4600F09D
:10D8C000F1FC13E005F1400000EB0410D0E9022167
:10D8D0001046FFF78FFE81460B4605F1400101EB34
:10D8E000041101F108004A4600F0DCFC6410002C31
:10D8F000B2DC022412E001260DE005F1400303EB47
:10D90000061203EB041104EB060C03EB0C101023BE
:10D91000FFF7BEFE761CA642EFDB6400102CEADBAC
:10D9200000BF00BF00206DE72DE9F04780460E469E
:10D9300017461C466FF06D09802C08D0C02C06D00D
:10D94000B4F5807F03D06FF01300BDE8F0870122AB
:10D9500021463046FBF761FC054615B96FF0130010
:10D96000F3E7284608B9002102E0017901F01F0120
:10D97000102902D06FF01300E7E74046FBF775FC73
:10D9800029464046FBF784FCB0F1000901D0484627
:10D99000DBE70123224639464046FBF796FCB0F10F
:10D9A000000901D04846D0E74046FFF714FFB0F128
:10D9B000000901D04846C8E70020C6E72DE9F04F2E
:10D9C00089B080460C4615460026002704A803901F
:10D9D000E07B00F00F0AE07B4FEA101B05EB0A1713
:10D9E000387A00F00F0938780207D7E902030009F6
:10D9F00040EA037042EA1312CDE90602D7E90001BA
:10DA0000000940EA01700909CDE904012D4830F808
:10DA100019000304DDE904215940CDE9042105EB97
:10DA20000B12102303990846FFF732FE0E2657E02B
:10DA3000A05D00F00F0AA05D4FEA101B069800F0F1
:10DA40000F0904980207DDE90601000940EA0170A8
:10DA50000B091A43CDE90602DDE90401000940EA99
:10DA600001700909CDE90401164830F81900DDE913
:10DA7000041282EA0040CDE9041005EB0A121023DB
:10DA800003990846FFF704FE069800F00F09049872
:10DA90000207DDE90603000940EA037042EA1312B7
:10DAA000CDE90602DDE90401000940EA0170090937
:10DAB000CDE90401034830F81900DDE9041203E060
:10DAC000344E0208364E020882EA0040CDE90410C6
:10DAD00005EB0B12102303990846FFF7D9FD761EBC
:10DAE000002EA5DAFC480078012809D1DDE90401FF
:10DAF00002460B46CDE90001404600F0D3FB0BE0A7
:10DB0000DDE904211046FFF775FD02460B46CDE91D
:10DB10000001404600F0C6FBEF48007801280AD11A
:10DB2000DDE9060102460B46CDE9000108F10800D7
:10DB300000F0B8FB0CE0DDE906211046FFF75AFDC6
:10DB400002460B46CDE9000108F1080000F0AAFBEF
:10DB500009B0BDE8F08F70B504460E46154694F83E
:10DB6000810130B904F1400231462846FFF726FF13
:10DB700000BF00BF70BD2DE9F04F89B004468B4651
:10DB800090461D466FF06D0007900020029025B171
:10DB900080EA00014040014304D06FF0130009B057
:10DBA000BDE8F08F04F58070002101664166816652
:10DBB000C166016741678167C16784F880B1C4F8B5
:10DBC0004011C4F84411C4F84811C4F84C110C2D8C
:10DBD00009D12A464146603014F09AF9012140F2F9
:10DBE0006F10015543E000200390049005900690CB
:10DBF0000820A5FB0067B8480078012805D1324607
:10DC00003B4605A800F04EFB0AE030463946FFF7D8
:10DC1000F1FC02460B46CDE9000105A800F042FBED
:10DC2000C14615E0102D01D2284600E010208246A2
:10DC300053464A4604F5B0710846FFF71DFD04F54A
:10DC4000B07211462046FFF786FFA5EB0A05D144C6
:10DC5000002DE7D1102303AA04F5B0710846FFF7A1
:10DC60000BFD04F5B07211462046FFF774FF02A8C1
:10DC700004F5A873102204F5B07100902046FBF75C
:10DC8000D1FB0790079808B1079888E7002086E73E
:10DC90002DE9FC5F04468B461546D4F84821D4F89C
:10DCA0004C01521940F10000CDE9002004F5A472A6
:10DCB0000CCADDE90070B91A984106D30198410FEA
:10DCC000002041404040014303D06FF01300BDE805
:10DCD000FC9F10220023D4F848713846D4F84C1128
:10DCE00014F0DAF89146DA46B9F1000F25D0C9F1FF
:10DCF0001006AE4200D92E4604F5B87202EB0901B7
:10DD000002EB090033465246FFF7B6FC09EB06006A
:10DD1000102805D104F5B87211462046FFF71BFF05
:10DD2000D4F84831D4F84C019A1940F10000C4F8F5
:10DD30004821C4F84C01AD1BB244D4F84821D4F8B2
:10DD40004C01521940F10000C4F84821C4F84C01BC
:10DD50000FE01023524604F5B8710846FFF78CFC1B
:10DD600004F5B87211462046FFF7F5FE103D0AF1A2
:10DD7000100A102DEDD235B12B46524604F5B8717C
:10DD80000846FFF779FC0020A1E770B50446524829
:10DD90000078012804D104F10C0000F075FA04E0C9
:10DDA00004F10C0000F070FA00BA05466D1C4A48F8
:10DDB0000078012805D1294604F10C0000F067FA2B
:10DDC00004E029BA04F10C0000F061FA70BD2DE9FD
:10DDD000FC4704460E4615469946DDE90AA76FF052
:10DDE0006D080020019001A83346102204F5B0719F
:10DDF00000902046FBF716FB8046B8F1000F06D0D6
:10DE00001021304604F056F94046BDE8FC8794F8EE
:10DE1000800138B904F5B872511950194B46524671
:10DE2000FFF72AFC71194B4652463846FFF724FC8F
:10DE300094F88001012807D104F5B87251195019DE
:10DE40004B463A46FFF718FC0020DEE72DE9F04F7D
:10DE500087B00546894614469A466FF06D000690D5
:10DE60004E4657460020029003900490059010986B
:10DE7000A04204D26FF0150007B0BDE8F08F1198F2
:10DE800004600CB90020F7E7CA4506D9AAEB0900DF
:10DE9000A04202D26FF01300EEE7D5F84021D5F88A
:10DEA0004401121940F10000D5F84031D5F8441171
:10DEB000D21A88410CD3D5F84021D5F84401131962
:10DEC00040F100006FF01F020F21D21A814105D2EC
:10DED0006FF01300D0E70000344E02080022D5F89E
:10DEE00040115140D5F844015040014313D1102254
:10DEF0000023D5F848B15846D5F84C1113F0CCFFA3
:10DF000000214A404B401A4305D005F5B87211462E
:10DF10002846FFF720FE10220023D5F840B15846CE
:10DF2000D5F8441113F0B8FF9046B8F1000F2BD08C
:10DF3000C8F1100BA34500D9A3465B46424602A98F
:10DF40002846CDE90067FFF742FF069008B1069822
:10DF500092E708EB0B00102805D105F5B8721146C1
:10DF60002846FFF7F8FDD5F84021D5F8440112EB1B
:10DF70000B0240F10000C5F84021C5F84401A4EBB4
:10DF80000B045E445F4400BFD5F84011D5F844014E
:10DF9000091940F10000C5F84011C5F8440118E026
:10DFA00005F5B070FFF7F1FE1023002202A9284604
:10DFB000CDE90067FFF70BFF069008B106985BE715
:10DFC00005F5B87211462846FFF7C5FD103C10361E
:10DFD0001037102CE4D27CB105F5B070FFF7D5FEF8
:10DFE0002346002202A92846CDE90067FFF7EFFE8D
:10DFF000069008B106983FE7102102A804F05AF8ED
:10E00000002039E72DE9F04F87B004469A46DDE954
:10E0100010B90020CAF8000004F5A07408210023FC
:10E02000D4E90002A0FB015E02FB01E100FB031644
:10E0300008234FF0000CD4E90212A1FB037E02FB7F
:10E0400003E201FB0C28D4E90010A4F5A07400231E
:10E0500059405840014312D104F5A47003C810225E
:10E06000CDE9000113F018FF00214A404B401A434C
:10E0700005D004F5B87211462046FFF76CFDB9F1E2
:10E08000100F02D8B9F1040F04D26FF0130007B0DB
:10E09000BDE8F08F04F5A07003C810220023CDE97D
:10E0A000000113F0F9FE00214A404B401A4305D00D
:10E0B00004F5B87211462046FFF74DFD4A4604F5B7
:10E0C000A871584613F024FF002185EA0100714031
:10E0D000084306D1002187EA010088EA01010843CC
:10E0E0004DD0002002900390049005907048007875
:10E0F000012804D1414602A800F0C9F804E098FACA
:10E1000088F102A800F0C3F869480078012804D11A
:10E11000394603A800F0BBF803E039BA03A800F0C1
:10E12000B6F863480078012804D1314604A800F00D
:10E13000AEF803E031BA04A800F0A9F85C48007812
:10E14000012804D1294605A800F0A1F803E029BA66
:10E1500005A800F09CF8102302AA04F5B87108463F
:10E16000FFF78AFA04F5B87211462046FFF7F3FC70
:10E170004B4604F5B87259465846FFF77DFA002021
:10E1800085E72DE9FF5F06460F4614461D46DDE98B
:10E1900010ABDDE90E896FF06D00039043462A460F
:10E1A00039463046FFF7E7FC039018B1039804B0F6
:10E1B000BDE8F09F524649463046FFF769FD03909F
:10E1C00008B10398F3E702A8CDE90040224659467A
:10E1D0003046129BFFF73AFE039008B10398E6E73A
:10E1E000DDE9131002AB0022CDE9000111463046F3
:10E1F000FFF708FF039008B10398D8E70020D6E79F
:10E200002DE9F04F8DB082460D4616461F46DDF8CB
:10E210005CB0DDF86C90DDF864806FF06D000C9000
:10E2200008A91A98CDE904980691039016983346E8
:10E230002A460021CDE9010B00975046FFF7A1FFC8
:10E240000C9018B10C980DB0BDE8F08F424608A9AB
:10E250001898FBF74DFD044634B12946484603F0B3
:10E2600029FF6FF01100EEE70020ECE710B504463F
:10E2700004B910BD2046FAF7F8FF4FF4C4712046E8
:10E2800003F018FF00BFF4E701460868704701601B
:10E2900070471CB502461068009050680190DDE997
:10E2A00000011CBD1FB502990160039941601FBDAB
:10E2B000344E020870B50446002004E00D5C165C84
:10E2C00075402554401C9842F8D370BD014603297F
:10E2D00002D0092904D101E0FA487047FA48FCE766
:10E2E0000020FAE70021016041608160704710B5AD
:10E2F00004460CB1206800B910BD606898B1206870
:10E300000078032802D0092808D103E0606800F0F3
:10E3100046FA04E0606811F025FE00E000BF00BF8F
:10E32000606815F0F1F8A06828B122689278510071
:10E33000A06803F0CAFE0C21204603F0BBFE00BF1C
:10E34000DAE770B505460C4645B1286830B12CB106
:10E35000206818B128682168884201D0DB4870BD68
:10E3600020680078032802D009280AD104E06168F7
:10E37000686800F01EFA06E06168686811F0FCFD4C
:10E3800001E0D248EBE700BF0020E8E770B50446A3
:10E390000D4616460CB9CD4870BD0DB9CB48FBE70C
:10E3A000256000206060A0602878032802D009283A
:10E3B00020D10FE000BF5821012013F025FE60603E
:10E3C000606810B9C1488038E6E7606800F0E0F99D
:10E3D00000BF11E000BF6821012013F015FE60604E
:10E3E000606810B9B9488038D6E7606811F0B0FDB0
:10E3F00000BF01E0B548CFE700BF66B1A9780220B1
:10E4000013F002FEA060A06828B92046FFF76FFF56
:10E41000AE488038C0E70020BEE710B504460CB116
:10E42000206808B9A94810BD20680078032802D0E8
:10E43000092809D103E0606800F0C4F9F3E700217E
:10E44000606811F0F8FDEEE7A048ECE770B504460F
:10E450000D4616460CB1206808B99C4870BD20686E
:10E460000078032802D009280CD105E0324629465D
:10E47000606801F00DF9F1E732462946606811F055
:10E48000E2FDEBE79148E9E770B504460D460CB1B3
:10E49000206808B98D4870BD20680078032802D034
:10E4A00009280AD104E02946606801F03CF9F2E746
:10E4B0002946606811F0D1FDEDE78448EBE72DE9CE
:10E4C000F04104460D4616461F4614B97F48BDE884
:10E4D000F0812078032802D009280DD105E03A46C2
:10E4E0003146284601F0C2F9F1E700233A463146A9
:10E4F000284606F091FDEAE77448E8E7014609B9C5
:10E50000002070474878FCE7014609B900207047B1
:10E510000878FCE76E48704770B505460DB90020D5
:10E5200070BD6C4C00E00834206828B12946206892
:10E5300013F04FFD0028F6D12079FFF7C7FEEFE773
:10E5400002460AB900207047624900E008310879A4
:10E5500018B1087913789842F8D10868F3E70146B2
:10E5600009B9002070470868FCE72DE9F04389B03D
:10E570000446884615466FF06D091CB1206808B145
:10E58000A06818B9514809B0BDE8F08320688078C8
:10E59000A8421BD22046FFF740FFB0F1000900D08F
:10E5A00043E02A4641462046FFF750FFB0F10009FC
:10E5B00000D03AE001A92046FFF766FFB0F100095C
:10E5C00000D032E0206845780DF10408A668216883
:10E5D0008978A0684718206881783622304613F081
:10E5E000B7FC206881785C22384613F0B1FC2B46DA
:10E5F000424631463046FFF75DFE2B4642463946DD
:10E600003846FFF757FE2046FFF707FFB0F1000935
:10E6100000D00AE02068827831462046FFF716FFD6
:10E62000B0F1000900D000E000BF202101A803F0F4
:10E6300041FD4846A7E770B504460D4616461CB195
:10E64000206808B1A06808B9204870BD3246294644
:10E650002046FFF7FBFEF8E7F0B589B004460E460A
:10E660006FF06D071CB1206808B1A06810B9174899
:10E6700009B0F0BD21688978A068451801A9204635
:10E68000FFF702FF071E01D03846F1E72046FFF7EB
:10E69000C4FE071E01D03846EAE720688278294682
:10E6A0002046FFF7D3FE071E01D03846E0E720687A
:10E6B000427801A92046FFF7C9FE071E0CD0384654
:10E6C000D6E70000584E02085B4E020800AFFFFF7D
:10E6D000604E02086C4E020831462046FFF7D4FE19
:10E6E000C6E770B504466FF06D061CB1206808B12E
:10E6F000A06808B9254870BDA5682046FFF78DFEC3
:10E70000061E01D03046F6E720688278294620466A
:10E71000FFF79CFEEFE72DE9FE4F04460E46174635
:10E720001D46DDE90C896FF06D0A14B91748BDE884
:10E73000FE8F6846FFF7D6FD012221466846FFF7A7
:10E7400025FEB0F1000A00D01AE03A46314668468C
:10E75000FFF70BFFB0F1000A00D011E04246294656
:10E760006846FFF768FFB0F1000A00D008E04946AC
:10E770006846FFF771FFB0F1000A00D000E000BF6B
:10E780006846FFF7B4FD5046D1E7000000AFFFFF39
:10E7900010B504465821204613F0E1FB10BD10B51A
:10E7A000044604B910BD5821204603F083FC00BF85
:10E7B000F8E770B504460D4658222946204613F066
:10E7C000A7FB70BD0146002008604860FE488860D5
:10E7D000FE4ACA60C2430A61FC4AD2434A61002031
:10E7E000704730B595B005460C46F94800780128C9
:10E7F00004D1204601F060F800BA02E0204601F0A2
:10E800005BF80190F2480078012804D1201D01F046
:10E8100053F800BA02E0201D01F04EF80290EC48D7
:10E820000078012805D104F1080001F045F800BA8C
:10E8300003E004F1080001F03FF80390E448007899
:10E84000012805D104F10C0001F036F800BA03E00C
:10E8500004F10C0001F030F80490DD480078012844
:10E8600005D104F1100001F027F800BA03E004F12B
:10E87000100001F021F80590D5480078012805D155
:10E8800004F1140001F018F800BA03E004F11400D8
:10E8900001F012F80690CE480078012805D104F165
:10E8A000180001F009F800BA03E004F1180001F0C3
:10E8B00003F80790C6480078012805D104F11C0030
:10E8C00000F0FAFF00BA03E004F11C0000F0F4FFCE
:10E8D0000890BF480078012805D104F1200000F01D
:10E8E000EBFF00BA03E004F1200000F0E5FF09901F
:10E8F000B7480078012805D104F1240000F0DCFFBE
:10E9000000BA03E004F1240000F0D6FF0A90B048FA
:10E910000078012805D104F1280000F0CDFF00BAED
:10E9200003E004F1280000F0C7FF0B90A84800782E
:10E93000012805D104F12C0000F0BEFF00BA03E06D
:10E9400004F12C0000F0B8FF0C90A14800780128D9
:10E9500005D104F1300000F0AFFF00BA03E004F18C
:10E96000300000F0A9FF0D9099480078012805D1EA
:10E9700004F1340000F0A0FF00BA03E004F1340019
:10E9800000F09AFF0E9092480078012805D104F11A
:10E99000380000F091FF00BA03E004F1380000F005
:10E9A0008BFF0F908A480078012805D104F13C00C4
:10E9B00000F082FF00BA03E004F13C0000F07CFFAD
:10E9C0001090A8681190E8681290286913906869FF
:10E9D000149000BFDDE913014840129908401499D2
:10E9E0004840019908447B49084411990844119012
:10E9F0001198C001119940EA516012990844119090
:10EA000000BF00BFDDE91201484011990840139989
:10EA100048400299084470490844149908441490E5
:10EA200014980003149940EA115011990844149065
:10EA300000BF00BFDDE91101484014990840129958
:10EA400048400399084465490844139908441390C1
:10EA500013984004139940EAD13014990844139054
:10EA600000BF00BF119914984840139908401199AC
:10EA70004840049908445A4908441299084412909D
:10EA800012988005129940EA912013990844129037
:10EA900000BF00BFDDE913014840129908401499F6
:10EAA0004840059908444F49084411990844119079
:10EAB0001198C001119940EA5160129908441190CF
:10EAC00000BF00BFDDE912014840119908401399C9
:10EAD000484006990844444908441499084414904D
:10EAE00014980003149940EA1150119908441490A5
:10EAF00000BF00BFDDE91101484014990840129998
:10EB00004840079908443949084413990844139028
:10EB100013984004139940EAD13014990844139093
:10EB200000BF00BF119914984840139908401199EB
:10EB30004840089908442E49084412990844129004
:10EB400012988005129940EA912013990844129076
:10EB500000BF00BFDDE91301484012990840149935
:10EB600048400999084423490844119908441190E0
:10EB70001198C001119940EA51601299084411900E
:10EB800000BF00BFDDE91201484011990840139908
:10EB900048400A99084418490844149908441490B4
:10EBA00014980003149940EA1150119908441490E4
:10EBB00000BF00BFDDE911014840149908401299D7
:10EBC00048400B99084419E00123456789ABCDEF14
:10EBD000844E020878A46AD756B7C7E8DB702024B1
:10EBE000EECEBDC1AF0F7CF52AC68747134630A8CD
:10EBF000019546FDD8988069AFF7448BA0F5244075
:10EC00004F3813990844139013984004139940EA1D
:10EC1000D13014990844139000BF00BF1199149883
:10EC2000484013990840119948400C990844FE49FE
:10EC3000084412990844129012988005129940EAEB
:10EC4000912013990844129000BF00BFDDE9130121
:10EC5000484012990840149948400D990844F349D6
:10EC600008441199084411901198C001119940EA83
:10EC7000516012990844119000BF00BFDDE91201F4
:10EC8000484011990840139948400E990844E849B2
:10EC9000084414990844149014980003149940EA05
:10ECA000115011990844149000BF00BFDDE9110113
:10ECB000484014990840129948400F990844DD498A
:10ECC000084413990844139013984004139940EA98
:10ECD000D13014990844139000BF00BF11991498C3
:10ECE0004840139908401199484010990844D24966
:10ECF000084412990844129012988005129940EA2B
:10ED0000912013990844129000BF00BFDDE9120161
:10ED10004840149908401399484002990844C7494B
:10ED2000084411990844119011984001119940EA42
:10ED3000D16012990844119000BF00BFDDE91101B4
:10ED40004840139908401299484007990844BC4923
:10ED5000084414990844149014984002149940EA05
:10ED6000D15011990844149000BF00BF1199149814
:10ED7000484012990840119948400C990844B149FB
:10ED8000084413990844139013988003139940EA98
:10ED9000914014990844139000BF00BFDDE91301AE
:10EDA0004840119908401499484001990844A649DF
:10EDB000084412990844129012980005129940EAEA
:10EDC000113013990844129000BF00BFDDE9120111
:10EDD00048401499084013994840069908449B49B3
:10EDE000084411990844119011984001119940EA82
:10EDF000D16012990844119000BF00BFDDE91101F4
:10EE0000484013990840129948400B99084490498A
:10EE1000084414990844149014984002149940EA44
:10EE2000D15011990844149000BF00BF1199149853
:10EE30004840129908401199484010990844854962
:10EE4000084413990844139013988003139940EAD7
:10EE5000914014990844139000BF00BFDDE91301ED
:10EE600048401199084014994840059908447A4946
:10EE7000084412990844129012980005129940EA29
:10EE8000113013990844129000BF00BFDDE9120150
:10EE9000484014990840139948400A9908446F491A
:10EEA000084411990844119011984001119940EAC1
:10EEB000D16012990844119000BF00BFDDE9110133
:10EEC000484013990840129948400F9908446449F2
:10EED000084414990844149014984002149940EA84
:10EEE000D15011990844149000BF00BF1199149893
:10EEF00048401299084011994840049908445949DA
:10EF0000084413990844139013988003139940EA16
:10EF1000914014990844139000BF00BFDDE913012C
:10EF200048401199084014994840099908444E49AD
:10EF3000084412990844129012980005129940EA68
:10EF4000113013990844129000BF00BFDDE912018F
:10EF5000484014990840139948400E990844434981
:10EF6000084411990844119011984001119940EA00
:10EF7000D16012990844119000BF00BFDDE9110172
:10EF80004840139908401299484003990844384969
:10EF9000084414990844149014984002149940EAC3
:10EFA000D15011990844149000BF00BF11991498D2
:10EFB00048401299084011994840089908442D4941
:10EFC000084413990844139013988003139940EA56
:10EFD000914014990844139000BF00BFDDE913016C
:10EFE000484011990840149948400D990844224915
:10EFF000084412990844129012980005129940EAA8
:10F00000113013990844129000BF00BFDDE91201CE
:10F0100048401499484006990844184908441199F1
:10F020000844119011982BE0BED75C892211906B97
:10F03000937198FD8E4379A62108B44962251EF686
:10F0400040B340C0515A5E26AAC7B6E95D102FD61C
:10F050005314440281E6A1D8C8FBD3E7E6CDE121F1
:10F06000D60737C3870DD5F4ED145A4505E9E3A952
:10F07000F8A3EFFCD9026F678A4C2A8D4239FAFF58
:10F080000001119940EA117012990844119000BFD3
:10F0900000BFDDE91101484013994840099908442F
:10F0A000FE4908441499084414901498C002149915
:10F0B00040EA515011990844149000BF00BF1199C3
:10F0C00014984840129948400C990844F44908445F
:10F0D00013990844139013980004139940EA1140BF
:10F0E00014990844139000BF00BFDDE913014840A4
:10F0F000119948400F990844EA4908441299084474
:10F1000012901298C005129940EA512013990844B0
:10F11000129000BF00BFDDE9120148401499484039
:10F1200002990844E0490844119908441190119843
:10F130000001119940EA117012990844119000BF22
:10F1400000BFDDE911014840139948400599084482
:10F15000D64908441499084414901498C00214998C
:10F1600040EA515011990844149000BF00BF119912
:10F17000149848401299484008990844CC490844DA
:10F1800013990844139013980004139940EA11400E
:10F1900014990844139000BF00BFDDE913014840F3
:10F1A000119948400B990844C249084412990844EF
:10F1B00012901298C005129940EA51201399084400
:10F1C000129000BF00BFDDE9120148401499484089
:10F1D0000E990844B84908441199084411901198AF
:10F1E0000001119940EA117012990844119000BF72
:10F1F00000BFDDE9110148401399484001990844D6
:10F20000AE4908441499084414901498C002149903
:10F2100040EA515011990844149000BF00BF119961
:10F22000149848401299484004990844A449084455
:10F2300013990844139013980004139940EA11405D
:10F2400014990844139000BF00BFDDE91301484042
:10F2500011994840079908449A490844129908446A
:10F2600012901298C005129940EA5120139908444F
:10F27000129000BF00BFDDE91201484014994840D8
:10F280000A9908449049084411990844119011982A
:10F290000001119940EA117012990844119000BFC1
:10F2A00000BFDDE911014840139948400D99084419
:10F2B000864908441499084414901498C00214997B
:10F2C00040EA515011990844149000BF00BF1199B1
:10F2D0001498484012994840109908447C490844C1
:10F2E00013990844139013980004139940EA1140AD
:10F2F00014990844139000BF00BFDDE91301484092
:10F3000011994840039908447249084412990844E5
:10F3100012901298C005129940EA5120139908449E
:10F32000129000BF00BF1499129860EA010013996F
:10F3300048400199084468490844119908441190CB
:10F3400011988001119940EA916012990844119036
:10F3500000BF00BF1399119860EA0100129948405C
:10F36000089908445D490844149908441490149875
:10F370008002149940EA915011990844149000BFFA
:10F3800000BF1299149860EA0100119948400F9942
:10F390000844534908441399084413901398C00330
:10F3A000139940EA514014990844139000BF00BFDC
:10F3B0001199139860EA010014994840069908448D
:10F3C000484908441299084412901298400512992D
:10F3D00040EAD12013990844129000BF00BF14994D
:10F3E000129860EA0100139948400D9908443E497B
:10F3F000084411990844119011988001119940EA2C
:10F40000916012990844119000BF00BF13991198A0
:10F4100060EA0100129948400499084433490844BD
:10F4200014990844149014988002149940EA915059
:10F4300011990844149000BF00BF1299149860EA13
:10F440000100119948400B9908442949084413992F
:10F45000084413901398C003139940EA514014993B
:10F460000844139000BF00BF1199139860EA01008F
:10F4700014994840029908441E49084412990844C6
:10F48000129012984005129940EAD120139908442D
:10F49000129000BF00BF149912982DE081F6718779
:10F4A00022619D6D0C38E5FD44EABEA4A9CFDE4B78
:10F4B000604BBBF670BCBFBEC67E9B28FA27A1EA94
:10F4C0008530EFD4051D880439D0D4D9E599DBE621
:10F4D000F87CA21F6556ACC4442229F497FF2A4346
:10F4E000A72394AB39A093FCC3595B6592CC0C8FD6
:10F4F0007DF4EFFFD15D848560EA010013994840F7
:10F5000009990844EF490844119908441190119849
:10F510008001119940EA916012990844119000BF4E
:10F5200000BF1399119860EA0100129948401099A0
:10F530000844E5490844149908441490149880023A
:10F54000149940EA915011990844149000BF00BFEB
:10F550001299149860EA01001199484007990844EB
:10F56000DA4908441399084413901398C003139977
:10F5700040EA514014990844139000BF00BF11990C
:10F58000139860EA0100149948400E990844D04944
:10F59000084412990844129012984005129940EAC2
:10F5A000D12013990844129000BF00BF14991298FB
:10F5B00060EA01001399484005990844C549084488
:10F5C00011990844119011988001119940EA9160B5
:10F5D00012990844119000BF00BF1399119860EA76
:10F5E0000100129948400C990844BB4908441499F9
:10F5F0000844149014988002149940EA915011998B
:10F600000844149000BF00BF1299149860EA0100EA
:10F610001199484003990844B04908441399084493
:10F6200013901398C003139940EA51401499084469
:10F63000139000BF00BF1199139860EA010014995C
:10F6400048400A990844A64908441299084412906F
:10F6500012984005129940EAD1201399084412905B
:10F6600000BFA86811990844A860E868129901448D
:10F67000E960286913990144296168691499014472
:10F680006961502101A802F015FD002015B030BDC0
:10F690002DE9F0470446884615466FF06D0915B907
:10F6A0000020BDE8F087207800F03F07C7F1400652
:10F6B000206828442060206820602068A84202D288
:10F6C0006068401C6060AFB1B54213D304F118010B
:10F6D000C8193246414612F01BFC04F118012046BD
:10F6E000FFF77FF8B0F1000901D04846D9E7B044F0
:10F6F000AD1B00270BE041462046FFF772F8B0F142
:10F70000000901D04846CCE708F14008403D402DB3
:10F71000F1D235B104F11801C8192A46414612F058
:10F72000F7FB0020BDE72DE9F04704460D466FF0DA
:10F730006D09207800F03F0680223046761C04F1E7
:10F7400018010A54382E07D8C6F1380104F11802FE
:10F75000901912F004FC14E0C6F1400104F1180203
:10F76000901912F0FCFB04F118012046FFF739F85C
:10F77000B0F1000900D073E0382104F1180012F054
:10F78000EEFB2068400F616840EAC10720684FEA3D
:10F79000C00854480078012806D198FA88F104F18D
:10F7A000500000F08CF804E0414604F1500000F0F5
:10F7B00086F84C480078012805D139BA04F1540084
:10F7C00000F07DF804E0394604F1540000F077F8C9
:10F7D00004F118012046FFF704F8B0F1000900D049
:10F7E0003EE040480078012805D1A06801BA2846CB
:10F7F00000F065F803E02846A16800F060F8394899
:10F800000078012805D1E06801BA281D00F057F8FA
:10F8100003E0281DE16800F052F832480078012822
:10F8200006D1206901BA05F1080000F048F804E0AB
:10F8300005F10800216900F042F82A480078012803
:10F8400006D1606901BA05F10C0000F038F804E057
:10F8500005F10C00616900F032F84FF0000900BFBB
:10F860002046FEF79CFF4846BDE8F087F0B597B00C
:10F8700004460D4616466FF06D0701A8FEF788FF97
:10F8800001A8FEF79FFF071E00D00FE02A46214681
:10F8900001A8FFF7FDFE071E00D007E0314601A8D2
:10F8A000FFF741FF071E00D000E000BF01A8FEF7F0
:10F8B00076FF384617B0F0BD014608687047016012
:10F8C000704700004F7EA86FE0E62CFE144301A3B2
:10F8D000A111084E827E53F735F23ABDBBD2D72A2A
:10F8E00091D386EB844E020870B50446F94D2E463E
:10F8F00005B10CB9002070BD0DE0706861688842E8
:10F9000007D1D4E90121306812F071FB08B928460B
:10F91000F1E714352E4630680028EED100BFEAE743
:10F9200070B506460C463046FFF7DEFF054615B9B2
:10F930006FF02D0070BD286920600020FAE770B5D7
:10F940000446E54D2E4605B10CB9002070BD0DE012
:10F9500070686168884207D1D4E90121306812F0EB
:10F9600046FB08B92846F1E714352E4630680028D2
:10F97000EED100BFEAE770B506460C463046FFF709
:10F98000DEFF054615B96FF02D0070BD28692060B7
:10F990000020FAE770B50446D04D2E4605B10CB9EB
:10F9A000002070BD0DE070686168884207D1D4E91D
:10F9B0000121306812F01BFB08B92846F1E7103529
:10F9C0002E4630680028EED100BFEAE770B5064643
:10F9D0000C463046FFF7DEFF054615B96FF02D00E7
:10F9E00070BDE86820600020FAE770B50446BC4DA1
:10F9F0002E4605B10CB9002070BD0DE0706861683D
:10FA0000884207D1D4E90121306812F0F0FA08B930
:10FA10002846F1E710352E4630680028EED100BFA9
:10FA2000EAE770B506460C463046FFF7DEFF0546AE
:10FA300015B96FF02D0070BDE86820600020FAE76E
:10FA400070B50446A74D2E4605B10CB9002070BD17
:10FA50000DE070686168884207D1D4E901213068FF
:10FA600012F0C5FA08B92846F1E714352E46306879
:10FA70000028EED100BFEAE770B506460C463046D6
:10FA8000FFF7DEFF054615B96FF02D0070BDE86881
:10FA900020600020FAE72DE9F04107460D461646A2
:10FAA0003846FFF7CDFF04461CB96FF02D00BDE8C6
:10FAB000F081207C2870607C30700020F7E730B542
:10FAC00004460D4687490CE0487CA04208D1087CDA
:10FAD000A84205D10868106048681860002030BD51
:10FAE000143108680028EFD16FF02D00F7E770B5EA
:10FAF00004467D4D2E4605B10CB9002070BD0DE0C9
:10FB000070686168884207D1D4E90121306812F039
:10FB10006EFA08B92846F1E714352E4630680028F9
:10FB2000EED100BFEAE770B506460C463046FFF757
:10FB3000DEFF054615B96FF02D0070BD287C2070E2
:10FB40000020FAE710B503460C46674909E0087C37
:10FB5000984205D10868206048681060002010BDF8
:10FB6000143108680028F2D16FF02D00F7E770B566
:10FB700004465E4D2E4605B10CB9002070BD0DE067
:10FB800070686168884207D1D4E90121306812F0B9
:10FB90002EFA08B92846F1E714352E4630680028B9
:10FBA000EED100BFEAE770B506460C463046FFF7D7
:10FBB000DEFF054615B96FF02D0070BD287C207062
:10FBC0000020FAE710B503460C46484909E0087CD6
:10FBD000984205D10868206048681060002010BD78
:10FBE000143108680028F2D16FF02D00F7E770B5E6
:10FBF00004463F4D2E4605B10CB9002070BD0DE006
:10FC000070686168884207D1D4E90121306812F038
:10FC1000EEF908B92846F1E714352E463068002879
:10FC2000EED100BFEAE770B506460C463046FFF756
:10FC3000DEFF054615B96FF02D0070BD287C2070E1
:10FC40000020FAE710B503460C46294909E0087C74
:10FC5000984205D10868206048681060002010BDF7
:10FC6000143108680028F2D16FF02D00F7E770B565
:10FC70000446204D2E4605B10CB9002070BD0DE0A4
:10FC800070686168884207D1D4E90121306812F0B8
:10FC9000AEF908B92846F1E714352E463068002839
:10FCA000EED100BFEAE770B506460C463046FFF7D6
:10FCB000DEFF054615B96FF02D0070BD287C207061
:10FCC0000020FAE770B504460B4D2E4605B1ACB9DD
:10FCD000002070BD884E02082C500208E050020837
:10FCE0006051020880510208D051020820520208D7
:10FCF0005C52020870520208E85202080DE0706877
:10FD00006168884207D1D4E90121306812F06FF9A7
:10FD100008B92846DDE714352E4630680028EED1B4
:10FD200000BFD6E770B506460C463046FFF7CAFF5F
:10FD3000054615B96FF02D0070BD287C207000209D
:10FD4000FAE710B503460C46F04909E0087C9842F2
:10FD500005D10868206048681060002010BD14318B
:10FD600008680028F2D16FF02D00F7E770B504465F
:10FD7000E74D2E4605B10CB9002070BD0DE070684E
:10FD80006168884207D1D4E90121306812F02FF967
:10FD900008B92846F1E714352E4630680028EED120
:10FDA00000BFEAE770B506460C463046FFF7DEFFB7
:10FDB000054615B96FF02D0070BD287C207000201D
:10FDC000FAE72DE9F74F82B00F4615466FF06D093F
:10FDD000029801903E460024B7F1004F04D36FF023
:10FDE000630005B0BDE8F08F686810B96FF05F0080
:10FDF000F7E74FF000084FE0B4F1007F02D36FF057
:10FE00006700EEE73CB9A86810F80800802802D126
:10FE10006FF06700E5E7E401A86810F8080000F05B
:10FE20007F000443A86810F8080000F0800088BB39
:10FE3000BE421AD1502C04D34FF0320AA4F1500B19
:10FE400009E0282C04D34FF0310AA4F1280B02E07A
:10FE50004FF0300AA3465346AEA23146CDF800B06B
:10FE6000019813F0D3F8814606E02346ABA2314651
:10FE7000019813F0CBF88146B9F1020F01DBB145CF
:10FE800002D36FF00A00ACE7A6EB090601984844DC
:10FE90000190002408F1010868684045ACD814B10D
:10FEA0006FF05F009DE7B81B9BE730B503466FF02E
:10FEB00067040020186015E00024994D1868A842D6
:10FEC00002D96FF0670030BD186800EB8000400079
:10FED00018601D6808680078303828441860086881
:10FEE000401C08600868904207D2086800783028F3
:10FEF00003DB086800783928DEDD2046E3E70146A9
:10FF0000002000BFC909401C0029FBD170472DE922
:10FF1000F04104460F4615462846FFF7F0FF064617
:10FF20002068381AB04203D26FF00A00BDE8F081B1
:10FF300005F07F01701E22681154ED09022008E0CF
:10FF400005F07F0141F08001331A2268D154ED0998
:10FF5000401CB042F4D92068304420600020E5E71E
:10FF60002DE9F04F89B004460F4693466FF06705C0
:10FF7000089707EB0B0600200790824600BF05E0BC
:10FF8000395C2E2901D10AF1010A401C5845F7D3EA
:10FF9000BAF1000F02D0BAF17F0F04D96FF06700F9
:10FFA00009B0BDE8F08F0520049004980AFB00F02A
:10FFB00003900121039812F027F8A060A06810B9FF
:10FFC0006FF06900ECE7A0680290A168039808440C
:10FFD0000190324608A906A8FFF767FF054605B15C
:10FFE0008CE00698022802D96FF0670586E0089831
:10FFF000B04203D2089800782E2802D06FF067052F
:020000040801F1
:100000007CE00898401C0890324608A905A8FFF734
:100010004CFF054605B171E00698022805D2059807
:10002000272802D96FF0670568E00898B0420AD225
:10003000089800782E2803D10898401C089002E008
:100040006FF067055AE0069800EB80004FF0FF3133
:10005000A1EBC0000599884202D26FF067054DE020
:10006000069800EB8000059901EBC00202A80199F7
:10007000FFF74DFF054605B140E01DE0324608A9F7
:1000800007A8FFF712FF054605B137E00898B04210
:100090000AD2089800782E2803D10898401C0890AE
:1000A00002E06FF0670529E002A8079A0199FFF7BF
:1000B0002EFF054605B121E00898B042DED3A068C6
:1000C0000299A1EB00080121404611F09DFF8146F5
:1000D000B9F1000F02D16FF069050FE042464846C2
:1000E000A16811F015FFA06813F00EFAC4F808908B
:1000F000C4F8048006202060002051E7A06813F0B7
:1001000003FA0020A0606060284649E7E852020830
:100110002453020825632E25750000002E25750046
:1001200099999919002101604160816070472DE91A
:10013000F04704460E4617463946304611F00FFF89
:10014000002532E02078302806DB2078392803DCCF
:100150002078A0F1300816E02078412806DB2078CE
:10016000462803DC2078A0F137080CE020786128CD
:1001700006DB2078662803DC2078A0F1570802E02F
:10018000FA48BDE8F08705F0010008B1404601E0FB
:100190004FEA0810814606EB5500007840EA090056
:1001A00006EB550108706D1C641CB5EB470FC9D3F5
:1001B0000020E6E72DE9F04F87B005460C461646CD
:1001C0001F46DDF840906FF06D0A04A8FEF78AF82C
:1001D0000320FEF77BF883460022594604A8FEF769
:1001E000D5F8B0F1000A00D064E004A8FEF715F9D4
:1001F000B0F1000A00D05DE04A46394604A8FEF797
:1002000025F9B0F1000A00D054E00822314604A8D4
:10021000FEF71CF9B0F1000A00D04BE0694604A8D3
:10022000FEF732F9B0F1000A00D043E0102C05D8F7
:1002300022466946284611F06BFE3BE010226946D3
:10024000284611F065FE04A8FEF7E7F8B0F1000AB1
:1002500000D02FE01022694604A8FEF7F7F8B0F1AD
:10026000000A00D026E04A46394604A8FEF7EEF818
:10027000B0F1000A00D01DE00822314604A8FEF7C4
:10028000E5F8B0F1000A00D014E0694604A8FEF7D2
:10029000FBF8B0F1000A00D00CE04FF01008202C61
:1002A00001D2A4F110084246694605F1100011F090
:1002B0002FFE00BF04A8FEF71AF81021684601F0CF
:1002C000F9FE504607B0BDE8F08F2DE9F04389B044
:1002D00004460D4616461F46DDF840806FF06D0956
:1002E00005A80FF0F9FC3B462246082103A8CDF8EB
:1002F0000080FFF75FFFB0F1000900D011E003A913
:1003000005A80FF0FEFCB0F1000900D009E000954F
:1003100023463246002105A801950FF021FD8146B4
:1003200000BF05A80FF0DEFC082103A801F0C2FE03
:10033000484609B0BDE8F0832DE9F04391B004468A
:100340000D4616461F46DDF860806FF06D0909A85E
:100350000FF049FD3B462246182103A8CDF8008046
:10036000FFF728FFB0F1000900D011E003A909A8A8
:100370000FF053FDB0F1000900D009E000952346CD
:100380003246002109A801950FF079FD814600BF92
:1003900009A80FF02FFD182103A801F08BFE484695
:1003A00011B0BDE8F0832DE9F04794B004460E4645
:1003B00015461F46DDE91C896FF06D0A0AA80FF08B
:1003C000B3FB43462246314602A8CDF80090FFF722
:1003D000F1FEB0F1000A00D012E0F20002A90AA872
:1003E0000FF0BEFBB0F1000A00D009E000952346F3
:1003F0003A4600210AA801950FF007FC824600BF8B
:100400000AA80FF098FB314602A801F053FE5046AF
:1004100014B0BDE8F08730B503461446481E1D5C95
:100420008D4201D9524830BD481B2060226805E04A
:10043000985CA84201D04E48F5E7521C8A42F7D397
:100440000020F0E72DE9FF4F89B0DDE9169A4FF063
:100450000008099818B947480DB0BDE8F08F0A990F
:100460000C9811F087FD04460CB94348F4E7DDE928
:100470000B1011F07FFD05460DB1A54201D83E4895
:10048000EAE70A9811F09EFD04442078202800D164
:10049000641C20780D2800D1641C20780A2801D122
:1004A000641C01E03448D7E72E460B9811F08AFD12
:1004B00006443078202800D1761C30780D2800D1F1
:1004C000761C30780A2800D1761C0C98311A1898BE
:1004D000016000200890281B162871DB162227A136
:1004E000204611F084FD00286AD10898401C08902D
:1004F000163420780D2800D1641C20780A2801D1F8
:10050000641C02E01C488038A6E7281B172815DB6E
:10051000172220A1204611F06AFD78B94FF0250876
:100520001734281B102805DB082203A92046FFF7F3
:10053000FEFD08B10D488FE7103444E0281B122857
:1005400041DB122219A1204611F051FD68B94FF08C
:1005500021081234281B102805DB082203A9204695
:10056000FFF7E5FD68B3014876E72CE000EEFFFFFA
:1005700080ECFFFF80EBFFFF80EFFFFF50726F63A7
:100580002D547970653A20342C454E4352595054BD
:100590004544000044454B2D496E666F3A20444562
:1005A000532D454445332D4342432C0044454B2DA8
:1005B000496E666F3A204445532D4342432C000058
:1005C0004BE0FFE71034281B0E2836DB0E2281A1FA
:1005D000204611F00CFD00282FD1281B162801DA27
:1005E000804839E7162280A1204611F000FD10B99D
:1005F0004FF0050813E0162281A1204611F0F7FC08
:1006000010B94FF006080AE0162283A1204611F027
:10061000EEFC10B94FF0070801E072481CE71634F1
:10062000281B202805DB102203A92046FFF77FFDA9
:1006300010B16C4880300FE72034B8F1000F01D1C1
:10064000684809E720780D2800D1641C20780A2822
:1006500001D1641C01E07648FEE6AC4201D3744847
:10066000FAE6281B234607AA002100900846F5F762
:10067000A2FD074607F12C0038B94FF4CE736DA2E6
:1006800039466B4800F0A1F8E6E6079808B97048CB
:10069000E2E60120079911F0B7FCB0F1000B02D19E
:1006A00063488038D8E6281B234607AA009058469E
:1006B0000799F5F780FD071E0BD05846079901F002
:1006C00004FD40F2A9135BA23946594800F07DF8B9
:1006D000C2E6089880B3B9F1000F06D158460799D1
:1006E00001F0F3FC3F488038B6E60027B8F1250F4B
:1006F00009D14B46CDF800A0594603A8079AFFF749
:100700001BFE07460BE0B8F1210F08D14B46CDF890
:1007100000A0594603A8079AFFF7D7FD0746B8F18E
:10072000050F0AD1CDE9009A5A46102103A8079B6C
:10073000FFF739FE074619E02FE0B8F1060F09D19F
:10074000CDE9009A5A46182103A8079BFFF72BFE14
:1007500007460BE0B8F1070F08D1CDE9009A5A46D9
:10076000202103A8079BFFF71EFE07462FB158461E
:10077000079901F0AAFC38466EE602AA5846079986
:10078000FFF749FE07462FB15846079901F09DFC37
:10079000384661E60298079000BF0998C0F800B09B
:1007A000079909984160002056E610B50446206874
:1007B00018B1D4E9000101F088FCA06812F0A4FE91
:1007C0000C21204601F076FC10BD10B504466018DF
:1007D00010BD000044454B2D496E666F3A204145DF
:1007E000532D000080EDFFFF44454B2D496E666F91
:1007F0003A204145532D3132382D4342432C0000DD
:1008000044454B2D496E666F3A204145532D313991
:10081000322D4342432C000044454B2D496E666FF8
:100820003A204145532D3235362D4342432C0000AA
:1008300000EFFFFF2E2E5C6D626564746C735C6C60
:100840006962726172795C70656D2E6300000000F0
:1008500080EBFFFF10B504460CB1206808B90020FA
:1008600010BD2068816820468847F9E7014609B134
:10087000086808B90020704708680078FBE7002185
:1008800001604160704710B5044604B910BD20688E
:1008900030B12068806A18B1D4E90020916A884795
:1008A0000821204601F006FC00BFEFE701460129C0
:1008B00004D0022904D0032906D103E0FB48704785
:1008C000FB48FCE7FB48FAE70020F8E770B505466F
:1008D0000C460CB1286808B1F74870BD606A28B1B1
:1008E000606A8047686008B9F448F6E72C60002029
:1008F000F3E72DE9F04704460E4617469846DDF823
:1009000020A0DFF8BC93206810B1EB48BDE8F08769
:10091000D9F824008047606008B9E848F6E7C4F8D1
:10092000009065682E606F60C5F80880C5F80CA05F
:100930000020EBE770B504460D460CB1206808B9FD
:10094000002070BD2068C16828468847F9E770B567
:1009500005460C46206808B1002070BD00BF28463F
:10096000FDF7B4FC0646FDF7C9FD2060206810B90C
:100970004FF0FF30F1E70020EFE72DE9FF4383B0B0
:1009800004460D461646DDE90F890E9F0DB90698FF
:1009900020B11EB9C84807B0BDE8F083206820B177
:1009A00006A92846FFF7D3FF08B1C348F3E720683C
:1009B000006910B9C0488038EDE7CDE900782068BB
:1009C000D0F810C0324629462046069BE047E2E7B1
:1009D0002DE9FE4304460D4616461F46DDE90A8909
:1009E00000203B4632462946CDE900890290204648
:1009F000FFF7C3FFBDE8FE832DE9F04F85B0064643
:100A00000C4615461F46DDF844A0DDE90E8917B9EE
:100A1000B9F1000F06D0B8F1000F03D1A64805B018
:100A2000BDE8F08F286808B9A348F8E731462846A2
:100A3000FFF780FF10B9A0488038F0E7062E0CD0F1
:100A40000CB19D48EBE710984B4642463946CDE93C
:100A5000000A2846FFF7BCFFE1E72846FFF706FF3C
:100A6000012801D09748DAE76FF06D0B0CB9924876
:100A7000D5E70494284600F05BF9504501D9924827
:100A8000CDE7D5E9000100F05BF9039004991098D7
:100A90004968049A12784346CDE9002102904A46FB
:100AA0003946039803F0D8FC8346BBF1000F01D010
:100AB0005846B4E7284600F03BF9504502D2814839
:100AC0008030ACE70020AAE72DE9FF4F85B004464F
:100AD0000D46164612AF97E8800F0DB9089820B161
:100AE0001EB9754809B0BDE8F08F206820B108A98B
:100AF0002846FFF72CFF08B16F48F3E720684069EC
:100B000010B96D488038EDE78DE8800F2068D0F887
:100B100014C0324629462046089BE047E2E72DE90B
:100B2000FF4F87B004460D46164614AF97E8800F76
:100B300000208DE8800F05903246294620460A9B0A
:100B4000FFF7C2FF0BB0BDE8F08F2DE9F04F85B085
:100B500006460C4615461F46DDE90FAB206818B95E
:100B6000554805B0BDE8F08F31462046FFF7E2FE5C
:100B700010B951488038F4E7062E0ED0DDE9112176
:100B80001398CDE900ABCDE9022104903A462946FD
:100B900020460E9BFFF7C3FFE3E7204600F0C8F8AE
:100BA000584501D94948DCE70EA92846FFF7CFFE92
:100BB00008B14148D5E7D4E9000100F0C1F880460A
:100BC0000E982B468DE881044046DDE9121203F0B1
:100BD000BCFA8146B9F1000F03D1D8F8041011987E
:100BE00001604846BDE72DE9FF5F04460D46164605
:100BF0001F46DDE910ABDDE90E89206818B92E48E3
:100C000004B0BDE8F09F2068806910B92A48803898
:100C1000F6E78DE8000F20683B4632462946D0F8BB
:100C200018C02046E047EBE72DE9FF5F04460D467C
:100C300016461F46DDE910ABDDE90E89206818B9BC
:100C40001D4804B0BDE8F09F2068C06910B91A487B
:100C50008038F6E78DE8000F20683B46324629468B
:100C6000D0F81CC02046E047EBE72DE9F0410546EF
:100C70000C4616461F46286808B1206810B90E4871
:100C8000BDE8F0810EB90C48FAE72068006A08B99F
:100C90000C48F5E720680078052819D12868007805
:100CA00001281FD004488038EAE700004C530208AE
:100CB0007C530208AC53020880C1FFFF80C0FFFFD5
:100CC000DC53020880C6FFFF80BCFFFF80C7FFFF28
:100CD00020680078072805D028682168884201D05C
:100CE0001C48CDE720683B4632462146D0F820C05C
:100CF0002846E047C4E770B504460D46206810B9A1
:100D00001448803070BD2068C06A08B91148F9E7FE
:100D100020682946C26A204690470020F2E7014633
:100D200009B1086808B90CA0704708684068FBE77B
:100D300010B504462046FFF78DFDC01DC00810BD4C
:100D400003B56846FFF792FD012801D101980CBD5B
:100D50000020FCE700C1FFFF696E76616C696420CA
:100D6000504B000070B504460D46D4E9000100F078
:100D700070F80646D4E9000100F05AF8007840B156
:100D8000D4E9000100F054F80078A84201D03948B5
:100D900070BD29463046FCF7C4FBF9E72DE9F04168
:100DA00005460E461746D5E9000100F052F8804688
:100DB00098F800003B4632464146FCF7F3F90446FA
:100DC0002CB12C482CA102191046BDE8F08100205E
:100DD000FBE72DE9FC470546884691461E460A9FDB
:100DE0006C6804F11C0304F1600204F16801204600
:100DF000CDE90067FCF720F8BDE8FC872DE9F0415C
:100E000005460E4617466C683B46324604F16801BB
:100E10002046FAF7A1FD8046B8F1000F02D0404607
:100E2000BDE8F08104F168012046FBF77AFFF7E79F
:100E300013B56846FFF71AFD022804D0032803D033
:100E4000042804D101E000BF00BF01981CBD0020B0
:100E5000FCE713B56846FFF709FD022804D0032814
:100E600003D0042804D101E000BF00BF01981CBDDD
:100E70000020FCE700C3FFFF2E2E5C6D62656474EA
:100E80006C735C6C6962726172795C706B5F6563D4
:100E9000632E63000146012901D0062901D10120FA
:100EA00070470020FCE770B504466568284602F0EC
:100EB000ABF870BD2DE9FC5F0446894615461E4619
:100EC000DDE90CA76FF06D0B60680190019802F0EE
:100ED000A2F88046474502D2CA48BDE8FC9F2B468F
:100EE00032464946CDF800A0019803F0F8FBB0F176
:100EF000000B01D05846F0E7474501D9C248ECE75E
:100F00000020EAE72DE9FF5F04460D4616461F461E
:100F1000DDE9108BDDE90E9A60680390039802F01A
:100F20007AF8C8F80000D8F80000504504D9B6484F
:100F3000803004B0BDE8F09F2B46CDE901690097F1
:100F40005946129A039803F05EFAF2E72DE9FF5F23
:100F500004460D4616461F46DDE910ABDDE90E8955
:100F600060680390039802F056F8B04203D0A74897
:100F700004B0BDE8F09F43465A4651468DE8A002B2
:100F8000039802F0D0FFF3E72DE9FE4F04460D462B
:100F900016461F46DDE90EABDDE90C89606802905C
:100FA000029802F038F8C8F80000D8F80000484568
:100FB00003D994488038BDE8FE8F33465A465146DF
:100FC000CDE90057029802F064FEF4E72DE9F04104
:100FD00004460D4616461F466968606802F090F99F
:100FE000BDE8F08110B57821012011F00DF804461C
:100FF00014B1204601F0DEFF204610BD10B50446B6
:10100000204601F0D9F8204612F07EFA10BD426861
:1010100001230B707EA34B6002F108038B600C313F
:1010200001230B707CA34B6002F110038B607047AF
:101030000146022903D0032901D0042901D101204E
:1010400070470020FCE701464A68D06B70472DE9E5
:10105000F04104460D4616461F4669683B46324637
:101060006068FCF72DF9BDE8F08110B58021012002
:1010700010F0CAFF044614B12046FAF79AF9204648
:1010800010BD10B504462046FAF7F1F9204612F0DB
:101090003BFA10BD426802230B7061A34B6002F162
:1010A00068038B6070470146022901D0032901D1F2
:1010B000012070470020FCE70146012900D170475C
:1010C0000020FCE770B504466568E9682868884731
:1010D000C00070BD2DE9FE4F06460F46904699466A
:1010E000DDE90CAB0E9D7468E168206888472860D4
:1010F0002868B0F5806F02D94B48BDE8FE8F28689C
:10110000584502D940488030F7E7CDE9018ACDF84B
:1011100000903B46D4F808C02068DDE90F12E04794
:10112000EBE72DE9F84F05460E4617469846DDE9F0
:101130000BABDDF828906C68E16820688847B842FE
:1011400002D03248BDE8F88FCDF800A043463246C1
:101150004946D4E9000CE047F4E72DE9F043ADF24D
:101160003C4D07460C4615461E46002006906FF083
:101170006D082046FFF7A6FF81463846FFF793FE2D
:10118000814504D029480DF23C4DBDE8F0832A2268
:10119000202107A810F0DCFE06A84FF4806102AA07
:1011A00061C201910FA8202307AA002100902046C8
:1011B000FFF790FFB0F1000801D04046E3E70FA928
:1011C0000698202307AACDE9001000213846FFF732
:1011D00071FE08B11548D6E70020D4E710B51021FC
:1011E000012010F011FF04461CB11021204610F020
:1011F000B6FE204610BD10B504461021204600F072
:1012000064FF10BD80BCFFFF00C7FFFF80BFFFFF72
:101210007273612E4E0000007273612E4500000053
:1012200065636B65792E510080C1FFFF00BEFFFF33
:101230000146302901D1012070470020FCE72DE94B
:10124000FE4305460C466FF06D06A8680290D5E98E
:10125000011000EB01096A46494602A8F4F7F7F9C4
:10126000061E07D07823F0A23146F74800F0FEFEB4
:10127000BDE8FE830098012802DB0098032801DD09
:10128000F148F5E7302301AA494602A8F4F74FF9DF
:10129000061E01D03046EBE7DDE9011047180623B2
:1012A00001AA394602A8F4F742F9061E01D03046D9
:1012B000DEE70198072805D1E4A1DDE9012010F05F
:1012C00096FE08B1E348D3E7DDE901100844029037
:1012D000221D394602A8F4F7D0F9061E06D0A12334
:1012E000D1A23146D84800F0C1FEC1E7201DF5F774
:1012F00075FAE0630298B84207D0A723CAA26FF03C
:101300006501D14800F0B2FEB2E7302301AA494698
:1013100002A8F4F70CF9061E01D03046A8E7DDE973
:10132000011000EB0108042301AA414602A8F4F7CA
:10133000FEF8061E07D104F10C00DDE90121F6F7E5
:1013400036F9061E06D0C123B7A23146BE4800F0CA
:101350008DFE8DE7DDE9011008440290042301AA07
:10136000414602A8F4F7E3F8061E07D104F1140081
:10137000DDE90121F6F71BF9061E06D0C823AAA253
:101380003146B14800F072FE72E7DDE90110084411
:101390000290032301AA414602A8F4F7C8F8061EEA
:1013A00003D1DDE90110084402900298404507D0BE
:1013B000D3239DA26FF06501A34800F057FE57E7C5
:1013C000042301AA494602A8F4F7B1F8061E06D084
:1013D000DB2395A231469C4800F048FE48E704F123
:1013E0001C012046DDE90132FAF7B6FA061E2AD0C2
:1013F00016F59D4F25D102980078022803D0029857
:10140000007803281DD1201DF5F7EFF9401C019944
:10141000884216D10198421E0299491C04F11C0011
:10142000F6F7C5F868B902980078811E04F1240027
:10143000F5F750F928B9012104F12C00F5F74AF924
:1014400008B1814814E7DDE901100844029004F175
:101450003402494602A8F4F710F9061E06D0F42318
:1014600071A23146784800F001FE01E704F1340032
:10147000F5F7B4F920640020FAE62DE9F04198B0C0
:1014800004460E4600276846F9F771FFF9F704FF96
:10149000054644E06846F9F7B4FF00BF297868467E
:1014A000FCF73FF8071E00D03EE000BFE06B0F994D
:1014B000884233D1206C109988422FD101A9201D78
:1014C000F5F719FC50BB03A904F10C00F5F713FC68
:1014D00020BB05A904F11400F5F70DFCF0B90DA926
:1014E00004F13400F5F707FCC0B907A904F11C00AA
:1014F000F5F701FC90B90BA904F12C00F5F7FBFB03
:1015000060B9002104F12400F5F705F980460021B7
:1015100009A8F5F700F9804500D103E06D1C287893
:101520000028B7D100BF00BF6846F9F76AFF2878E6
:10153000307017B9287800B9474F384618B0BDE861
:10154000F08170B598B004460D466FF06D066846A0
:10155000F9F70DFF69462046FFF771FE061E00D021
:1015600005E029466846FFF788FF064600BF0DA83C
:10157000F4F7F5FF01A8F4F7F2FF03A8F4F7EFFF83
:1015800005A8F4F7ECFF07A8F9F721FF304618B0DB
:1015900070BD2DE9F04105460E4614466FF06D070B
:1015A0002868301A012809DA4FF4B1731EA26FF0CF
:1015B0005F01254800F05AFDBDE8F08128680078F9
:1015C0002060206806280CD02068FFF731FE40B963
:1015D0004FF4B57314A26FF061011B4800F046FD93
:1015E000EAE7221D314628462368F3F7A0FF071ECD
:1015F00007D040F26F130CA23946134800F036FDB5
:10160000DAE72868A06028686168084428602868CC
:10161000B04223D04FF4BB7303A26FF065010A48B8
:1016200000F024FDC8E700002E2E5C6D6265647436
:101630006C735C6C6962726172795C706B70617200
:1016400073652E630000000000C3FFFF2A8648CEAA
:101650003D01010080C6FFFF80B1FFFF0020ABE726
:10166000F8B504460D466FF06D062068062806D1D1
:1016700069462046FEF797FA48B1F848F8BD694632
:101680002046FFF75EFF06460EB13046F6E79DF8AE
:1016900000102846FFF766FBF0E72DE9FE430746FA
:1016A000884615461C46DDF828906FF06D06002030
:1016B00020606060A06023466A4641463846F4F7E1
:1016C000E5F8061E0AD04FF4F173AFF2A4023146DA
:1016D000E248803800F0CAFCBDE8FE83294668462F
:1016E000FEF721FA064606F12E0038B9494668464B
:1016F000FEF799FA06460EB9022028700EB1D848B6
:10170000EAE72878012809D12068052801D0206857
:1017100008B9606810B1D1488038DDE70020DBE708
:101720002DE9F04387B004460E4617466FF06D056D
:10173000002002900190302306AA31462046F3F79C
:10174000F6FE051E0BD040F21123AFF224122946FB
:10175000C348803800F08AFC07B0BDE8F0832068F9
:101760000699461801A803AB02AA3146009020460C
:10177000FFF793FF051E01D02846EDE706AA314684
:101780002046F4F719F8051E08D040F21B23AFF2EB
:1017900068122946B34800F069FCDDE72068069925
:1017A0000844B04209D040F21F23AFF284126FF018
:1017B0006501AC4800F05AFCCEE79DF80800FFF741
:1017C00075F8B0F1000801D1A548C5E74146384693
:1017D000FFF77CF8051E01D02846BDE79DF80800FC
:1017E000012823D1D7E9000100F036FC81462068AA
:1017F000321A0146484601F060F8054625B92068CE
:10180000311A084420602CE015F1600F0CDC15F152
:101810006C0F09DB4FF40D73AFF2F41229469148B7
:1018200000F024FC05461CE08E4D1AE09DF80800EF
:10183000032803D09DF80800022811D1394603A8D7
:10184000FFF70EFF054665B92068321A0146384693
:10185000FFF7D4FA05462068311A0844206000E0FA
:101860007F4D65B92068B04209D040F24D23AFF2F8
:1018700048226FF065017B4800F0F8FB054615B182
:101880003846FFF700F8284666E72DE9FF4F89B094
:101890000746884691466FF06D040020049005903D
:1018A0000690CDF80C80039800EB0906302307AAB8
:1018B000314603A8F3F73BFE041E0BD040F275231C
:1018C000AFF29C2221466648803800F0CFFB0DB075
:1018D000BDE8F08F07990398461808AA314603A877
:1018E000F3F7B5FE041E09D040F27B23AFF2C82205
:1018F00021465B48803800F0B9FBE8E708980128EA
:1019000001D05948E3E7042307AA314603A8F3F7B7
:101910000EFE041E09D040F28323AFF2F4222146CA
:101920004F48803800F0A2FBD1E703980290DDF821
:101930001CB007990398084403904FF0000A0398DD
:10194000B04225D0A02307AA314603A8F3F7EFFD44
:10195000041E10D1079A0398811804AA03A8FFF760
:1019600018FE041E05D1394604A8FFF779FE041EAF
:101970000ED02046ABE704F1620048B140F29A2352
:10198000AFF25C3221463648803800F06FFB9EE7AC
:101990005A4638460299FFF701FA04460CB1204630
:1019A00095E70398B04249D0A12307AA314603A87E
:1019B000F3F7BDFD041E34D107990398451807AA13
:1019C000294603A8F3F7F8FE041E09D040F2B1231C
:1019D000AFF2AC3221462248803800F047FB76E770
:1019E000079903980844A8420AD040F2B523AFF201
:1019F000C8326FF065011A48803800F037FB66E79F
:101A000003982A1A01463846FFF7F8F9041E02D156
:101A10004FF0010A12E014F59D4F0FD010488038A6
:101A200055E704F1620048B140F2C523AFF2084225
:101A300021460B48803800F019FB48E7BAF1000F47
:101A400014D1169800905A4638460C9B0299FFF71D
:101A5000C0F9041E0AD0204639E7000000C6FFFF87
:101A600080C3FFFF00C5FFFF80C2FFFF00202EE7FD
:101A70002DE9F04F89B004460D4616469946DDF82B
:101A800048A00395039800EB0608002002900190FF
:101A9000302307AA414603A8F3F749FD071E0AD0E1
:101AA00040F20B33AFF280423946F84800F0DEFADC
:101AB00009B0BDE8F08F0799039800EB010808AA68
:101AC000414603A8F3F7C3FD071E08D040F21133C7
:101AD000AFF2AC423946ED4800F0C8FAE8E70898A2
:101AE00048B140F21533AFF2C0423946E74880387A
:101AF00000F0BCFADCE701A804AB02AA4146009062
:101B000003A8FFF7CAFD071E01D03846D0E704231B
:101B100007AA414603A8F3F70AFD071E08D040F2C2
:101B20001D33AFF2FC423946D84800F09FFABFE7B8
:101B3000079848B940F22133AFF214526FF05F01B9
:101B4000D24800F093FAB3E79DF80800FEF7AEFE26
:101B5000B0F1000B02D1CD488030A9E759462046AC
:101B6000FEF7B4FE071E01D03846A1E79DF8080035
:101B700001280FD1D4E9000100F06EFA0090079A15
:101B8000039900F04EFD071E24D02046FEF77BFE91
:101B900038468DE79DF80800022803D09DF808001C
:101BA000032814D1214604A8FFF75AFD071E09D1C6
:101BB0004B46CDF800A02046079A0399FFF765FE33
:101BC000071E07D02046FEF75EFE384670E7AF4896
:101BD00080306DE70799039800EB0108A81940458C
:101BE00009D04FF45473AFF2C0526FF06501A748AB
:101BF00000F03CFA5CE700205AE72DE9F04F89B08D
